:100000000C94420D0C946F0D0C946F0D0C946F0DAD
:100010000C946F0D0C946F0D0C946F0D0C946F0D70
:100020000C946F0D0C946F0D0C946F0D0C946F0D60
:100030000C946F0D0C944AAD0C946F0D0C946F0DD5
:100040000C946F0D0C9467760C946F0D0C946F0DDF
:100050000C946F0D0C946F0D0C94047F0C94C6A936
:100060000C946F0D0C947C250C946F0D0C946F0DFB
:100070000C946F0D0C946F0D0C946F0D0C946F0D10
:100080000C946F0D0C946F0D0C946F0D0C946F0D00
:100090000C946F0D0C946F0D0C946F0D0C944DA679
:1000A0000C946F0D0C946F0D0C946F0D0C946F0DE0
:1000B0000C946F0D0C946F0D0C946F0D0C946F0DD0
:1000C0000C946F0D0C946F0D0C946F0D0C946F0DC0
:1000D0000C946F0D0C946F0D0C946F0D0C946F0DB0
:1000E0000C946F0D084AD73B3BCE016E84BCBFFD1C
:1000F000C12F3D6C74319ABD56833DDA3D00C77FF8
:1001000011BED9E4BB4C3E916BAAAABE0000008090
:100110003F05A84CCDB2D44EB93836A9020C50B91F
:10012000918688083CA6AAAA2ABE000000803F4DFE
:10013000383420582059205A2045006563686F3AAA
:100140000043616E6E6F7420656E74657220737506
:10015000626469723A20004D3234004D32332025FA
:1001600073006175746F25692E67004572726F7236
:100170003A006572726F722077726974696E6720D7
:10018000746F2066696C65004E6F74205344207054
:1001900072696E74696E67002F0053442070726933
:1001A0006E74696E67206279746520002E00446564
:1001B0006C6574696F6E206661696C65642C20469D
:1001C000696C653A200046696C652064656C6574ED
:1001D00065643A002E006F70656E206661696C651B
:1001E000642C2046696C653A200057726974696E08
:1001F0006720746F2066696C653A20002E006F706E
:10020000656E206661696C65642C2046696C653A90
:1002100020002E006F70656E206661696C65642C2D
:100220002046696C653A200046696C652073656CF0
:100230006563746564002053697A653A20004669F5
:100240006C65206F70656E65643A20002E006F70DB
:10025000656E206661696C65642C2046696C653A40
:1002600020004E6F772066726573682066696C6542
:100270003A20004E6F7720646F696E672066696C64
:10028000653A20002220706F730022207061726531
:100290006E743A2200535542524F5554494E4520F0
:1002A00043414C4C207461726765743A2200747249
:1002B00079696E6720746F2063616C6C207375625E
:1002C0002D67636F64652066696C65732077697458
:1002D0006820746F6F206D616E79206C6576656C37
:1002E000732E204D4158206C6576656C2069733AF9
:1002F0000053442063617264206F6B006F70656E01
:10030000526F6F74206661696C656400766F6C75FE
:100310006D652E696E6974206661696C6564005351
:100320004420696E6974206661696C006563686F5A
:100330003A0048617264636F646564204465666175
:10034000756C742053657474696E6773204C6F61AB
:10035000646564002044002049002020204D333093
:10036000312050005049442073657474696E67737E
:100370003A00205A0020590020204D3230362058B3
:1003800000486F6D65206F666673657420286D6D1B
:10039000293A00204500205A002058002042002021
:1003A000540020204D323035205300416476616E78
:1003B000636564207661726961626C65733A20538B
:1003C0003D4D696E20666565647261746520286DB7
:1003D0006D2F73292C20543D4D696E207472617607
:1003E000656C20666565647261746520286D6D2F8B
:1003F00073292C20423D6D696E696D756D207365A2
:10040000676D656E742074696D6520286D73292C85
:1004100020583D6D6178696D756D205859206A6569
:10042000726B20286D6D2F73292C20205A3D6D6131
:1004300078696D756D205A206A65726B20286D6D24
:100440002F73292C2020453D6D6178696D756D20D5
:1004500045206A65726B20286D6D2F73290020542A
:100460000020204D323034205300416363656C65B9
:10047000726174696F6E3A20533D616363656C65A8
:10048000726174696F6E2C20543D72657472616381
:100490007420616363656C65726174696F6E0020BE
:1004A0004500205A0020590020204D32303120587C
:1004B000004D6178696D756D20416363656C65728F
:1004C0006174696F6E20286D6D2F7332293A002098
:1004D0004500205A0020590020204D32303320584A
:1004E000004D6178696D756D206665656472617433
:1004F000657320286D6D2F73293A00204500205A1E
:100500000020590020204D39322058005374657066
:10051000732070657220756E69743A006563686F48
:100520003A004572726F723A0053544F505045442E
:100530002E20005072696E7465722073746F707033
:1005400065642064756520746F206572726F7273C4
:100550002E2046697820746865206572726F72205B
:10056000616E6420757365204D39393920746F20B0
:10057000726573746172742E202854656D70657293
:1005800061747572652069732072657365742E20BD
:100590005365742069742061667465722072657396
:1005A00074617274696E6729004B494C4C45442E46
:1005B00020005072696E7465722068616C746564A5
:1005C0002E206B696C6C28292063616C6C6564213A
:1005D000006F6B00526573656E643A20002200550F
:1005E0006E6B6E6F776E20636F6D6D616E643A2017
:1005F00022007A5F6D61783A20007A5F6D696E3A09
:100600002000795F6D61783A2000795F6D696E3AFC
:100610002000785F6D61783A2000785F6D696E3AEE
:1006200020005A3A00593A0020436F756E742058E2
:100630003A2000453A005A3A00593A00583A0046E2
:1006400049524D574152455F4E414D453A4D6172B9
:100650006C696E2056313B20537072696E746572FE
:100660002F6772626C206D617368757020666F729F
:100670002067656E36204649524D574152455F55B9
:10068000524C3A687474703A2F2F7777772E6D65D5
:100690006E64656C2D70617274732E636F6D205083
:1006A000524F544F434F4C5F56455253494F4E3A69
:1006B000312E30204D414348494E455F54595045F5
:1006C0003A627120576974626F78204558545255C8
:1006D0004445525F434F554E543A310A00627120EF
:1006E000576974626F78204F66662E0062712057DA
:1006F0006974626F782052656164792E0042656486
:1007000020646F6E652E0020423A0020453A005466
:100710003A004265642048656174696E672E00483E
:10072000656174696E6720646F6E652E0020573AAC
:100730000020453A00543A0048656174696E672E9E
:100740002E2E002042403A0020403A00202F003A4E
:1007500000205400202F0020423A00202F006F6B11
:1007600020543A002569206D696E2C20256920737C
:10077000656300456E642066696C65206C697374FE
:1007800000426567696E2066696C65206C697374E8
:10079000004E6F206D6F76652E00526573756D6922
:1007A0006E67207072696E74005761697420666F9D
:1007B0007220757365722E2E2E00536C6565702E37
:1007C0002E2E000080944300005243000048430155
:1007D00001FF00809443000052430000000000002D
:1007E00000000000000000000000008094430000B2
:1007F0005243000048430000A0400000A040000019
:100800000040256920686F757273202569206D6925
:100810006E7574657300446F6E65207072696E74D6
:10082000696E672066696C650053544F50504544AB
:100830002E20005072696E7465722073746F707030
:1008400065642064756520746F206572726F7273C1
:100850002E2046697820746865206572726F722058
:10086000616E6420757365204D39393920746F20AD
:10087000726573746172742E202854656D70657290
:1008800061747572652069732072657365742E20BA
:100890005365742069742061667465722072657393
:1008A00074617274696E6729006F6B004E6F204C23
:1008B000696E65204E756D62657220776974682077
:1008C000636865636B73756D2C204C617374204C89
:1008D000696E653A20004E6F20436865636B7375DF
:1008E0006D2077697468206C696E65206E756D6225
:1008F00065722C204C617374204C696E653A20003F
:10090000636865636B73756D206D69736D61746386
:10091000682C204C617374204C696E653A20004C41
:10092000696E65204E756D626572206973206E6F09
:1009300074204C617374204C696E65204E756D6235
:1009400065722B312C204C617374204C696E653AB2
:1009500020004D31313000446F6E6520736176693F
:100960006E672066696C652E006F6B004D32390032
:100970002020506C616E6E657242756666657242CB
:10098000797465733A20002046726565204D656D67
:100990006F72793A2000466562202036203230316D
:1009A0003400436F6D70696C65643A2000285061B3
:1009B000626C6F20436C656D656E74652C2062718E
:1009C00020576974626F782046572076312E31297E
:1009D00000207C20417574686F723A200046656281
:1009E00020203620323031342031353A30313A351A
:1009F0003300204C61737420557064617465643AEF
:100A00002000312E302E30004D61726C696E200056
:100A100020536F6674776172652052657365740048
:100A2000205761746368646F672052657365740052
:100A30002042726F776E206F7574205265736574F3
:100A4000002045787465726E616C20526573657420
:100A500000506F7765725570007374617274002274
:100A600000656E717565696E672022002200656EF3
:100A7000717565696E672022006563686F3A0020B2
:100A8000746F6F206C6F6E67206578747275736910
:100A90006F6E2070726576656E7465640020636F9A
:100AA0006C6420657874727573696F6E20707265FE
:100AB00076656E746564007C3C3E5E2B3D3F2F5B2B
:100AC0005D3B2C2A225C0045313A200045303A201B
:100AD000005A3A2000593A2000583A20004D53312C
:100AE0002C4D53322050696E730A0024F404D9202F
:100AF0001BC40C5C0E9804C4095F0265077101F405
:100B000005F900FB04B30048048700C103690058DD
:100B100003550003034500BE023A0084023100532E
:100B2000022A002902250004022000E4011C00C85A
:100B3000011900AF0117009801140084011300711E
:100B40000110006101100051010E0043010D00363B
:100B5000010B002B010B0020010B00150109000CFB
:100B600001090003010800FB000800F3000800EB86
:100B7000000700E4000600DE000600D8000600D2F0
:100B8000000600CC000500C7000500C2000500BD3E
:100B9000000400B9000400B5000400B1000400AD79
:100BA000000400A9000400A5000300A20003009FA8
:100BB0000004009B000300980003009500020093CE
:100BC000000300900003008D0002008B00030088EA
:100BD0000002008600020084000300810002007F02
:100BE0000002007D0002007B000200790002007715
:100BF0000001007600020074000200720001007122
:100C00000002006F0002006D0001006C0002006A2B
:100C10000001006900020067000100660001006534
:100C20000001006400020062000100610001006038
:100C30000001005F0002005D0001005C0001005B3C
:100C40000001005A0001005900010058000100573E
:100C5000000100560001005500010054000100533E
:100C6000000000530001005200010051000100503B
:100C70000001004F0001004E0000004E0001004D39
:100C80000001004C0001004B0000004B0001004A35
:100C90000001004900010048000000480001004731
:100CA000000100460000004600010045000000452C
:100CB0000001004400010043000000430001004225
:100CC000000000420001004100000041000100401E
:100CD0000001003F0000003F0001003E0000003E18
:100CE0000001003D0000003D0001003C0000003C10
:100CF0000000003C0001003B0000003B0001003A06
:100D00000000003A000100390000003900010038FD
:100D100000000038000000380001003700000037F4
:100D200000010036000000360000003600010035EA
:100D300000000035000000350001003400000034E0
:100D400000000034000100330000003300000033D5
:100D500000010032000000320000003200010031CA
:100D600000000031000000310001003000000030C0
:100D7000000000300001002F0000002F0000002FB5
:100D80000000002F0001002E0000002E0000002EA9
:100D90000001002D0000002D0000002D0000002D9E
:100DA0000001002C0000002C0000002C0000002C92
:100DB0000001002B0000002B0000002B0000002B86
:100DC0000001002A0000002A0000002A0000002A7A
:100DD000000100290000002900000029000000296E
:100DE0000000002900010028000000280000002861
:100DF0000000002800000028000100270000002754
:100E00000000002700000027000000270001002646
:100E1000000000260000002600000026000000263A
:100E2000000100250000002500000025000000252D
:100E3000000000250000002500010024000000241F
:100E40000000002400000024000000240001002312
:100E50000000002300000023000000230000002306
:100E600000000023000000230001002200000022F7
:100E700000000022000000220000002200000022EA
:100E800000010021000000210000002100000021DD
:100E900000000021000000210000002100010020CE
:100EA00000000020000000200000002000000020C2
:100EB0000000002000000020000000200001001FB2
:100EC0000000001F0000001F0000001F0000001FA6
:100ED0000000001F0000001F0001001E0000001E97
:100EE0000000001E0000001E00000024F4D430505A
:100EF000C38E20C2A24017828B7011127A910D818D
:100F00006CD90AA861E108C7586607615143061EFB
:100F10004B5D05C145A7041A411104093D980371B1
:100F20003931034036DB0265339102D430540280FC
:100F30002E1D02632CEE01752AC501B028A00110F8
:100F40002781018F2564012B244B01E0223401AC61
:100F5000211F018D200D01801FFC00841EED0097D4
:100F60001DDF00B81CD200E61BC600201BBC0064BD
:100F70001AB200B219A8000A19A0006A189900D183
:100F800017910040178B00B516840031167E00B310
:100F90001579003A157300C7146F0058146A00EEF3
:100FA0001366008813630025135E00C7125B006C94
:100FB00012570015125400C111510070114F002139
:100FC000114B00D61049008D104700461044000216
:100FD000104200C00F4000800F3E00420F3C000650
:100FE0000F3B00CB0E3800930E37005C0E35002708
:100FF0000E3400F30D3200C10D3100900D30006051
:101000000D2E00320D2D00050D2C00D90C2B00AE3D
:101010000C2900850C29005C0C2700350C27000EDC
:101020000C2600E80B2400C40B2400A00B23007D39
:101030000B23005A0B2100390B2100180B2000F85C
:101040000A1F00D90A1E00BB0A1E009D0A1D00804F
:101050000A1D00630A1C00470A1B002C0A1B001112
:101060000A1A00F7091A00DD091900C4091900ABB2
:10107000091900920917007B091800630917004C31
:1010800009160036091600200916000A091500F590
:10109000081500E0081400CC081400B8081400A4D7
:1010A000081400900813007D0812006B0813005804
:1010B000081200460812003408110023081100121B
:1010C00008110001081100F0071000E0071000D01F
:1010D000071000C0071000B0070F00A10710009113
:1010E000070E0083070F0074070F0065070E0057F7
:1010F000070E0049070E003B070D002E070E0020CB
:10110000070D0013070D0006070D00F9060C00ED92
:10111000060D00E0060C00D4060C00C8060C00BC4E
:10112000060C00B0060C00A4060B0099060C008DFE
:10113000060B0082060B0077060B006C060B0061A5
:10114000060A0057060B004C060A0042060A003841
:10115000060A002E060A0024060A001A060A0010D3
:1011600006090007060A00FD050900F4050900EB61
:10117000050900E2050900D9050900D0050900C7E5
:10118000050900BE050900B5050800AD050800A564
:101190000509009C050800940508008C05080084DA
:1011A0000508007C050800740508006C050700654B
:1011B0000508005D050700560508004E05070047B5
:1011C0000507004005080038050700310507002A1B
:1011D000050700230507001C050600160507000F7C
:1011E0000507000805060002050700FB040600F5D8
:1011F000040700EE040600E8040600E2040700DB32
:10120000040600D5040600CF040600C9040600C386
:10121000040600BD040600B7040600B1040500ACD6
:10122000040600A6040600A00405009B0406009521
:10123000040500900406008A04050085040500806A
:101240000406007A04050075040500700405006BAF
:1012500004050066040500610405005C04050057F0
:10126000040500520405004D040500480405004330
:101270000405003E0404003A04050035040500306E
:101280000404002C04050027040400230405001EA8
:101290000404001A04040016040500110404000DDF
:1012A000040400090405000404040000040400FC14
:1012B000030400F8030400F4030400F0030400EC4A
:1012C000030400E8030400E4030400E0030400DC7A
:1012D000030400D8030400D4030400D0030400CCAA
:1012E000030400C8030300C50303006563686F3A85
:1012F00000656E6473746F7073206869743A205A65
:1013000000205A3A00656E6473746F7073206869C8
:10131000743A20590020593A00656E6473746F70F6
:1013200073206869743A20580020583A00656E644A
:1013300073746F7073206869743A20004572726F1D
:10134000723A004572723A204D415854454D502032
:101350004245440054656D70657261747572652014
:10136000686561746564206265642073776974637D
:10137000686564206F66662E204D415854454D5077
:101380002074726967676572656420212100457267
:10139000723A204D494E54454D50003A20457874DC
:1013A0007275646572207377697463686564206F11
:1013B00066662E204D494E54454D50207472696723
:1013C00067657265642021004572723A204D41586C
:1013D00054454D50003A204578747275646572200A
:1013E0007377697463686564206F66662E204D416B
:1013F0005854454D50207472696767657265642062
:101400002100202D20496E76616C69642065787416
:101410007275646572206E756D6265722021005070
:101420004944204175746F74756E652066696E69F4
:1014300073686564212050757420746865204B7052
:101440002C204B6920616E64204B6420636F6E73A7
:1014500074616E747320696E746F20436F6E666979
:101460006775726174696F6E2E680050494420413F
:1014700075746F74756E65206661696C6564212092
:1014800074696D656F75740020403A006F6B20546D
:101490003A006F6B20423A00504944204175746F06
:1014A00074756E65206661696C6564212054656D94
:1014B000706572617475726520746F6F20686967FA
:1014C0006800204B643A2000204B693A2000204BF2
:1014D000703A200020436C617369632050494420B6
:1014E000002054753A2000204B753A2000206D6191
:1014F000783A2000206D696E3A200020643A20007E
:1015000020626961733A200070012C01900127016B
:10151000B0012201C0011D01F001180110021301E8
:1015200030020E016002090190020401C002FF00B6
:101530000003FA004003F5008003F000D003EB0045
:101540002004E6007004E100E004DC004005D70060
:10155000C005D2004006CD00D006C8008007C300F9
:101560003008BE00F008B900C009B400B00AAF00EE
:10157000B00BAA00D00CA500000EA000500F9B00DD
:10158000C01096005012910000148C00C015870006
:10159000B0178200B0197D00D01B7800001E7300C8
:1015A00040206E0090226900F024640040275F0014
:1015B00090295A00E02B5500102E500020304B008F
:1015C00010324600E033410090353C0010373700C0
:1015D00070383200A0392D00B03A2800A03B23001B
:1015E000603C1E00103D1900903D1400103E0F009D
:1015F000703E0A00C03E0500003F00002D2D3A2D30
:101600002D002D2D2D0053440020590001200043B2
:101610006F6E74726F6C005370656564004E6F205E
:1016200043617264005072696E742066726F6D203F
:1016300053440053746F70205072696E7400526589
:1016400073756D65205072696E74005061757365B5
:10165000205072696E7400496E666F207363726504
:10166000656E005072656865617400436F6F6C64ED
:101670006F776E004C6576656C20706C61746500E8
:101680004D6F766520417869730046696C616D65C0
:101690006E74004D61696E004A6F67004D3834000A
:1016A00044697361626C6520537465707065727310
:1016B00000473238004175746F20486F6D650043F4
:1016C0006F6E74726F6C004D6F766520302E316DC9
:1016D0006D004D6F766520316D6D004D6F76652024
:1016E00031306D6D004A6F670045787472756465BE
:1016F00072004D6F7665205A004D6F766520590057
:101700004D6F76652058004D6F766520417869737E
:10171000004578747275646572005A00590058006B
:10172000556E6C6F6164004C6F616400436F6E7442
:10173000726F6C004D3730310001200048656174D4
:10174000696E672E2E2E0041626F727400012000B8
:1017500048656174696E672E2E2E0041626F727447
:10176000004D37303000496E73657274202620506A
:10177000726573730041626F7274005370656564C3
:1017800000052E2E004D61696E004D3234004D3241
:1017900033202573004D383420582059205A2045D5
:1017A000004D333030205331353637205033303010
:1017B000004D333030205331313734205031353003
:1017C000004D3330302053302050313530004D3310
:1017D00030302053313137342050333030004731EE
:1017E00020583239382059323038205A32303000BF
:1017F00047393000436172642072656D6F766564AD
:10180000004361726420696E73657274656400766A
:10181000312E3100627120576974626F7800205058
:101820006C617465206C6576656C656421002020B0
:101830002020204973206974206F6B3F20202020D6
:101840002020202020507265737320746F20656EF5
:10185000640041646A7573742074686972642070EE
:101860006F696E7420202026205072657373207477
:10187000686520627574746F6E0041646A75737474
:10188000207365636F6E6420706F696E742020260C
:101890002050726573732074686520627574746F6C
:1018A0006E002041646A75737420666972737420D7
:1018B000706F696E742020262050726573732074D7
:1018C000686520627574746F6E0020204C657665C3
:1018D0006C696E6720706C6174652E2E2E2020203E
:1018E00020507265737320746F207374617274205A
:1018F000202000202020507265737320746F2061B7
:10190000626F72740001200054656D703A00436F7D
:101910006F6C696E672E2E2E004D3630320000003F
:101920002100240027002A002D003000330001018F
:101930000000040107010A01000022002500280020
:101940002B002E00310034000201000005010801C7
:101950000B01000020002300260029002C002F008E
:10196000320000010000030106010901050505051B
:10197000070508080808020202020A0A0808040407
:101980000404010101010101010103030303030335
:101990000303040707070C0C0C0C0C0C0C0C0202C4
:1019A000020206060606060606060B0B0B0B0B0BC1
:1019B0000B0B01021020200808102040102040804E
:1019C0000201020108040201010204081020408003
:1019D0008040201008040201800402018040201091
:1019E00008040201080402010102040810204080DA
:1019F00001020408102040800000090A02080B0CB4
:101A00000D070603040100000000000000000000B4
:101A100000000000000000000000000000000000C6
:101A20000000000011100F00000000000000000086
:101A3000000000000000000000000000000002495B
:101A40004E46494E4954594E414ECDCCCC3D0AD715
:101A5000233C17B7D13877CC2B329595E6241FB1AC
:101A60004F0A000020410000C84200401C4620BC34
:101A7000BE4CCA1B0E5AAEC59D741026BD28AF9C25
:101A8000BCA5B82811241FBECFEFD1E2DEBFCDBF69
:101A900000E00CBF14E0A0E0B2E0E4E0FCE601E00E
:101AA0000BBF02C007900D92A23CB107D9F71BBE35
:101AB00013E1A2ECB4E001C01D92AE31B107E1F731
:101AC0001AE1C2E8DAE104C02297FE010E94A8B53B
:101AD000CA37D107C9F70E94A4AC0C94F6B50C9490
:101AE0000000A0E0B0E0E7E7FDE00C94C5B5EC0134
:101AF0005B016115710519F0FB0191838083F990F9
:101B00008F2D90E00E94ACB5892BC9F7FDE2FF163E
:101B100021F4F990EE24E39405C02BE2F21609F4C7
:101B2000F990EE248E0101501040C8016FE37AE174
:101B300043E050E069D2892BF9F48E010E5F1F4F0C
:101B4000C80162E47AE145E050E05ED2892B19F4E5
:101B50008E01095F1F4FA114B10419F0F501118323
:101B60000083E0FC04C070E090E080E813C070E007
:101B700090E080E86FEF07C1C80167E47AE143E0D5
:101B800050E042D2892B69F4A114B10429F470E029
:101B900090E080EC6FE7F7C02296F501D183C08317
:101BA000F6CF8824992440E050E060E070E0EF2D0B
:101BB000E053EA30A0F5F2E0EF2A8E2D90E09C0190
:101BC00028703070E2FE06C0232B79F50894811C42
:101BD000911C2BC0232B19F0089481089108DB017C
:101BE000CA0112E0880F991FAA1FBB1F1A95D1F7CF
:101BF000480F591F6A1F7B1F440F551F661F771F11
:101C00004E0F511D611D711D483929E9520729E9FF
:101C1000620729E1720748F084E0E82A06C0EE3F37
:101C200031F4E3FC39C098E0E92AF990C0CFE533FC
:101C300011F0E53189F529912D3219F4E0E1EE2A10
:101C400005C02B3219F081E090E003C0299182E0B9
:101C500090E0E22FE053EA3018F0C81BD90B1CC00B
:101C600020E030E0FCE020383F075CF4C901880F39
:101C7000991F880F991F280F391F220F331F2E0F0E
:101C8000311DE991E053EA3068F3E4FE03C030957A
:101C900021953F4F820E931ECE2CDD24E1FE07C01E
:101CA000A114B10421F02197F501D183C083CB01A8
:101CB000BA010E9411B27B018C01F3E0CF22DD2436
:101CC00023E0C216D10421F417FB109517F91095E3
:101CD00057016801C801B70120E030E040E050E062
:101CE0000E9471B1882309F44AC097FE0DC02EE509
:101CF000E22E2AE1F22E9094819491089394C0E20E
:101D0000D0E000E010E012C096E7E92E9AE1F92E4B
:101D1000F6CFF7012591359145915491C601B50152
:101D20000E9451B45B016C018C1A9D0A8C169D06B1
:101D300084F7D595C7950F5F1F4F0630110529F021
:101D40008CEF9FEFE80EF91EF1CFC501D6017C01A3
:101D50008D018C2D880F8D2D881F8F3F51F0C6016E
:101D6000B50120E030E040E050E00E9471B18823EE
:101D700031F482E290E090931D1380931C137E2D2A
:101D80009F2D802F612F272F392F482F562FB901D4
:101D9000CA01CDB7DEB7ECE00C94E1B52F923F92CB
:101DA0005F926F927F928F929F92AF92BF92CF92EB
:101DB000DF92EF92FF920F931F93CF93DF938C01EB
:101DC0001B01EA016115710519F0FB019183808304
:101DD000209749F0CE010297839728F020E030E069
:101DE00040E050E0F6C0F801A1908F018A2D90E00C
:101DF0000E94ACB5892BB9F7FDE2AF1631F4F801BA
:101E0000A1908F015524539407C0FBE2AF1619F43B
:101E1000F801A1908F015524209719F0C031D10508
:101E2000C1F4F0E3AF1679F4F8018081883711F03E
:101E3000883549F4F801A1800E5F1F4FF2E05F2A58
:101E4000C0E1D0E006C0209721F480E3A816E9F4B1
:101E500027C0C830D10531F1C930D10524F4C230D2
:101E6000D10531F50CC0CA30D10589F0C031D1059A
:101E7000F9F4C12CD12CE12CB8E0FB2E28C0C12CE8
:101E8000D12CE12CA0E4FA2E22C0CAE0D0E0FCEC78
:101E9000CF2EFCECDF2EFCECEF2EFCE0FF2E17C06B
:101EA000C8E0D0E0C12CD12CE12CE0E1FE2E0FC027
:101EB0009E01442737FD4095542F60E070E080E09C
:101EC00090E80E9469B5C901DA016C017D0120E04A
:101ED00030E040E050E060E03E01882477FC8094F0
:101EE000982C70EDB72EBA0CE9E0EB1570F48A2D42
:101EF00081548A3118F499ECB92E06C08A2D815686
:101F00008A3150F589EAB82EBA0C8B2D90E08C17E7
:101F10009D0714F56F3FE1F0C216D306E406F506FF
:101F2000B0F0CA01B901A40193010E9423B59B013D
:101F3000AC012B0D311D411D511D2130F0E03F073B
:101F4000F0E04F07F0E85F0710F461E001C06FEFC9
:101F5000F801A1908F01C5CF2114310481F06623CF
:101F600031F001501040F1011183008308C051FE8F
:101F70001AC002501040F1011183008314C067FFA2
:101F800012C050FC05C02FEF3FEF4FEF5FE704C0DA
:101F900020E030E040E050E882E290E090931D13B2
:101FA00080931C1316C050FE08C050954095309584
:101FB00021953F4F4F4F5F4F0CC057FF0AC082E241
:101FC00090E090931D1380931C132FEF3FEF4FEF82
:101FD0005FE7B901CA01DF91CF911F910F91FF9087
:101FE000EF90DF90CF90BF90AF909F908F907F90B9
:101FF0006F905F903F902F900895FB01DC0105905A
:102000000D920020E1F70895FB01DC0141505040A2
:1020100088F08D9181341CF08B350CF4805E6591D5
:1020200061341CF06B350CF4605E861B611171F33A
:10203000990B0895881BFCCFFB01DC0141505040F7
:1020400048F005900D920020C9F701C01D92415043
:102050005040E0F70895FB0155915523A9F0BF01C9
:10206000DC014D9145174111E1F759F4CD0105907F
:10207000002049F04D9140154111C9F3FB01411178
:10208000EFCF81E090E001970895FB01DC0104C0EF
:102090008D910190801921F441505040C8F7881B60
:1020A000990B0895FB01DC0102C001900D92415093
:1020B0005040D8F70895FB01DC010D900020E9F7AE
:1020C000119701900D920020E1F70895FC01819194
:1020D000861721F08823D9F7992708953197CF01E2
:1020E0000895FB01DC0101900D920020E1F70895B5
:1020F000FB01DC014150504030F08D91019080197E
:1021000019F40020B9F7881B990B0895FB01DC0135
:102110004150504048F001900D920020C9F701C095
:102120001D9241505040E0F70895AEE0B0E0EBE979
:10213000F0E10C94CDB50E891F898EE08C831A8353
:1021400009838FEF9FE79E838D839E01265E3F4F1D
:10215000CE010196688D798DA9010AD02F8138852D
:10216000020F131FF80110822E96E4E00C94E9B5DB
:10217000ABE0B0E0EEEBF0E10C94BFB53C012B011D
:102180005A01FC0117821682838181FD03C06FEF23
:102190007FEFB9C19AE0892E1E010894211C311CE1
:1021A000F3012381F20123FD859123FF81912F010A
:1021B000882309F4A5C1853239F423FD859123FFD5
:1021C00081912F01853221F490E0B301B7D1E8CF9E
:1021D000982FFF24EE249924FFE1FF15D0F09B32C5
:1021E00069F09C3228F4903259F0933291F40EC089
:1021F0009D3249F0903369F441E024C052E0F52A61
:1022000084E0F82A28C098E0F92A25C0E0E1FE2AF7
:1022100022C0F7FC29C0892F80538A3070F4F6FE63
:1022200005C0989C902C1124980E15C0E89CE02CB9
:102230001124E80EF0E2FF2A0EC09E3229F4F6FCCB
:102240005FC140E4F42A07C09C3619F450E8F52A2F
:1022500002C0983649F4F20123FD959123FF919134
:102260002F01992309F0B8CF892F8554833018F0B6
:102270008052833038F444E050E0A40EB51E5FE392
:1022800059830FC0933631F0933779F0933509F0C5
:1022900052C01FC0F5018081898342E050E0A40E46
:1022A000B51E610101E010E011C0F501C080D180D0
:1022B000F6FC03C06FEF7FEF02C0692D70E042E0D3
:1022C00050E0A40EB51EC6012ED18C015FE7F522A9
:1022D00013C0F501C080D180F6FC03C06FEF7FEF23
:1022E00002C0692D70E042E050E0A40EB51EC601A8
:1022F0000FD18C0150E8F52AF3FE06C018C080E229
:1023000090E0B3011BD1EA948E2D90E008171907D5
:10231000B0F30DC0F601F7FC8591F7FE81916F01D6
:1023200090E0B3010BD1E110EA9401501040011587
:10233000110581F7E2C0943611F0993661F5F7FE88
:1023400008C0F501208131814281538184E090E011
:102350000AC0F501808191819C01442737FD409599
:10236000542F82E090E0A80EB91E9FE6F92257FF95
:1023700009C050954095309521953F4F4F4F5F4F85
:10238000E0E8FE2ACA01B901A1012AE030E002D149
:10239000D82ED2183FC0953729F41F2D1F7E2AE072
:1023A00030E01DC01F2D197F9F3661F0903720F45B
:1023B000983509F0A5C00FC0903739F0983709F06B
:1023C0009FC004C028E030E00AC0106114FD146012
:1023D00020E130E004C014FD166020E132E017FF78
:1023E00008C0F501608171818281938144E050E0F1
:1023F00008C0F50180819181BC0180E090E042E05D
:1024000050E0A40EB51EA101C5D0D82ED2188FE77A
:10241000F82EF122F6FE0BC05EEFF522D91438F447
:10242000F4FE07C0F2FC05C08FEEF82202C01D2D9D
:1024300001C0192DF4FE0DC0FE01ED0DF11D8081CE
:10244000803319F499EEF92208C01F5FF2FE05C02F
:1024500003C08F2D867809F01F5F0F2DF3FC13C08A
:10246000F0FE0EC01E1510F09D2C0AC09D2C9E0C77
:10247000911A1E2D05C080E290E0B3015FD01F5F6E
:102480001E15C8F304C01E1510F4E11A01C0EE2495
:1024900004FF0EC080E390E0B30150D002FF1BC0E8
:1024A00001FD03C088E790E00EC088E590E00BC016
:1024B000802F867881F001FF02C08BE201C080E2AC
:1024C000F7FC8DE290E0B30139D005C080E390E0E5
:1024D000B30134D09A94D914C8F3DA94F101ED0D14
:1024E000F11D808190E0B30129D0DD20B1F705C056
:1024F00080E290E0B30122D0EA94EE20C9F750CEFA
:10250000F30166817781CB012B96E2E10C94DBB578
:10251000FC010590615070400110D8F780959095AE
:102520008E0F9F1F0895FC016150704001900110B3
:10253000D8F7809590958E0F9F1F08950F931F9346
:10254000CF93DF938C01EB018B8181FF1BC082FF56
:102550000DC02E813F818C819D812817390764F43D
:10256000E881F9810193F983E88306C0E885F9855C
:10257000802F1995892B31F48E819F8101969F833D
:102580008E8302C00FEF1FEFC801DF91CF911F9123
:102590000F910895FA01AA27283051F1203181F1D5
:1025A000E8946F936E7F6E5F7F4F8F4F9F4FAF4F5B
:1025B000B1E03ED0B4E03CD0670F781F891F9A1F6E
:1025C000A11D680F791F8A1F911DA11D6A0F711D22
:1025D000811D911DA11D20D009F468943F912AE02E
:1025E000269F11243019305D3193DEF6CF01089516
:1025F000462F4770405D4193B3E00FD0C9F7F6CF47
:10260000462F4F70405D4A3318F0495D31FD40520E
:10261000419302D0A9F7EACFB4E0A69597958795A4
:1026200077956795BA95C9F7009761057105089583
:102630009B01AC010A2E069457954795379527952F
:10264000BA95C9F7620F731F841F951FA01D0895C7
:10265000FC01128213820895FC018381882311F00A
:1026600081E082830895FC018281811112820895A4
:10267000CF93DF93DC01FC01EB55FE4F808191810C
:102680000097C9F1019791838083ED01CC5ADF4F08
:10269000FD01ED58FF4F8BE1019009928150E1F768
:1026A000FD01EE5AFF4FAF58BF4F8D919C9111978E
:1026B000A157B04091838083FD01ED58FF4F20E08A
:1026C00030E0AD014B555E4F10C02F5F3F4FEF0123
:1026D000DF015F968BE10D9009928150E1F7858DC6
:1026E000968D329791838083B196DA018D919C917A
:1026F0002817390750F3DF91CF910895FC018AE53F
:1027000094E0918380838781882321F0CF01049610
:102710000C9486680895CF92DF92EF92FF920F9308
:102720001F93DF93CF93CDB7DEB76F970FB6F894B3
:10273000DEBF0FBECDBF8C016B01095A1F4FD80100
:102740008C9107551040882321F42FE2E22EF12CC2
:1027500003C090E5E92EF12CE00EF11E8AE594E02D
:102760009A8389831C821B8218861D82B7016C5F45
:102770007F4FCE010596A60121E00E94726F88234B
:1027800091F5EBE3F1E0949108C08091C00085FFE2
:10279000FCCF9093C600319694919923B1F7E1E470
:1027A000F1E0949108C08091C00085FFFCCF909328
:1027B000C600319694919923B1F709C08091C00069
:1027C00085FFFCCF0894C11CD11C9093C600F60174
:1027D0009081992399F78091C00085FFFCCF8AE012
:1027E0008093C6005AC0F801EB55FE4F208131811D
:1027F0002A30310508F040C02F5F3F4F31832083DE
:1028000021503040F90185E0EE0FFF1F8A95E1F776
:10281000E21BF30BED58FF4FE00FF11F13C0AF01A8
:10282000415E5F4FBF018BE1DB010D90BD01DA011D
:102830000D92AD018150C1F7929182913296968F9F
:10284000858F7F9721503040BFEF2E3F3B0739F7F0
:10285000D801AD58BF4FF70134968BE101900D922E
:102860008150E1F70F581F4FF70182819381D80102
:102870008D939C9301571040D801AC5ABF4FFE0175
:1028800035968BE101900D928150E1F70E5A1F4F62
:102890008B819C81F80191838083CE0101962EDF8C
:1028A0006F960FB6F894DEBF0FBECDBFCF91DF910C
:1028B0001F910F91FF90EF90DF90CF900895EF92CE
:1028C000FF920F931F938C013EECE32E31E0F32E29
:1028D000E80EF91EC7010E943968C7010E94866888
:1028E000F801108211821F910F91FF90EF900895CF
:1028F000CF92DF92EF92FF920F931F93CF93DF93CC
:102900007C016B01DB010D900020E9F78D01015086
:102910001040061B170BEEECF1E0EE0EFF1ED70188
:102920001C92E2E3FEEFEE0EFF1ECB016EE470E0C0
:10293000CDDBEC01009731F4F8013197EC0DFD1D72
:1029400086010CC060E270E0C1DB8C010F5F1F4F9D
:10295000CE016AE270E0BADBFC0131978DE0818341
:102960008AE082831382C70186539E4FB8010E947A
:102970006B708EEC91E0E80EF91ED7018C918823E4
:1029800019F1EBE6F1E0949108C08091C00085FF59
:10299000FCCF9093C600319694919923B1F7E2E76A
:1029A000F1E0949108C08091C00085FFFCCF909326
:1029B000C600319694919923B1F78091C00085FFAC
:1029C000FCCF8AE08093C600DF91CF911F910F91D9
:1029D000FF90EF90DF90CF900895CF93DF93EC01BD
:1029E0008B81882309F43BC0EAE9F1E0949108C0A7
:1029F0008091C00085FFFCCF9093C60031969491E2
:102A00009923B1F7CD57DD4F488159816A817B8188
:102A1000C358D24086E495E02AE030E00E94A9261F
:102A2000E8E9F1E0949108C08091C00085FFFCCFF7
:102A30009093C600319694919923B1F7C558DD4F14
:102A4000488159816A817B8186E495E02AE030E003
:102A50000E94A9268091C00085FFFCCF12C0E8E843
:102A6000F1E0949108C08091C00085FFFCCF909365
:102A7000C600319694919923B1F78091C00085FFEB
:102A8000FCCF8AE08093C600DF91CF9108952F920A
:102A90003F924F925F926F927F928F929F92AF92EE
:102AA000BF92CF92DF92EF92FF920F931F93DF932B
:102AB000CF93CDB7DEB7AC970FB6F894DEBF0FBE9D
:102AC000CDBF5C014B01FC018381882309F434C133
:102AD000C50182539E4F0E948668F50112821A8AB0
:102AE0001D8A198A188A8AE594E09F878E875EE49A
:102AF000C52ED12CCA0CDB1C2FE230E0A20EB31E77
:102B0000F601B182A08221ED3FEFA20EB31EF401C7
:102B100080818F3209F08DC0C4016FE270E0D6DA97
:102B20007C010894E11CF11C3E010894611C711C9D
:102B3000260142E1242E312C2C0E3D1E75C0C7010A
:102B40006FE270E0C3DA6C01009709F480C0E81608
:102B5000F90608F07CC08C010E191F09C301B701EA
:102B6000A801D4DA060D171DF8011082F30107C081
:102B70008091C00085FFFCCF31969093C600908174
:102B80009923B1F78091C00085FFFCCFFAE0F09364
:102B9000C600F201608171816115710519F460E070
:102BA00070E002C06C5F7F4FC101A30121E00E9471
:102BB000726F882371F5E6EDF1E0949108C0809181
:102BC000C00085FFFCCF9093C60031969491992365
:102BD000B1F7FE01319607C08091C00085FFFCCFA0
:102BE00031969093C60090819923B1F7E4EDF1E01E
:102BF000949108C08091C00085FFFCCF9093C600DF
:102C0000319694919923B1F78091C00085FFFCCF54
:102C10008DC02EE030E02C0F3D1FF2013183208368
:102C200076010894E11CF11CE114F10409F087CF4E
:102C30000BC080E590E0A80EB91EF601B182A0821B
:102C400020EB3FEFA20EB31ED82C092D02C0DE2CC4
:102C50000F2D8EE490E0A80EB91EF50180819181C0
:102C600022EB3FEFA20EB31E009719F480E090E034
:102C700001C004966D2D702F0E943E70882339F19B
:102C8000E6ECF1E0949108C08091C00085FFFCCF94
:102C90009093C600319694919923B1F78D2D902F82
:102CA0009C01F90107C08091C00085FFFCCF3196DF
:102CB0009093C60090819923B1F783E892E0A80E23
:102CC000B91EF501108211821282138232C0EEEA1F
:102CD000F1E0949108C08091C00085FFFCCF9093F3
:102CE000C600319694919923B1F78D2D902F9C01B8
:102CF000F90107C08091C00085FFFCCF3196909309
:102D0000C60090819923B1F7ECEAF1E0949108C0F4
:102D10008091C00085FFFCCF9093C60031969491BE
:102D20009923B1F78091C00085FFFCCF8AE08093A2
:102D3000C600CE010E96E2DCAC960FB6F894DEBF6C
:102D40000FBECDBFCF91DF911F910F91FF90EF90FC
:102D5000DF90CF90BF90AF909F908F907F906F90BB
:102D60005F904F903F902F900895BF92CF92DF9247
:102D7000EF92FF920F931F93CF93DF938C01EB01A0
:102D80008FE28993EE24E394FF2475EAC72E71E065
:102D9000D72EC00ED11E6FE1B62E14C0FB9CC00111
:102DA00011248D589F4F800F911FBE010E9496687D
:102DB00002C02196E3948881882319F08CE88E154F
:102DC000C0F7F3942F2D30E0F60180819181281710
:102DD000390720F3E7FC07C0C80182539E4FBE01AC
:102DE0000E94966801C01882DF91CF911F910F91C8
:102DF000FF90EF90DF90CF90BF9008952F923F9279
:102E00004F925F926F927F928F929F92AF92BF92FA
:102E1000CF92DF92EF92FF920F931F93DF93CF93A6
:102E2000CDB7DEB7AD970FB6F894DEBF0FBECDBFFE
:102E30006C014B014DA7DC0113968C91882309F49A
:102E400048C3E1EDF1E0CE0EDF1ED6018C91EFE23A
:102E5000FEEFCE0EDF1E882309F418C1222309F0ED
:102E6000E0C029EE31E0C20ED31ED6018C91E7E11D
:102E7000FEEFCE0EDF1E882371F1EBE6F1E09491B8
:102E800008C08091C00085FFFCCF9093C6003196AA
:102E900094919923B1F7EEEAF2E0949108C0809101
:102EA000C00085FFFCCF9093C60031969491992382
:102EB000B1F786E495E061E070E04AE050E00E94FE
:102EC000F8268091C00085FFFCCF8AE08093C60081
:102ED0000E940A29FEC2EBE3F1E0949108C08091C0
:102EE000C00085FFFCCF9093C60031969491992342
:102EF000B1F7E5E9F2E0949108C08091C00085FF48
:102F0000FCCF9093C600319694919923B1F7F401C8
:102F100007C08091C00085FFFCCF31969093C6001A
:102F200090819923B1F7EAE8F2E0949108C080918A
:102F3000C00085FFFCCF9093C600319694919923F1
:102F4000B1F7C6012EEE31E0C20ED31EB6010DDF81
:102F50004BEF5FEFC40ED51ED6019C91E7E1FEEF6B
:102F6000CE0EDF1E8DE8989FF0011124E251FE4F36
:102F7000EC0DFD1D07C08091C00085FFFCCF319690
:102F80009093C60090819923B1F7E4E8F2E0949120
:102F900008C08091C00085FFFCCF9093C600319699
:102FA00094919923B1F723E832E0C20ED31ED601E3
:102FB0004D915D916D917C91EDE7FDEFCE0EDF1EA1
:102FC00086E495E02AE030E00E94A9268091C000C6
:102FD00085FFFCCF8AE08093C600A60147515E4F73
:102FE000DA012C91E22FF0E0EE0FFF1FEE0FFF1F32
:102FF000EC0DFD1DE651FE4F83E892E0C80ED91E90
:10300000D6014D905D906D907C908DE79DEFC80E40
:10301000D91E40825182628273822F5FDA012C9323
:103020002FC0EBE3F1E0949108C08091C00085FFD0
:10303000FCCF9093C600319694919923B1F7E3E7C2
:10304000F2E0949108C08091C00085FFFCCF90937E
:10305000C600319694919923B1F7F40107C080918D
:10306000C00085FFFCCF31969093C60090819923D4
:10307000B1F78091C00085FFFCCF8AE08093C60045
:10308000C60182539E4F0E94866839C0E9EEF1E086
:10309000CE0EDF1ED6011C92E7E1FEEFCE0EDF1E44
:1030A000EBE3F1E0949108C08091C00085FFFCCF74
:1030B0009093C600319694919923B1F7E2E6F2E03D
:1030C000949108C08091C00085FFFCCF9093C6000A
:1030D000319694919923B1F7F40107C08091C00013
:1030E00085FFFCCF31969093C60090819923B1F76C
:1030F0008091C00085FFFCCF8AE08093C600D60196
:1031000012961C921A8A1D8A198A188A8AE594E0F6
:103110009F878E87FEE4AF2EB12CAC0CBD1CEFE276
:10312000F0E0CE0EDF1ED501CD92DC92E1EDFFEF97
:10313000CE0EDF1ED4018C918F3209F090C0C401F5
:103140006FE270E00E9466107C010894E11CF11CA3
:103150003E010894611C711C2501E2E12E2E312CE8
:103160002C0E3D1E77C0C7016FE270E00E94661012
:103170005C01009709F481C0E816F90608F07DC0EB
:103180008C010E191F09C301B701A8010E94861006
:10319000060D171DF8011082F30107C08091C000D1
:1031A00085FFFCCF31969093C60090819923B1F7AB
:1031B0008091C00085FFFCCFFAE0F093C600D201F9
:1031C0006D917C916115710519F460E070E002C0A9
:1031D0006C5F7F4FC101A30121E00E94726F8823C1
:1031E00071F5EEE4F2E0949108C08091C00085FF93
:1031F000FCCF9093C600319694919923B1F7FE01CC
:10320000319607C08091C00085FFFCCF3196909326
:10321000C60090819923B1F7ECE4F2E0949108C0E4
:103220008091C00085FFFCCF9093C60031969491A9
:103230009923B1F78091C00085FFFCCF1BC12EE020
:1032400030E02C0F3D1FF20131832083750108947B
:10325000E11CF11CE114F10409F085CF0BC040E53D
:1032600050E0C40ED51ED501CD92DC92E0EBFFEF0D
:10327000CE0EDF1E082DF92C01C00E2DF601E25BEB
:10328000FF4F2DA5222309F4B1C060817181611522
:10329000710519F460E070E002C06C5F7F4FC601F9
:1032A00082539E4F402F5F2D21E00E94726F882332
:1032B00009F46CC04FED51E0C40ED51ED6014D91FE
:1032C0005D916D917C91ECE9F0E0CE0EDF1ED601B0
:1032D0004D935D936D937C931397E5E8FDEFCE0ED0
:1032E000DF1EEEE3F2E0949108C08091C00085FFFC
:1032F000FCCF9093C600319694919923B1F7802F1B
:103300009F2D9C01F90107C08091C00085FFFCCF73
:1033100031969093C60090819923B1F7E6E3F2E0ED
:10332000949108C08091C00085FFFCCF9093C600A7
:10333000319694919923B1F786E495E02AE030E044
:103340000E94A9268091C00085FFFCCF8AE080936F
:10335000C60023E832E0C20ED31ED6011D921D9294
:103360001D921C921397E8E2F2E0949108C08091BC
:10337000C00085FFFCCF9093C600319694919923AD
:10338000B1F78091C00085FFFCCF99C0E4E1F2E085
:10339000949108C08091C00085FFFCCF9093C60037
:1033A000319694919923B1F7802F9F2D9C01F901BB
:1033B00007C08091C00085FFFCCF31969093C60076
:1033C00090819923B1F7E2E1F2E0949108C08091F5
:1033D000C00085FFFCCF9093C6003196949199234D
:1033E000B1F78091C00085FFFCCF44C0608171813E
:1033F0006115710519F460E070E002C06C5F7F4FE9
:10340000C60182539E4F402F5F2D26E50E94726FAA
:10341000882309F033C0EEEFF1E0949108C0809169
:10342000C00085FFFCCF9093C600319694919923FC
:10343000B1F7802F9F2D9C01F90107C08091C0003A
:1034400085FFFCCF31969093C60090819923B1F708
:10345000ECEFF1E0949108C08091C00085FFFCCFB3
:103460009093C600319694919923B1F78091C00052
:1034700085FFFCCF8AE08093C60028C081E0F6017A
:103480008083EAEEF1E0949108C08091C00085FF4E
:10349000FCCF9093C600319694919923B1F7F40133
:1034A00007C08091C00085FFFCCF31969093C60085
:1034B00090819923B1F78091C00085FFFCCF8AE00D
:1034C0008093C600802F9F2D0E94E49CCE010E9613
:1034D00015D9AD960FB6F894DEBF0FBECDBFCF9114
:1034E000DF911F910F91FF90EF90DF90CF90BF90F1
:1034F000AF909F908F907F906F905F904F903F9094
:103500002F900895EF92FF920F931F93CF93DF9325
:10351000EC010E944C768E0107511E4FD8018C9110
:103520009EECE92E91E0F92EEC0EFD1E882399F118
:10353000C7010E948668F8016081615060838DE850
:10354000689FB001112462517E4F6C0F7D1FCE0128
:1035500041E021E053DCD801EC91F0E0EE0FFF1FD9
:10356000EE0FFF1FEC0FFD1FE651FE4F4081518112
:1035700062817381CD57DD4F488359836A837B8392
:10358000C358D240C7010E946F678B81882389F19D
:1035900081E08A832EC00E942976C7010E94866836
:1035A0001A828FE291E00E94194D80914B0A882384
:1035B00001F110924B0A80910308C82FD0E0CC0F84
:1035C000DD1FC257DE4E68817981882777FD80959F
:1035D000982F0E9413B22091AB033091AC0340911D
:1035E000AD035091AE030E947FB3181614F41982F4
:1035F0001882DF91CF911F910F91FF90EF90089566
:10360000FC0181E08183CF0140E021E0F7CBEF9224
:10361000FF920F931F93CF93DF938C01FC011382D2
:1036200086A9882321F0C801C3960E94866827EAEC
:10363000E22E21E0F22EE00EF11EC70160E045E32C
:103640000E943566882309F5EBE3F1E0949108C008
:103650008091C00085FFFCCF9093C6003196949175
:103660009923B1F7EFE1F3E0949108C08091C00095
:1036700085FFFCCF9093C600319694919923B1F7C2
:103680008091C00085FFFCCF7DC0E801C455DE4FAE
:10369000CE01B70141E00E94FC70882341F5CE01C4
:1036A000B70140E00E94FC70882309F5EBE6F1E0E9
:1036B000949108C08091C00085FFFCCF9093C60014
:1036C000319694919923B1F7ECE0F3E0949108C01E
:1036D0008091C00085FFFCCF9093C60031969491F5
:1036E0009923B1F78091C00085FFFCCF4BC0C80182
:1036F000C396BE010E94786B882309F5EBE6F1E0E2
:10370000949108C08091C00085FFFCCF9093C600C3
:10371000319694919923B1F7ECEFF2E0949108C0BF
:103720008091C00085FFFCCF9093C60031969491A4
:103730009923B1F78091C00085FFFCCF23C081E0C1
:10374000F8018383EBE3F1E0949108C08091C0001D
:1037500085FFFCCF9093C600319694919923B1F7E1
:10376000E1EFF2E0949108C08091C00085FFFCCFAA
:103770009093C600319694919923B1F78091C0003F
:1037800085FFFCCF8AE08093C600D801AC5ABF4FBA
:10379000F801F3968BE101900D928150E1F7F80169
:1037A00081A992A90E5A1F4FF80191838083025577
:1037B0001040C8018F96025B1F4FF80191838083F0
:1037C000DF91CF911F910F91FF90EF9008952F926D
:1037D0003F924F925F926F927F929F92AF92BF9271
:1037E000CF92DF92EF92FF920F931F93DF93CF93CD
:1037F000CDB7DEB7CC55D0400FB6F894DEBF0FBEC4
:10380000CDBF6C01662311F527E832E0C20ED31E4E
:10381000D6018C91E9E7FDEFCE0EDF1E882309F477
:10382000E3C02FE732E0C20ED31ED601ED90FD902B
:103830000D911C91E1E8FDEFCE0EDF1E0E940EAA55
:10384000E616F7060807190708F4CEC027E832E0A5
:10385000C20ED31ED6011C92E9E7FDEFCE0EDF1E8D
:10386000D60113968C91882339F4C601D0DEF60177
:103870008381882309F4B8C000D000D0EDB7FEB72B
:1038800031967E010894E11CF11CADB7BEB71296CB
:10389000FC92EE92119782E691E093838283D601A7
:1038A0009D968D919C919E97958384830E949510FF
:1038B0008701EDB7FEB736960FB6F894FEBF0FBE80
:1038C000EDBF57010AC0D8018C91992787FD9095CB
:1038D0000E94B4B5F80181938F01F5010190002099
:1038E000E9F73197EA19FB09802F8E198E175CF3DF
:1038F00063E3A62EB12CAC0CBD1CC50140E050E02A
:1039000060E070E00E946F6799245DE3E52EF12C82
:10391000EC0EFD1E2E010894411C511C4FE1642E3B
:10392000712C6C0E7D1E3BE5232E31E0332E42C000
:10393000D8018C9190E00E94B4B5F80181938F0179
:10394000D7010D900020E9F71197AE19BF09802F1C
:103950008E198A176CF327968FAD27978E3751F102
:10396000C701B20145E050E00E947810009711F5C0
:1039700000D000D0EDB7FEB73196ADB7BEB7129606
:103980007C926E92119733822282558244820E94E9
:103990009510EDB7FEB736960FB6F894FEBF0FBE82
:1039A000EDBFC3010E94924D87E591E00E94194D41
:1039B00099249394C501B70140E050E00E94976AB2
:1039C000181614F48701BCCF992041F48FEF9FEFB4
:1039D000D6019E969C938E939D9706C0F60185A571
:1039E00096A5019696A785A7C45ADF4F0FB6F894FF
:1039F000DEBF0FBECDBFCF91DF911F910F91FF9022
:103A0000EF90DF90CF90BF90AF909F907F906F909E
:103A10005F904F903F902F9008952F923F924F923A
:103A20005F926F927F928F929F92AF92BF92CF924E
:103A3000DF92EF92FF920F931F93DF93CF93CDB757
:103A4000DEB7CF58D0400FB6F894DEBF0FBECDBF63
:103A50008C013B016A0184E090E0C80ED91EF80198
:103A60007196C757DF4FF983E883C958D040C80122
:103A70000496CA57DF4F99838883C658D040C857E9
:103A8000DF4F1882C858D040B6E6EB2EF12CEC0E72
:103A9000FD1EF7013B96C557DF4FF983E883CB58EE
:103AA000D040A8E88A2EA2E09A2E800E911EFAE855
:103AB000AF2EF2E0BF2EA00EB11EEEE02E2E312C66
:103AC0002C0E3D1E77E4472E512C4C0E5D1EC2017C
:103AD0000496C357DF4F99838883CD58D040EBE3DA
:103AE000F1E09491C157DF4F9883CF58D0404EC139
:103AF000F7018385482F50E0BA016871707060311A
:103B0000710509F051C1F401208131812130310565
:103B100009F44AC12230310509F446C1F701DE013A
:103B200011969081903239F08E2F8E19883011F4D1
:103B30008EE28D939D933196C557DF4F8881998191
:103B4000CB58D040E817F90761F71C921E86F301A5
:103B50008081882329F4C10160E072E00E945B103B
:103B6000C101B3010E945B10C101BE016F5F7F4FB5
:103B70000E945B10C10160E072E00E945B101CA615
:103B80001FA61BA61AA68AE594E099A788A7CE01CE
:103B90008C96B601AE014F5F5F4F21E00E94726FBD
:103BA000882309F03FC0F40180819181892BD1F5F0
:103BB000C157DF4F9881CF58D040EBE3F1E008C008
:103BC0008091C00085FFFCCF9093C6003196949100
:103BD0009923B1F7E2E0F2E007C08091C00085FFD1
:103BE000FCCF31969093C60090819923B1F78091D4
:103BF000C00085FFFCCFFAE0F093C600FE013196CD
:103C000007C08091C00085FFFCCF31969093C6001D
:103C100090819923B1F78091C00085FFFCCF8AE0A5
:103C20008093C600C357DF4FA881B981CD58D040DB
:103C3000FE01BC968BE101900D928150E1F78AA5BF
:103C40009BA5F201938382838AE594E0918380832C
:103C5000C801B101A201E1DEC2010E947E13CE01C2
:103C600088960E947E1392C0953E09F48FC09E32C2
:103C700009F48CC09F3509F489C0F8019189992312
:103C800031F09E3209F482C09F3509F47FC043FDB4
:103C90007DC080E06031710509F481E0F80184A7FE
:103CA000882349F4F7018085873409F06FC0818546
:103CB0008E3709F46BC0CA57DF4FA881B981C65847
:103CC000D040F7018081803241F08E2F8E198830EC
:103CD00011F48EE28D9380818D933196C557DF4F1D
:103CE00088819981CB58D040E817F90759F71C9281
:103CF000F40180819181009729F5F30107C080913B
:103D0000C00085FFFCCF31969093C6009081992327
:103D1000B1F7CA57DF4FE881F981C658D04007C0D4
:103D20008091C00085FFFCCF31969093C6009081B2
:103D30009923B1F78091C00085FFFCCFFAE0F093A2
:103D4000C60024C08130910539F4F501808191814C
:103D50000196918380831AC00297C1F4C857DF4F40
:103D6000F881C858D0402F2F30E0F5018081918133
:103D700028173907F1F0C857DF4FF881C858D040ED
:103D8000FF5FC857DF4FF883C858D040C601B7015E
:103D9000C757DF4F48815981C958D0400E94976A60
:103DA00018160CF4A5CE05C0F7019081992309F0EF
:103DB0005BCFC157DF4F0FB6F894DEBF0FBECDBF4C
:103DC000CF91DF911F910F91FF90EF90DF90CF90F7
:103DD000BF90AF909F908F907F906F905F904F902B
:103DE0003F902F900895EF92FF920F931F93DF93D0
:103DF000CF93CDB7DEB76F970FB6F894DEBF0FBE87
:103E0000CDBF7C018C01025B1F4F805B9F4FF8018F
:103E10009183808328E832E0E20EF31E21E030E057
:103E2000F701219331937F011182108226E73DEF44
:103E3000E20EF31E049640E050E060E070E00E9465
:103E40006F67F80120813181DE011596F901349602
:103E50008BE101900D928150E1F7F901828193810C
:103E60009C838B838AE594E09A838983C70165E10B
:103E700072E08E010F5F1F4FA801CFDDC8010E94C5
:103E80007E13F701E657FD4F808191816F960FB643
:103E9000F894DEBF0FBECDBFCF91DF911F910F9180
:103EA000FF90EF900895EF92FF920F931F93DF938F
:103EB000CF93CDB7DEB76F970FB6F894DEBF0FBEC6
:103EC000CDBF7C018C01025B1F4F805B9F4FF801CF
:103ED0009183808328E832E0E20EF31E22E030E096
:103EE000F7013183208328E73DEFE20EF31EF7014F
:103EF000E657FD4F60831182049640E050E060E099
:103F000070E00E946F67F80120813181DE01159613
:103F1000F90134968BE101900D928150E1F7F9019E
:103F2000828193819C838B838AE594E09A83898341
:103F3000C70165E172E08E010F5F1F4FA8016DDDC3
:103F4000C8010E947E136F960FB6F894DEBF0FBEB5
:103F5000CDBFCF91DF911F910F91FF90EF9008950A
:103F6000EF92FF920F931F93DF93CF93CDB7DEB7FE
:103F70006F970FB6F894DEBF0FBECDBF7C0188E807
:103F800092E0E80EF91EF7011182108288E79DEF9A
:103F9000E80EF91E87010D5C1F4FC80140E050E09C
:103FA00060E070E00E946F67DE011596F8018BE11A
:103FB00001900D928150E1F7F70181A992A99C83AC
:103FC0008B838AE594E09A838983C70165E172E077
:103FD0008E010F5F1F4FA80120DDC8010E947E13D4
:103FE0006F960FB6F894DEBF0FBECDBFCF91DF91B5
:103FF0001F910F91FF90EF9008950F931F93CF9310
:10400000DF93DC01D3961C92D397D6961C92D69759
:10401000D2961C921E92D1978AE594E0D0969C93FA
:104020008E939F97AC5ABF4F1C9213961C92A75524
:10403000B040FD01E05BFF4FAE5ABF4F11961C929E
:104040001E92A255B04091838083ED01C159DF4F8C
:10405000FE0120E030E0482F148217821382128282
:1040600040839183215E3F4F7F9681E0263338075E
:1040700099F7A855BE4F89E18C9313961C925896D8
:104080001C921B961C9213961C92A15DB140FD01DF
:10409000E653FE4FA453BE4F11961C921E924083CE
:1040A0009183A155BF4F1D921D921D921C92139793
:1040B00018961D921D921D921C921397A358B24000
:1040C00012961C92129713961C9213971C9211969B
:1040D0001C9211978D0101581D4FF8011082118219
:1040E00012821382AB55BE4F11961C921E92AC5B8E
:1040F000BF4F1C92FE01C90111920197E9F7A25628
:10410000BF4F81E08C93A758B2409E961C921E929E
:104110009D970E940EAA68577C4E8F4F9F4FF801C3
:104120006083718382839383DF91CF911F910F917D
:104130000895DF93CF93CDB7DEB7E0970FB6F8942D
:10414000DEBF0FBECDBFDE011196EAE0F4E080E1F4
:1041500001900D928150E1F7DE015196EAEFF3E014
:1041600080E101900D928150E1F7DE019196EAEE37
:10417000F3E080E101900D928150E1F789819A810D
:10418000AB81BC818093EF099093F009A093F10972
:10419000B093F20989899A89AB89BC898093DF0938
:1041A0009093E009A093E109B093E20989A19AA153
:1041B000ABA1BCA18093FF099093000AA093010AD0
:1041C000B093020A8D819E81AF81B8858093F309F7
:1041D0009093F409A093F509B093F6098D899E890F
:1041E000AF89B88D8093E3099093E409A093E50922
:1041F000B093E6098DA19EA1AFA1B8A58093030A53
:104200009093040AA093050AB093060A89859A85BB
:10421000AB85BC858093F7099093F809A093F909C1
:10422000B093FA09898D9A8DAB8DBC8D8093E70987
:104230009093E809A093E909B093EA0989A59AA5A2
:10424000ABA5BCA58093070A9093080AA093090A1E
:10425000B0930A0A8D859E85AF85B8898093FB0946
:104260009093FC09A093FD09B093FE098D8D9E8D5E
:10427000AF8DB8A18093EB099093EC09A093ED0961
:10428000B093EE098DA59EA5AFA5B8A980930B0AA2
:1042900090930C0AA0930D0AB0930E0A0E94B65296
:1042A00080E090E8ABE3B5E48093130A9093140A9E
:1042B000A093150AB093160A80E090E4ACE9B5E447
:1042C0008093170A9093180AA093190AB0931A0AB8
:1042D00020E030E040E050E020930F0A3093100AD5
:1042E0004093110A5093120A80E29EE4A0E0B0E0ED
:1042F0008093DB099093DC09A093DD09B093DE097C
:104300002093270A3093280A4093290A50932A0AB7
:1043100080E090E0A0EAB1E480931B0A90931C0A2D
:10432000A0931D0AB0931E0A8DEC9CECACECBEE38E
:1043300080931F0A9093200AA093210AB093220A27
:1043400080E090E0A0EAB0E48093230A9093240AEE
:10435000A093250AB093260A2093F3073093F4071D
:104360004093F5075093F6072093EF073093F0073B
:104370004093F1075093F2072093EB073093EC073B
:104380004093ED075093EE0788EC90E09093E01196
:104390008093DF111092E2111092E1112FEF30E0C3
:1043A0003093E4112093E3118CED90E09093E611AB
:1043B0008093E51184E690E09093E8118093E711F3
:1043C0003093EA112093E9118AE097EDA7E4B1E474
:1043D0008093BC039093BD03A093BE03B093BF032F
:1043E00062E578EB8EE19FE30E94687E6093C003F4
:1043F0007093C1038093C2039093C30364EA70E790
:104400008AE792E40E94747E6093C4037093C503AC
:104410008093C6039093C7030E94297E80E090E0BA
:10442000A0E8BFE38093C8039093C903A093CA0395
:10443000B093CB03ECE2F3E0949108C08091C0000C
:1044400085FFFCCF9093C600319694919923B1F7E4
:10445000E2E3F3E0949108C08091C00085FFFCCFB7
:104460009093C600319694919923B1F78091C00042
:1044700085FFFCCF8AE08093C600E0960FB6F894E3
:10448000DEBF0FBECDBFCF91DF910895CF93DF93F5
:10449000CCE2D3E0FE01949108C08091C00085FF7A
:1044A000FCCF9093C600319694919923B1F7ECE03C
:1044B000F5E0949108C08091C00085FFFCCF9093F7
:1044C000C600319694919923B1F78091C00085FF81
:1044D000FCCF8AE08093C600FE019491ECE2F3E009
:1044E00008C08091C00085FFFCCF9093C600319634
:1044F00094919923B1F74091EF095091F00960919F
:10450000F1097091F20984E095E00E94902D4091AC
:10451000F3095091F4096091F5097091F60981E071
:1045200095E00E94902D4091F7095091F809609113
:10453000F9097091FA098EEF94E00E94902D409154
:10454000FB095091FC096091FD097091FE098BEF08
:1045500094E00E94902DE6E1F2E007C08091C00057
:1045600085FFFCCF31969093C60090819923B1F7D7
:104570008091C00085FFFCCF8AE08093C600FE01D9
:104580009491ECE2F3E008C08091C00085FFFCCF7D
:104590009093C600319694919923B1F7E1EEF4E03F
:1045A000949108C08091C00085FFFCCF9093C60015
:1045B000319694919923B1F78091C00085FFFCCF8B
:1045C0008AE08093C600FE019491ECE2F3E008C01B
:1045D0008091C00085FFFCCF9093C60031969491E6
:1045E0009923B1F74091DF095091E0096091E10909
:1045F0007091E20988ED94E00E94902D4091E309CA
:104600005091E4096091E5097091E60985ED94E027
:104610000E94902D4091E7095091E8096091E909C5
:104620007091EA0982ED94E00E94902D4091EB098F
:104630005091EC096091ED097091EE098FEC94E0D6
:104640000E94902DE6E1F2E007C08091C00085FF56
:10465000FCCF31969093C60090819923B1F7809159
:10466000C00085FFFCCF8AE08093C600FE019491D4
:10467000ECE2F3E008C08091C00085FFFCCF90938E
:10468000C600319694919923B1F7E1EBF4E094914F
:1046900008C08091C00085FFFCCF9093C600319682
:1046A00094919923B1F78091C00085FFFCCF8AE0F7
:1046B0008093C600FE019491ECE2F3E008C0809183
:1046C000C00085FFFCCF9093C6003196949199234A
:1046D000B1F74091FF095091000A6091010A709171
:1046E000020A88EA94E00E94A22D4091030A5091A8
:1046F000040A6091050A7091060A85EA94E00E9416
:10470000A22D4091070A5091080A6091090A709100
:104710000A0A82EA94E00E94A22D40910B0A50916D
:104720000C0A60910D0A70910E0A8FE994E00E94C4
:10473000A22DE6E1F2E007C08091C00085FFFCCF2A
:1047400031969093C60090819923B1F78091C00073
:1047500085FFFCCF8AE08093C600FE019491ECE2D5
:10476000F3E008C08091C00085FFFCCF9093C600A5
:10477000319694919923B1F7EAE6F4E0949108C058
:104780008091C00085FFFCCF9093C6003196949134
:104790009923B1F78091C00085FFFCCF8AE0809318
:1047A000C600FE019491ECE2F3E008C08091C000E5
:1047B00085FFFCCF9093C600319694919923B1F771
:1047C0004091130A5091140A6091150A7091160ACB
:1047D00081E694E00E94902D4091170A5091180AAA
:1047E0006091190A70911A0A8EE594E00E94902D4A
:1047F000E6E1F2E007C08091C00085FFFCCF319672
:104800009093C60090819923B1F78091C00085FFF5
:10481000FCCF8AE08093C600FE019491ECE2F3E0C5
:1048200008C08091C00085FFFCCF9093C6003196F0
:1048300094919923B1F7EBEAF3E0949108C0809149
:10484000C00085FFFCCF9093C600319694919923C8
:10485000B1F78091C00085FFFCCF8AE08093C6004D
:10486000FE019491ECE2F3E008C08091C00085FF66
:10487000FCCF9093C600319694919923B1F7409163
:104880000F0A5091100A6091110A7091120A82EA7F
:1048900093E00E94902D4091270A5091280A609140
:1048A000290A70912A0A8FE993E00E94902D409185
:1048B000DB095091DC096091DD097091DE098CE91A
:1048C00093E00E94A22D40911B0A50911C0A609116
:1048D0001D0A70911E0A89E993E00E94902D409173
:1048E0001F0A5091200A6091210A7091220A86E9DC
:1048F00093E00E94902D4091230A5091240A6091E8
:10490000250A7091260A83E993E00E94902DE6E142
:10491000F2E007C08091C00085FFFCCF31969093F4
:10492000C60090819923B1F78091C00085FFFCCF2C
:104930008AE08093C600FE019491ECE2F3E008C0A7
:104940008091C00085FFFCCF9093C6003196949172
:104950009923B1F7E1E8F3E0949108C08091C00099
:1049600085FFFCCF9093C600319694919923B1F7BF
:104970008091C00085FFFCCF8AE08093C600FE01D5
:104980009491ECE2F3E008C08091C00085FFFCCF79
:104990009093C600319694919923B1F74091EB071B
:1049A0005091EC076091ED077091EE0788E793E076
:1049B0000E94902D4091EF075091F0076091F10710
:1049C0007091F20785E793E00E94902D4091F307E4
:1049D0005091F4076091F5077091F60782E793E034
:1049E0000E94902DE6E1F2E007C08091C00085FFB3
:1049F000FCCF31969093C60090819923B1F78091B6
:104A0000C00085FFFCCF8AE08093C600FE01949130
:104A1000ECE2F3E008C08091C00085FFFCCF9093EA
:104A2000C600319694919923B1F7E4E6F3E09491AE
:104A300008C08091C00085FFFCCF9093C6003196DE
:104A400094919923B1F78091C00085FFFCCF8AE053
:104A50008093C600FE019491ECE2F3E008C08091DF
:104A6000C00085FFFCCF9093C600319694919923A6
:104A7000B1F74091BC035091BD036091BE037091AA
:104A8000BF038AE593E00E94902D6091C00370916E
:104A9000C1038091C2039091C3030E946E7EAB015B
:104AA000BC0187E593E00E94902D6091C403709152
:104AB000C5038091C6039091C7030E947A7EAB0123
:104AC000BC0184E593E00E94902DE6E1F2E007C08E
:104AD0008091C00085FFFCCF31969093C6009081F5
:104AE0009923B1F78091C00085FFFCCF8AE08093C5
:104AF000C600DF91CF9108951F920F920FB60F92CB
:104B00000BB60F9211242F933F934F938F939F9344
:104B1000EF93FF934091C600E0914205F091430569
:104B200031969F012F773070319780914405909195
:104B300045052817390739F0EE53FB4F4083309372
:104B4000430520934205FF91EF919F918F914F91E3
:104B50003F912F910F900BBE0F900FBE0F901F90A3
:104B600018959A01AB01203081EE380780E04807A4
:104B700080E0580749F182E08093C00060E079E06E
:104B80008DE390E00E948BB5215030404040504072
:104B9000CA01B90122E030E040E050E00E948BB54C
:104BA0003093C5002093C4008091C1008061809340
:104BB000C1008091C10088608093C1008091C100D4
:104BC00080688093C10008951092C00020E130E019
:104BD000E7CF2091440530914505809142059091A1
:104BE00043058217930719F42FEF3FEF0EC0F90129
:104BF000EE53FB4F80812F5F3F4F2F773070309304
:104C0000450520934405282F30E0C901089580917F
:104C1000440590914505909343058093420508957E
:104C200008952F923F924F925F926F927F928F9250
:104C30009F92AF92BF92CF92DF92EF92FF920F932B
:104C40001F93DF93CF93CDB7DEB7A0970FB6F8943D
:104C5000DEBF0FBECDBF1C016A017B0141155105AE
:104C60006105710541F440E350E060E070E020E050
:104C700030E08BD055C0882499245401422E55240D
:104C80006624772401E010E00C0F1D1F080D191D8C
:104C9000C701B601A30192010E9469B5F8016083C2
:104CA0000894811C911CA11CB11CC701B601A30171
:104CB00092010E9469B5C901DA016C017D01C1143C
:104CC000D104E104F104F1F681E0E82EF12CEC0EC0
:104CD000FD1EE80CF91C3E010894611C711CD501F5
:104CE000C4010197A109B1096C01C818D90815C000
:104CF000F601EE0DFF1D40814A3010F4405D01C009
:104D0000495C552747FD5095652F752FC10120E05F
:104D100030E03BD00894E108F1086E147F0441F7BD
:104D2000A0960FB6F894DEBF0FBECDBFCF91DF9136
:104D30001F910F91FF90EF90DF90CF90BF90AF90B9
:104D40009F908F907F906F905F904F903F902F90AB
:104D500008952115310539F48091C00085FFFCCFFD
:104D60004093C60008955DCFEF92FF920F931F937B
:104D70009A01E62EFF2400E010E0B801A701E9DF68
:104D80001F910F91FF90EF900895EF92FF920F9374
:104D90001F93CF93DF93EC017A018B01211531052D
:104DA00039F48091C00085FFFCCFE092C60019C0A5
:104DB0002A303105A9F477FF0FC04DE250E060E0E2
:104DC00070E020E030E0E1DF10950095F094E09491
:104DD000E11CF11C011D111DCE01B801A7012AE043
:104DE00020DFDF91CF911F910F91FF90EF900895F9
:104DF000EF92FF920F931F937B019A010027F7FC1C
:104E00000095102FB801A701C0DF1F910F91FF90EF
:104E1000EF9008950F931F938C014DE050E060E0F8
:104E200070E020E030E0B1DFC8014AE050E060E02F
:104E300070E020E030E0A9DF1F910F910895CF923C
:104E4000DF92EF92FF920F931F938C019A016B01F7
:104E5000EE24FF24B701A6017CDFC801DBDF1F9130
:104E60000F91FF90EF90DF90CF9008959F92AF92B7
:104E7000BF92CF92DF92EF92FF920F931F93CF9347
:104E8000DF93EC017A018B01922ECB01BA0120E075
:104E900030E040E050E00E9471B1882364F4CE011C
:104EA0004DE250E060E070E020E030E06EDF17FBA4
:104EB000109517F9109520E030E040E05FE3AA2458
:104EC0000BC0CA01B90120E030E040E251E40E9489
:104ED00078B19B01AC01A394A91498F3C801B70160
:104EE0000E9498B07B018C010E94E5B15B016C01CE
:104EF0000E9411B29B01AC01C801B7010E9497B09A
:104F00007B018C01CE01B601A5012AE030E021DF52
:104F1000992099F1E7E1F2E007C08091C00085FF98
:104F2000FCCF31969093C60090819923B1F725C0AC
:104F3000C801B70120E030E040E251E40E9451B4E2
:104F40007B018C010E94E0B15B016C01CC24B7FCB9
:104F5000C094DC2CCE01B601A5012AE030E015DFBB
:104F6000C601B5010E9413B29B01AC01C801B70193
:104F70000E9497B07B018C019A949920C9F6DF9129
:104F8000CF911F910F91FF90EF90DF90CF90BF9046
:104F9000AF909F9008956ACF0895EF92FF920F937C
:104FA0001F93CF93DF93EC01E090F707F090F807A1
:104FB0000091F9071091FA07688179818A819B81B4
:104FC000A80197010E9471B1882324F4E882F98234
:104FD0000A831B83E090FB07F090FC070091FD071C
:104FE0001091FE076C817D818E819F81A8019701C0
:104FF0000E9471B1882324F4EC82FD820E831F830A
:10500000E090FF07F090000800910108109102085D
:10501000688579858A859B85A80197010E9471B171
:10502000882324F4E886F9860A871B87E09090039A
:10503000F09091030091920310919303688179811C
:105040008A819B81A80197010E947FB3181624F4DE
:10505000E882F9820A831B83E0909403F090950321
:1050600000919603109197036C817D818E819F81C1
:10507000A80197010E947FB3181624F4EC82FD82E8
:105080000E831F83E0909803F090990300919A0398
:1050900010919B03688579858A859B85A801970176
:1050A0000E947FB3181624F4E886F9860A871B87C6
:1050B000DF91CF911F910F91FF90EF900895809114
:1050C0000E0808950F931F93CF93DF9381309105BE
:1050D00049F46F5F7F4F09F046C087E495E00E9476
:1050E000FD1F41C0892B09F03EC06F5F7F4FD9F58E
:1050F0008AE594E090931207809311078091180736
:10510000882321F085E197E00E948668CDECD6E007
:105110000AE514E005C06F9785E0C739D80751F05C
:10512000198308838F818823B1F3CE0104960E94EE
:105130008668F1CF8AE594E0998388838F818823FC
:1051400021F0CE0104960E9486688AE594E090934F
:1051500077058093760580917D05882321F08AE785
:1051600095E00E948668DF91CF911F910F9108957D
:1051700080E090E06FEF7FEFA5CF81E090E06FEFF0
:105180007FEFA0CF0E944C7E80910E08882309F00B
:105190003AC081E080930E08809111089091120826
:1051A000A0911308B09114088093150890931608E5
:1051B000A0931708B0931808E2E2F5E0949108C0B4
:1051C0008091C00085FFFCCF9093C60031969491EA
:1051D0009923B1F7E3E3F5E0949108C08091C00012
:1051E00085FFFCCF9093C600319694919923B1F737
:1051F0008091C00085FFFCCF8AE08093C60089E2E1
:1052000095E00C94C29C089589E260E00E94BFABD7
:10521000A09A0895F8940E944C7E5F9A8A9A8FB75C
:10522000F894909108019160909308018FBF129AB1
:105230008CE060E00E94BFABE2E2F5E0949108C030
:105240008091C00085FFFCCF9093C6003196949169
:105250009923B1F7E2EBF5E0949108C08091C0008A
:1052600085FFFCCF9093C600319694919923B1F7B6
:105270008091C00085FFFCCF8AE08093C60089EA58
:1052800095E00E94D19CFFCF0E940EAA609319085E
:1052900070931A0880931B0890931C08E0914208B1
:1052A000F0914308EC5BF74F80818823A9F4E1ED8E
:1052B000F5E0949108C08091C00085FFFCCF9093E9
:1052C000C600319694919923B1F78091C00085FF73
:1052D000FCCF8AE08093C6000895EF92FF920F936F
:1052E0001F930E940EAAE0901D08F0901E080091E6
:1052F0001F08109120082091190830911A08409138
:105300001B0850911C08621B730B840B950BE6164F
:10531000F7060807190730F4E114F1040105110537
:1053200009F078DF80919E0390919F03A091A003E4
:10533000B091A1030097A105B10561F10E940EAAE9
:105340002091190830911A0840911B0850911C08AF
:10535000621B730B840B950B20919E0330919F036E
:105360004091A0035091A10326173707480759071A
:1053700088F490911C0F80911D0F981759F45F9A33
:105380008A9A9FB7F8948091080181608093080100
:105390009FBF129A909901C03DDF0E9423551F9133
:1053A0000F91FF90EF9008956F927F928F929F924E
:1053B000AF92BF92CF92DF92EF92FF920F931F9323
:1053C000F82E609121087091220880912308909115
:1053D00024082091250830912608409127085091F3
:1053E00028080E948CB33B014C0100D000D00DB7BF
:1053F0001EB70F5F1F4F60918C0370918D0388273C
:1054000077FD8095982F0E9413B22091A2033091CE
:10541000A3034091A4035091A5030E9451B420E03E
:1054200030E040E752E40E9478B120E030E048EC00
:1054300052E40E9478B15B016C01F80160827182D4
:1054400082829382F4828091030885838BED97E0BA
:105450006DE278E041E258E020E001E032E0E32E46
:105460000E940B4E80912D0890912E08A0912F083C
:10547000B09130088093DB079093DC07A093DD07A1
:10548000B093DE078091310890913208A0913308E3
:10549000B09134088093DF079093E007A093E10771
:1054A000B093E2078091350890913608A0913708B3
:1054B000B09138088093E3079093E407A093E50741
:1054C000B093E6078091390890913A08A0913B0883
:1054D000B0913C088093E7079093E807A093E90711
:1054E000B093EA078DB79EB706960FB6F8949EBFA5
:1054F0000FBE8DBF0E940EAA6093190870931A0800
:1055000080931B0890931C081F910F91FF90EF90C0
:10551000DF90CF90BF90AF909F908F907F906F90D3
:105520000895CF92DF92EF92FF920F931F938DE237
:1055300098E033DD0E940EAA6093190870931A0850
:1055400080931B0890931C086091DB077091DC0727
:105550008091DD079091DE0720912D0830912E0873
:1055600040912F08509130080E9471B1882309F0B2
:105570007AC06091DF077091E0078091E107909118
:10558000E207209131083091320840913308509160
:1055900034080E9471B1882309F065C06091A203AC
:1055A0007091A3038091A4039091A50320E030E0C3
:1055B00040E752E40E9478B17B018C018DE298E0D3
:1055C00061E378E045E358E029E338E0E3E0CE2EFC
:1055D000E8E0DE2E0E942E5880912D0890912E0832
:1055E000A0912F08B09130088093DB079093DC07DF
:1055F000A093DD07B093DE078091310890913208C7
:10560000A0913308B09134088093DF079093E007AE
:10561000A093E107B093E207809135089091360896
:10562000A0913708B09138088093E3079093E4077E
:10563000A093E507B093E6078091390890913A0866
:10564000A0913B08B0913C088093E7079093E8074E
:10565000A093E907B093EA071F910F91FF90EF9095
:10566000DF90CF90089560918C0370918D0388270F
:1056700077FD8095982F0E9413B22091A20330915C
:10568000A3034091A4035091A5030E9451B420E0CC
:1056900030E040E752E40E9478B120E030E048EC8E
:1056A00052E488CF86E495E0B2DAE4EDF5E0949137
:1056B00008C08091C00085FFFCCF9093C600319652
:1056C00094919923B1F7409111085091120860917B
:1056D0001308709114084F5F5F4F6F4F7F4F86E440
:1056E00095E02AE030E051DB8091C00085FFFCCFDF
:1056F0008AE08093C600C8CD6F927F928F929F926E
:10570000AF92BF92CF92DF92EF92FF920F931F93CF
:105710006090A2037090A3038090A4039090A503CF
:105720000F2EF0E0AF2EF0E0BF2EFAEFCF2EF5E413
:10573000DF2EF02DA092A203B092A303C092A40387
:10574000D092A503EBEDF7E06093DB077093DC07E5
:105750008093DD079093DE072093DF073093E00707
:105760004093E1075093E207AF01485F5F4FE0923B
:10577000E307F092E4070093E5071093E6079F0123
:10578000245F3F4FCF013496BF010F2EF5E5EF2E7A
:10579000F5E5FF2EF5E00F2FF3E41F2FF02DF3E0DA
:1057A000CF2EF8E0DF2E0E942E580E944C76609299
:1057B000A2037092A3038092A4039092A5031F9169
:1057C0000F91FF90EF90DF90CF90BF90AF909F90A0
:1057D0008F907F906F9008952F923F924F925F929B
:1057E0006F927F928F929F92AF92BF92CF92DF92F1
:1057F000EF92FF920F931F93DF93CF9300D000D0CF
:10580000CDB7DEB78330910508F050C1FC01E153FC
:10581000F84FD4903C01660C771C660C771C930102
:105820002552384F3A83298380E090E0A0E0B0E031
:10583000F90180839183A283B3838BED97E06FEDB1
:1058400077E043EE57E027EE37E00E94FE52F30187
:10585000ED53F84FE590F590059114916D2D772754
:1058600067FD7095882777FD8095982F0E9413B269
:105870001B012C019301235D374F3E832D83C8010B
:10588000B70120E030E040EC5FE30E9451B4A20198
:1058900091010E9451B4AD81BE816D937D938D9332
:1058A0009C931397F301E458FC4FFC83EB836081D6
:1058B0007181828193816093A2037093A30380938B
:1058C000A4039093A50320E030E040E752E40E9457
:1058D00078B17B018C018DE298E061E378E045E3EB
:1058E00058E029E338E0B3E0CB2EB8E0DB2E0E948D
:1058F0002E580E944C7680E090E0A0E0B0E0E98174
:10590000FA8180839183A283B3838BED97E06FED5F
:1059100077E043EE57E027EE37E00E94FE52F301B6
:10592000EA50F84F85909590A590B490C501B401C8
:105930009058A20191010E9451B4AD81BE816D9336
:105940007D938D939C9313976091A2037091A30311
:105950008091A4039091A50320E030E040E752E459
:105960000E9478B17B018C018DE298E061E378E0E0
:1059700045E358E029E338E00E942E580E944C7617
:10598000C501B401A50194010E9498B0A201910142
:105990000E9451B4ED81FE81608371838283938381
:1059A000AB81BC816D917D918D919C9120E030E027
:1059B00040E05FE30E9451B46093A2037093A3039D
:1059C0008093A4039093A50320E030E040E752E4E5
:1059D0000E9478B17B018C018DE298E061E378E070
:1059E00045E358E029E338E00E942E580E944C76A7
:1059F000F301EE52F84F6591759185919491F30101
:105A0000E551F84FA080B180C280D380A6019501F6
:105A10000E9498B07B018C01CB01D801E981FA8109
:105A200080839183A283B383F301E252F84F65919F
:105A3000759185919491A7EF8A2EA7E09A2E860CF6
:105A4000971CA60195010E9498B0D4016D937D9397
:105A50008D939C931397F301E651F84F65917591DF
:105A600085919491E0E9F3E06E0E7F1EA601950109
:105A70000E9498B0D3016D937D938D939C9313975F
:105A8000C701D801ED81FE8180839183A283B38316
:105A900080E090E0A0E0B0E08093A2039093A303A5
:105AA000A093A403B093A5030E942E7526960FB66B
:105AB000F894DEBF0FBECDBFCF91DF911F910F9144
:105AC000FF90EF90DF90CF90BF90AF909F908F901E
:105AD0007F906F905F904F903F902F9008954091EE
:105AE00042085091430820E630E0B901469F9001FA
:105AF000479F300D569F300D1124682F772767FD83
:105B00007095C901825B974F0E9466109C0190932B
:105B10004D0880934C0880E0232B09F081E0089524
:105B2000FC01949108C08091C00085FFFCCF909348
:105B3000C600319694919923B1F786E495E022E06E
:105B400030E029CAFC01949108C08091C00085FF13
:105B5000FCCF9093C600319694919923B1F786E4D7
:105B600095E02AE030E0F5C880914C0890914D080E
:105B7000019660E070E04AE050E00C94CE0E809117
:105B80004C0890914D08019660E070E00C94710D06
:105B9000CF93DF93EC01809103088093100884E594
:105BA0009EDF882309F46DC0EADF0E94E5B1262F4D
:105BB00060931008662309F464C0ECE1F5E0949169
:105BC00008C08091C00085FFFCCF9093C60031963D
:105BD00094919923B1F7C936D10599F0CA36D10508
:105BE00024F4C836D105F1F50FC0CD36D10531F01A
:105BF000CA3DD105B9F5E9E1F2E031C0E0E3F2E0F8
:105C000023C0E7E4F2E015C0EEE5F2E007C08091C2
:105C1000C00085FFFCCF31969093C60090819923F8
:105C2000B1F720C08091C00085FFFCCF31969093E2
:105C3000C60090819923B1F715C08091C00085FFFF
:105C4000FCCF31969093C60090819923B1F70AC09A
:105C50008091C00085FFFCCF31969093C600908163
:105C60009923B1F786E495E0622F40E050E07CD8BC
:105C70008091C00085FFFCCF8AE08093C60081E060
:105C800001C080E0DF91CF910895AF92BF92CF9293
:105C9000DF92EF92FF920F931F93CF93DF930BED61
:105CA000E02E07E0F02ECDE2D8E000E010E0F801B1
:105CB000E65EFB4F808113DF882331F160DF5B01FB
:105CC0006C01F801EB52F84F8081882311F061E0FC
:105CD00002C060913D0870E0882777FD8095982F7D
:105CE0000E9413B2F70120813181428153810E94C9
:105CF00051B49B01AC01C601B5010E9498B0688304
:105D000079838A839B8309C0F70180819181A28175
:105D1000B38188839983AA83BB830F5F1F4F84E07D
:105D200090E0E80EF91E24960430110509F0BFCF6B
:105D300086E4D5DE8823D9F022DF7B018C016093D5
:105D40003E0870933F08809340089093410820E0FC
:105D500030E040E050E00E947FB3181644F4E09237
:105D6000A203F092A3030093A4031093A503DF9171
:105D7000CF911F910F91FF90EF90DF90CF90BF9048
:105D8000AF90089582DF89E4AADE882351F0F7DE20
:105D9000609321087093220880932308909324082D
:105DA0000CC080E090E0A0E0B0E0809321089093E8
:105DB0002208A0932308B09324088AE490DE882365
:105DC00051F0DDDE60932508709326088093270844
:105DD00090932808089580E090E0A0E0B0E08093E0
:105DE000250890932608A0932708B09328080895C3
:105DF0002F923F924F925F926F927F928F929F92DB
:105E0000AF92BF92CF92DF92EF92FF920F931F93C8
:105E1000DF93CF93CDB7DEB76E970FB6F894DEBFA2
:105E20000FBECDBF87E45BDE882309F4E1C3A7DEA4
:105E30000E94E0B16430710509F43CC06530710521
:105E400054F46230710531F16330710554F57723F4
:105E5000CCF40C9478466A35710509F478C36B3537
:105E6000710534F46C31710511F00C94784665C0FD
:105E70006B35710509F46FC36C35710511F00C9425
:105E800078466EC380910E08882321F4FEDE49DB3C
:105E90000C949F4680910E08882319F473DF81E0EB
:105EA00006C080910E08882329F46CDF80E07CDA3C
:105EB0000C949F468AEB97E00E94C29C80E50FDE1F
:105EC000882321F4EE24FF24870105C058DE0E94B8
:105ED000E5B17B018C0183E502DE882359F04FDEBA
:105EE00020E030E04AE754E40E9451B40E94E5B15A
:105EF0007B018C010E944C760E940EAA5B016C0112
:105F0000AE0CBF1CC01ED11E0E940EAA60931908C1
:105F100070931A0880931B0890931C0805C00E9478
:105F20000F82DBD90E94C19E0E940EAA6A157B05D2
:105F30008C059D05A0F30C9478468091A203909166
:105F4000A303A091A403B091A50380934808909364
:105F50004908A0934A08B0934B0880918C03909114
:105F60008D039093DA078093D90784E690E09093AD
:105F70008D0380938C030E940EAA6093190870937E
:105F80001A0880931B0890931C0881E00E943575C5
:105F90008091DB079091DC07A091DD07B091DE07CF
:105FA00080932D0890932E08A0932F08B09330086B
:105FB0008091DF079091E007A091E107B091E2079F
:105FC0008093310890933208A0933308B09334083B
:105FD0008091E3079091E407A091E507B091E6076F
:105FE0008093350890933608A0933708B09338080B
:105FF0008091E7079091E807A091E907B091EA073F
:106000008093390890933A08A0933B08B0933C08DA
:1060100080E090E0A0E0B0E08093A2039093A3031F
:10602000A093A403B093A50388E559DD882351F418
:1060300089E555DD882331F48AE551DD882311F4A3
:1060400081E001C080E08093A603882351F488E5B5
:1060500046DD882309F4D3C189E541DD882309F4AD
:10606000CEC180E090E0A0E0B0E08093DB079093A9
:10607000DC07A093DD07B093DE078093DF079093E2
:10608000E007A093E107B093E207FFEC8F2EF7E063
:106090009F2EF401E4908BED97E06FED77E043EEF7
:1060A00057E027EE37E00E94FE52E3ECF7E06591FF
:1060B00075918591949120E030E040EC5FE30E947F
:1060C00051B45B016C01FF24E7FCF0940027F7FC5E
:1060D0000095102FC801B7010E9413B29B01AC01BB
:1060E000C601B5010E9451B460932D0870932E082B
:1060F00080932F0890933008E7ECF7E06591759155
:10610000859194910894811C911CF401D49020E015
:1061100030E040EC5FE30E9451B47B018C016D2DB7
:10612000772767FD7095872F972F0E9413B29B01E9
:10613000AC01C801B7010E9451B46093310870935B
:106140003208809333089093340820917C03309177
:106150007D0340917E0350917F032093A2033093EF
:10616000A3034093A4035093A503E0908003F09011
:1061700081030091820310918303C801B7010E943B
:1061800071B1882344F4E092A203F092A303009338
:10619000A4031093A5036091A2037091A3038091BF
:1061A000A4039091A50320E030E040E752E40E9470
:1061B00078B17B018C018DE298E061E378E045E302
:1061C00058E029E338E0E3E0CE2EE8E0DE2E0E943E
:1061D0002E580E944C76E2EDF7E06591759185911D
:1061E00094912091EB073091EC074091ED0750918D
:1061F000EE070E9498B06093DB077093DC078093F2
:10620000DD079093DE07EEEDF7E0659175918591DE
:1062100094912091EB073091EC074091ED0750915C
:10622000EE070E9498B06093F7077093F807809389
:10623000F9079093FA07EAEEF7E065917591859179
:1062400094912091EB073091EC074091ED0750912C
:10625000EE070E9498B0609390037093910380932F
:10626000920390939303E6EDF7E065917591859124
:1062700094912091EF073091F0074091F1075091F0
:10628000F2070E9498B06093DF077093E007809355
:10629000E1079093E207E2EEF7E065917591859151
:1062A00094912091EF073091F0074091F1075091C0
:1062B000F2070E9498B06093FB077093FC078093ED
:1062C000FD079093FE07EEEEF7E0659175918591DD
:1062D00094912091EF073091F0074091F107509190
:1062E000F2070E9498B06093940370939503809393
:1062F0009603909397038BED97E06FED77E043EE75
:1063000057E027EE37E00E94FE528091DB07909124
:10631000DC07A091DD07B091DE0780932D089093F4
:106320002E08A0932F08B09330088091DF0790913A
:10633000E007A091E107B091E207809331089093C4
:106340003208A0933308B09334086091A20370918F
:10635000A3038091A4039091A50320E030E040E7DF
:1063600052E40E9478B17B018C018DE298E061E3F8
:1063700078E045E358E029E338E00E942E5880E0B9
:1063800090E0A0E0B0E08093A2039093A303A093D9
:10639000A403B093A5030E944C760E942E758091B1
:1063A0002D0890912E08A0912F08B091300880936D
:1063B000DB079093DC07A093DD07B093DE078091A5
:1063C000310890913208A0913308B091340880933D
:1063D000DF079093E007A093E107B093E207809175
:1063E000350890913608A0913708B091380880930D
:1063F000E3079093E407A093E507B093E607809145
:10640000A603882321F488E56ADB882319F080E05D
:1064100090E0E2D98091A603882321F489E55FDB2F
:10642000882319F081E090E0D7D98091A6038823D2
:1064300021F48AE554DB882319F082E090E0CCD97E
:1064400088E54DDB8823C9F08FDB61157105810577
:10645000910599F094DB2091EB073091EC07409186
:10646000ED075091EE070E9498B06093DB077093A0
:10647000DC078093DD079093DE0789E530DB882316
:10648000C9F072DB611571058105910599F077DB23
:106490002091EF073091F0074091F1075091F207FA
:1064A0000E9498B06093DF077093E0078093E10744
:1064B0009093E2078AE513DB8823C9F055DB611569
:1064C00071058105910599F05ADB2091F307309110
:1064D000F4074091F5075091F6070E9498B0609339
:1064E000E3077093E4078093E5079093E6078BED4D
:1064F00097E06FED77E043EE57E027EE37E00E943C
:10650000FE528091480890914908A0914A08B091A4
:106510004B088093A2039093A303A093A403B0938A
:10652000A5038091D9079091DA0790938D0380930A
:106530008C030E940EAA6093190870931A08809326
:106540001B0890931C080E942E750C94784610929C
:106550003D080C94784681E080933D080C94784681
:1065600085E4BDDA882311F40E944C765BEDE52EBC
:1065700057E0F52E4BEEC42E47E0D42E00E010E09D
:10658000F801E65EFB4F8081AADA882321F103300F
:1065900059F4F5DAF701608371838283938387EE80
:1065A00097E00E94E15217C0EADAF60120813181BA
:1065B000428153810E9498B0F70160837183828386
:1065C00093838BED97E06FED77E043EE57E027EE96
:1065D00037E00E94FE520F5F1F4F24E030E0E20ED2
:1065E000F31EC20ED31E0430110551F60C947846EA
:1065F0008DE475DA882311F40C949A45C0DA0E9470
:10660000E0B16D36710509F4DEC56E3671050CF02A
:106610009CC06E31710509F497C26F3171050CF0A1
:1066200042C06631710509F4F7C167317105E4F4C0
:106630006131710509F4A9C16231710534F4623028
:10664000710510F00C94784645C16431710509F468
:10665000ADC1653171050CF0D9C16231710511F020
:106660000C9478460C94423C6931710509F406C2D9
:106670006A31710554F46731710509F4D3C1683189
:10668000710511F00C947846E9C16B31710509F47C
:1066900018C26B3171050CF4F7C16C31710511F042
:1066A0000C94784614C26335710511F40C943D3C8A
:1066B0006435710514F56A32710509F4E5C36B326E
:1066C000710554F46F31710509F42FC360327105FF
:1066D00011F00C9478467EC26135710511F40C946A
:1066E0001C3C6235710514F00C94393C6035710521
:1066F00011F00C9478460C940F3C6836710509F43F
:106700000DC4693671058CF46535710511F40C946E
:106710009B3C6535710514F40C94423C6C35710555
:1067200011F00C9478460C94B23C6A36710511F461
:106730000C94D83B6A3671050CF421C46B36710594
:1067400011F00C9478460C94093C6C3D710511F4E1
:106750000C943A406D3D71050CF04FC06C387105DA
:1067600009F4FCC36D38710524F56537710511F422
:106770000C94483D6637710564F46237710511F475
:106780000C945F3D6337710511F00C9478460C94BE
:10679000383D6837710511F40C94543E6937710522
:1067A00011F40C94593E6737710511F00C9478463A
:1067B0008DC06B3C710511F40C94803F6C3C7105ED
:1067C0005CF46E3B710509F4E0C6693C710511F09B
:1067D0000C9478460C945E3F6D3C710511F40C945A
:1067E000BE3F6D3C710514F40C949E3F6E3C7105E8
:1067F00011F00C9478460C941C4031E0653F73070F
:1068000011F40C94B94141E0663F74074CF551E036
:106810006D32750711F40C948F4081E06E32780769
:1068200064F46D3D710511F40C9449406C52714053
:1068300011F00C9478460C945840E1E06F327E07DA
:1068400011F40C947641F1E06F327F0714F40C944C
:1068500067416059714011F00C9478460C94B64130
:1068600032E06C3B730751F142E06D3B740794F4E6
:1068700051E0673F750711F40C94C14181E0673F17
:10688000780714F40C94BE416A55724011F00C94D0
:10689000784618C0E3E0603A7E0709F40BC2F3E0E3
:1068A000673E7F0711F40C9483456D5B724011F0D5
:1068B0000C947846E5E7F2E00C941A45E2E8F2E041
:1068C0000C94CC44EDE8F2E00C94CB41E5EAF2E024
:1068D0000C94653E89EA97E00E94C29C80E5FFD84F
:1068E000882321F4EE24FF24870105C048D90E94A3
:1068F000E5B17B018C0183E5F2D8882359F03FD9BB
:1069000020E030E04AE754E40E9451B40E94E5B12F
:106910007B018C010E944C760E940EAA609319089C
:1069200070931A0880931B0890931C08E114F104DB
:106930000105110501F10E940EAA5B016C01AE0C6C
:10694000BF1CC01ED11E0E940EAA6A157B058C05B5
:106950009D05A8F40E945E88882389F40E940F8216
:106960000E946D290E94C19EEECF0E940F820E945C
:106970006D290E94C19E0E945E888823B1F38AE936
:1069800097E00E94C29C0C94784681E997E00E94AF
:10699000C29C5F988A989FB7F894809108018E7F77
:1069A000809308019FBF12980C947846E1E8F7E0C5
:1069B000949108C08091C00085FFFCCF9093C600E1
:1069C000319694919923B1F78091C00085FFFCCF57
:1069D0008AE08093C60087E495E00E94B01FE3E759
:1069E000F7E0949108C08091C00085FFFCCF9093A0
:1069F000C600319694919923B1F78091C00085FF2C
:106A0000FCCF8AE08093C6000C94784687E495E03A
:106A10000E94071B0C94784687E495E00E94281397
:106A20000C94784680914C0890914D0804966AE247
:106A300070E00E946610FC01009711F031971082FF
:106A400060914C0870914D086C5F7F4F87E495E032
:106A500041E021E00E94FE160C94784687E495E020
:106A60000E942C130E940EAA6093060870930708D8
:106A700080930808909309080C94784687E495E081
:106A80000E9433130C94784680914A05882311F4B0
:106A90000C94784683E523D8882311F40C94784627
:106AA00063D8AB01BC014093CA075093CB078093D6
:106AB000CC077093CD0785E197E00E946F670C9437
:106AC000784687E495E00E94ED140C947846809116
:106AD0004C0890914D0804966AE270E00E9466109E
:106AE0008C01009719F1209142083091430880E60B
:106AF00090E0AC01249FC001259F900D349F900D24
:106B00001124825B974F6EE470E00E94661060E291
:106B100070E00E9466109C012F5F3F4F30934D083C
:106B200020934C0801501040F801108260914C08ED
:106B300070914D086C5F7F4F87E495E040E021E065
:106B40000E94FE160C94784680914A05882311F421
:106B50000C94784687E495E060E00E945F14809191
:106B60004C0890914D0804966AE270E00E9466100D
:106B70008C01009719F1209142083091430880E67A
:106B800090E0AC01249FC001259F900D349F900D93
:106B90001124825B974F6EE470E00E94661060E201
:106BA00070E00E9466109C012F5F3F4F30934D08AC
:106BB00020934C0801501040F801108260914C085D
:106BC00070914D086C5F7F4F87E495E00E944715F8
:106BD0000C94784680914905882311F00E944C76E8
:106BE000E0904C08F0904D0824E030E0E20EF31EF7
:106BF000C7016AE270E00E9466108C01C70161E281
:106C000070E00E946610009721F07C010894E11C5E
:106C1000F11C0115110521F001501040F8011082FE
:106C200080E50E946F2D182F80914C0890914D089F
:106C3000E816F90608F410E080914A05882311F45B
:106C40000C94784621E0212787E495E0B70141E0E4
:106C50000E94FE1683E50E946F2D8823B9F0809173
:106C60004C0890914D088E159F0580F40E94B42D1C
:106C7000AB01BC014093CA075093CB078093CC076C
:106C80007093CD0785E197E00E946F6787E495E0F8
:106C90000E942C13112311F00C9478460E940EAA26
:106CA000609306087093070880930808909309087A
:106CB0000C94784680914C0890914D0805966AE2B4
:106CC00070E00E9466108C01009719F12091420833
:106CD0003091430880E690E0AC01249FC001259FDD
:106CE000900D349F900D1124825B974F6EE470E0FD
:106CF0000E94661060E270E00E9466109C012F5FA7
:106D00003F4F30934D0820934C0801501040F8013C
:106D1000108260914C0870914D086B5F7F4F87E443
:106D200095E00E94001B0C9478460E940EAA609386
:106D30000A0870930B0880930C0890930D0820911B
:106D40000608309107084091080850910908621B15
:106D5000730B840B950B28EE33E040E050E00E946B
:106D600069B5F22EE32ED42EC52E2DB73EB728508E
:106D700030400FB6F8943EBF0FBE2DBF0DB71EB703
:106D80000F5F1F4FCE010196EDB7FEB7928381834F
:106D900084E697E0F801938382836F2D7E2D842F04
:106DA000952F2CE330E040E050E00E9469B5F801F7
:106DB000358324836F2D7E2D8D2D9C2D2CE330E08B
:106DC00040E050E00E9469B5F801778366830E9435
:106DD0009510ECE1F5E094912DB73EB7285F3F4F59
:106DE0000FB6F8943EBF0FBE2DBF08C08091C00003
:106DF00085FFFCCF9093C600319694919923B1F70B
:106E0000FE01319607C08091C00085FFFCCF31960E
:106E10009093C60090819923B1F78091C00085FFBF
:106E2000FCCF8AE08093C600CE0101960E94E49CCC
:106E300080914B0A882311F40C94784610924B0AE7
:106E400080910308082F10E0000F111F02571E4EFB
:106E5000F80160817181882777FD8095982F0E94C5
:106E600013B22091AB033091AC034091AD0350912C
:106E7000AE030E947FB3181614F00C947846F80104
:106E8000118210820C94784683E50E946F2D88232E
:106E900011F40C9478460E94BF2D0E94E0B17B0152
:106EA0008C016B0180E50E946F2D882369F0F7FC4F
:106EB0000BC0FFEFEF16F10409F034F40E94BF2D70
:106EC0000E94E0B18B0102C00DE010E0EEE1F4E0C1
:106ED000808191818017910711F40C947846329645
:106EE00024E0EE38F207A1F70930110529F4D09219
:106EF0000508C092040804C017FF02C00C9478462D
:106F0000802F61E00E94BFAB802F6C2D0E9472AC7D
:106F1000802FB6010E94E1AA0C94784688E690E0A2
:106F20000E94C82D882311F00C94784683E50E94B6
:106F30006F2D882379F00E94BF2D20911008022F19
:106F400010E0000F111F02571E4E0E94E0B1F80121
:106F5000718360830E944B7E0C94784683E50E9487
:106F60006F2D882311F40C9478460E94BF2D0E9447
:106F7000E0B170939111609390110C94784689E67A
:106F800090E00E94C82D882311F00C947846EEE51D
:106F9000F7E0949108C08091C00085FFFCCF9093EA
:106FA000C600319694919923B1F7E0911008F0E072
:106FB000EE0FFF1FEE0FFF1FEC56FE4E408151817A
:106FC0006281738186E495E021E030E00E94CB2766
:106FD000EBE5F7E0949108C08091C00085FFFCCFFD
:106FE0009093C600319694919923B1F7E0911008DF
:106FF000F0E0EE0FFF1FE257FE4E6081718188279F
:1070000077FD8095982F0E9413B2AB01BC0186E4F6
:1070100095E021E030E00E94CB27E7E5F7E094918E
:1070200008C08091C00085FFFCCF9093C6003196C8
:1070300094919923B1F740919A1150919B116091CD
:107040009C1170919D1186E495E021E030E00E9452
:10705000CB27E4E5F7E0949108C08091C00085FF5C
:10706000FCCF9093C600319694919923B1F760912B
:10707000901170919111882777FD8095982F0E942B
:1070800013B2AB01BC0186E495E021E030E00E9440
:10709000CB27E1E5F7E0949108C08091C00085FF1F
:1070A000FCCF9093C600319694919923B1F786E472
:1070B00095E060E070E04AE050E00E94F826EFE4DE
:1070C000F7E0949108C08091C00085FFFCCF9093B9
:1070D000C600319694919923B1F740919411509143
:1070E0009511609196117091971186E495E021E0D9
:1070F00030E00E94CB27ECE4F7E0949108C0809147
:10710000C00085FFFCCF9093C600319694919923DF
:10711000B1F760918E1170918F11882777FD80955E
:10712000982F0E9413B2AB01BC0186E495E021E0E8
:1071300030E00E94CB27E8E4F7E0949108C080910A
:10714000C00085FFFCCF9093C6003196949199239F
:10715000B1F7809110080E94407EBC0186E495E062
:107160004AE050E00E94F826E3E4F7E0949108C07A
:107170008091C00085FFFCCF9093C600319694911A
:107180009923B1F78FEF9FEF0E94407EBC0186E408
:1071900095E04AE050E00E94F826EEEBF2E007C0EE
:1071A0008091C00085FFFCCF31969093C6009081FE
:1071B0009923B1F78091C00085FFFCCF8AE08093CE
:1071C000C6000C949F468DE690E00E94C82D88234F
:1071D00011F00C94784688E397E00E94C29C1092CC
:1071E0004B0A83E50E946F2D882399F00E94BF2DE2
:1071F00020911008022F10E0000F111F02571E4EA1
:107200000E94E0B1F8017183608381E080939D0367
:1072100016C082E50E946F2D882389F00E94BF2D41
:1072200020911008022F10E0000F111F02571E4E70
:107230000E94E0B1F8017183608310929D0383E5A1
:107240000E946F2D882351F00E94BF2D6093AB03E5
:107250007093AC038093AD039093AE0382E40E94DD
:107260006F2D882351F00E94BF2D6093A703709368
:10727000A8038093A9039093AA0386E40E946F2D2C
:10728000882369F00E94BF2D6093AF037093B00311
:107290008093B1039093B20381E080934B0A0E94E4
:1072A0004B7E0E940EAA4B015C0120911008022F18
:1072B00010E010920F08000F111FF801E257FE4E68
:1072C00060817181882777FD8095982F0E9413B285
:1072D000000F111F0C561E4EF80120813181428192
:1072E00053810E947FB318161CF481E080930F082D
:1072F000CC24CA94DC2C7601E5E3F7E05490E1E37A
:10730000F7E06490EDE2F7E074904AE0442E30C17B
:10731000952DE5E3F7E008C08091C00085FFFCCF24
:107320009093C600319694919923B1F7E09110089B
:10733000F0E0EE0FFF1FEE0FFF1FEC56FE4E4081F8
:1073400051816281738186E495E021E030E00E9402
:10735000CB27962DE1E3F7E008C08091C00085FFC0
:10736000FCCF9093C600319694919923B1F7609128
:10737000100886E495E070E04AE050E00E94F826AC
:10738000972DEDE2F7E008C08091C00085FFFCCFAB
:107390009093C600319694919923B1F7F7FE03C0FC
:1073A000EFEBF2E028C00E940EAAA7019601205F31
:1073B000384D4F4F5F4F261B370B480B590BCA01F7
:1073C000B90128EE33E040E050E00E9469B586E460
:1073D00095E0BA01A9012AE030E00E94A926809137
:1073E000C00085FFFCCF0EC08091C00085FFFCCFA0
:1073F00031969093C60090819923B1F78091C00097
:1074000085FFFCCF4092C6000E940EAA4B015C0192
:107410000E940F820E946D290E94C19EFFEFCF162D
:10742000FFEFDF06FFEFEF06FFEFFF0609F052C0A8
:1074300080910F08E0911008882331F1F0E08F016E
:10744000000F111F000F111F0C561E4EEE0FFF1FD5
:10745000E257FE4E60817181882777FD8095982FD5
:107460000E9413B220E030E040E85FE30E9497B052
:107470009B01AC01F80160817181828193810E943E
:107480007FB387FF58C05EC0F0E08F01000F111F6F
:10749000000F111F0C561E4EEE0FFF1FE257FE4E3F
:1074A00060817181882777FD8095982F0E9413B2A3
:1074B00020E030E040E85FE30E9498B09B01AC011F
:1074C000F80160817181828193810E9471B11816E7
:1074D00094F538C0F7FC36C0E0911008F0E08F0159
:1074E000000F111F000F111F0C561E4EEE0FFF1F35
:1074F000E257FE4E60817181882777FD8095982F35
:107500000E9413B29B01AC01F801608171818281FC
:1075100093810E9497B00E94E0B197FF07C09095B9
:107520008095709561957F4F8F4F9F4F64307105A7
:10753000810591053CF00E940EAAAC01CB01DA0155
:107540006C017D01FFEFCF16FFEFDF06FFEFEF06C7
:10755000FFEFFF0669F0F7FE02C00C947B460E9425
:107560000EAA6C197D096051774210F00C947B468D
:107570000E940EAA681979098A099B09695E7340FD
:107580008040904008F0C4CE43CF82E197E00E9453
:10759000C29C83E50E946F2D882361F00E94BF2D5D
:1075A0000E94E0B1709391116093901181E08093FB
:1075B0009D030FC082E50E946F2D882351F00E9429
:1075C000BF2D0E94E0B170939111609390111092C1
:1075D0009D030E940EAA7B018C0110920F086091FE
:1075E000901170919111882777FD8095982F0E94B6
:1075F00013B220919A1130919B1140919C1150919E
:107600009D110E947FB318160CF082C081E0809318
:107610000F087EC00E940EAA6E197F09800B910B85
:10762000695E73408040904008F46BC0E0910308AD
:10763000F0E0EE0FFF1FEE0FFF1FEC56FE4E4081F5
:107640005181628173819B2DEFE0F7E008C080914A
:10765000C00085FFFCCF9093C6003196949199238A
:10766000B1F786E495E022E030E00E94CB279C2D24
:10767000EBE0F7E008C08091C00085FFFCCF90935D
:10768000C600319694919923B1F76091030886E47E
:1076900095E070E04AE050E00E94F8269D2DE7E07A
:1076A000F7E008C08091C00085FFFCCF9093C60032
:1076B000319694919923B1F740919A1150919B1171
:1076C00060919C1170919D1186E495E021E030E07D
:1076D0000E94CB27EEEBF2E007C08091C00085FF4F
:1076E000FCCF31969093C60090819923B1F7809199
:1076F000C00085FFFCCFA092C6000E940EAA7B01AD
:107700008C010E940F820E946D290E94C19E0BC0B5
:10771000EFE0F7E0B490EBE0F7E0C490E7E0F7E0EB
:10772000D4905AE0A52E80910F08209190113091AD
:1077300091118823A9F0B901882777FD8095982FAA
:107740000E9413B220919A1130919B1140919C118B
:1077500050919D110E947FB318160CF45BCF18C096
:10776000B901882777FD8095982F0E9413B2209148
:107770009A1130919B1140919C1150919D110E9442
:1077800071B188232CF480919D03882309F442CFA2
:107790008DEF96E00E94C29C0E940EAA6093190889
:1077A00070931A0880931B0890931C080C947846D9
:1077B00083E50E946F2D882321F10E94BF2D20E0D8
:1077C00030E040E050E00E9471B188231CF460E09A
:1077D00070E011C00E94BF2D20E030E04FE753E47D
:1077E0000E947FB318161CF46FEF70E004C00E9473
:1077F000BF2D0E94E0B170930508609304080C94BB
:1078000078468FEF90E090930508809304080C94DD
:10781000784610920508109204080C947846269A2F
:107820002E9881E080939C038CEE96E00E94C29C8F
:107830000E94C19E0C9478460E944C7E0E944C7619
:10784000129A0E945A76109205081092040868EE67
:1078500073E080E090E00E941CAA269A2E9A109273
:107860009C038DED96E00E94C29C0E94C19E0C94E8
:1078700078461092D8070C94784681E08093D80718
:107880000C94784683E50E946F2D8823A1F00E9416
:10789000BF2D20E030E04AE754E40E9451B40E943A
:1078A000E5B160939E0370939F038093A003909330
:1078B000A1030C94784688E50E946F2D882311F06F
:1078C0000C94944689E50E946F2D882311F00C9446
:1078D00094468AE50E946F2D882311F00C949446FB
:1078E00085E40E946F2D882311F00C9494460E9429
:1078F0004C76129A0E945A760C9478465F9A89E5E3
:107900000E946F2D81118A9A8AE50E946F2D88232B
:1079100041F09FB7F894809108018160809308013D
:107920009FBF85E40E946F2D882311F40C94784644
:10793000129A0C94784683E50E946F2D0E94BF2D09
:1079400020E030E04AE754E40E9451B40E94E5B1DF
:1079500060931D0870931E0880931F089093200861
:107960000C9478464FEE642E49E0742E3FED232EA2
:1079700039E0332E2BE2422E2AE0522E882499241D
:10798000F401E65EFB4F80810E946F2D882309F48D
:107990005DC053E0851609F052C00E94BF2D5B0107
:1079A0006C0120E030E040EA51E40E9471B188238C
:1079B0000CF03FC0F3016081718182819381A60147
:1079C00095010E9478B17B018C016091230A70912E
:1079D000240A8091250A9091260AA80197010E9405
:1079E00051B46093230A7093240A8093250A9093DC
:1079F000260AF1016081718182819381A80197013A
:107A00000E9451B4F1016083718382839383F201F8
:107A100060817181828193810E9411B2A8019701D6
:107A20000E9451B40E94E5B1F201608371838283A8
:107A30009383F301A082B182C282D38207C00E94E5
:107A4000BF2DF30160837183828393830894811C2B
:107A5000911C24E030E0620E731E220E331E420E93
:107A6000531E34E08316910409F08ACF0C947846B3
:107A7000EFE3F6E0949108C08091C00085FFFCCF51
:107A80009093C600319694919923B1F70C9478465F
:107A900080914C0890914D0805966AE270E00E9432
:107AA0006610FC01009711F03197108280914C080C
:107AB00090914D0805960E94E49C0C947846ECE366
:107AC000F6E0949108C08091C00085FFFCCF9093B0
:107AD000C600319694919923B1F74091DB075091FC
:107AE000DC076091DD077091DE0786E495E022E017
:107AF00030E00E94CB27E9E3F6E0949108C0809142
:107B0000C00085FFFCCF9093C600319694919923D5
:107B1000B1F74091DF075091E0076091E107709164
:107B2000E20786E495E022E030E00E94CB27E6E31E
:107B3000F6E0949108C08091C00085FFFCCF90933F
:107B4000C600319694919923B1F74091E307509183
:107B5000E4076091E5077091E60786E495E022E08E
:107B600030E00E94CB27E3E3F6E0949108C08091D7
:107B7000C00085FFFCCF9093C60031969491992365
:107B8000B1F74091E7075091E8076091E9077091DC
:107B9000EA0786E495E022E030E00E94CB27E8E2A5
:107BA000F6E0949108C08091C00085FFFCCF9093CF
:107BB000C600319694919923B1F780E00E94177620
:107BC0000E9413B22091EF093091F0094091F10920
:107BD0005091F2090E9478B1AB01BC0186E495E0B6
:107BE00022E030E00E94CB27E5E2F6E0949108C065
:107BF0008091C00085FFFCCF9093C6003196949190
:107C00009923B1F781E00E9417760E9413B2209168
:107C1000F3093091F4094091F5095091F6090E9459
:107C200078B1AB01BC0186E495E022E030E00E942F
:107C3000CB27E2E2F6E0949108C08091C00085FF76
:107C4000FCCF9093C600319694919923B1F782E0CE
:107C50000E9417760E9413B22091F7093091F8091B
:107C60004091F9095091FA090E9478B1AB01BC0129
:107C700086E495E022E030E00E94CB27EEEBF2E0D4
:107C800007C08091C00085FFFCCF31969093C6005D
:107C900090819923B1F78091C00085FFFCCF8AE0E5
:107CA0008093C6000C94784680E00E9435750C9451
:107CB000784681E00E9435750C9478468091C0002A
:107CC00085FFFCCF31969093C60090819923B1F740
:107CD0008091C00085FFFCCF8AE08093C600EAE176
:107CE000F6E0949108C08091C00085FFFCCF90938E
:107CF000C600319694919923B1F7659B03C0E1ECDE
:107D0000F2E00AC0E6ECF2E007C08091C00085FF17
:107D1000FCCF31969093C60090819923B1F7809162
:107D2000C00085FFFCCF8AE08093C600E2E1F6E068
:107D3000949108C08091C00085FFFCCF9093C6004D
:107D4000319694919923B1F7649B03C0E1ECF2E082
:107D50000AC0E6ECF2E007C08091C00085FFFCCFCE
:107D600031969093C60090819923B1F78091C0001D
:107D700085FFFCCF8AE08093C600EAE0F6E09491AC
:107D800008C08091C00085FFFCCF9093C60031965B
:107D900094919923B1F78091030181FF03C0E1EC35
:107DA000F2E00AC0E6ECF2E007C08091C00085FF77
:107DB000FCCF31969093C60090819923B1F78091C2
:107DC000C00085FFFCCF8AE08093C600E2E0F6E0C9
:107DD000949108C08091C00085FFFCCF9093C600AD
:107DE000319694919923B1F78091030180FF03C0EC
:107DF000E1ECF2E00AC0E6ECF2E007C08091C000DE
:107E000085FFFCCF31969093C60090819923B1F7FE
:107E10008091C00085FFFCCF8AE08093C600EAEF26
:107E2000F5E0949108C08091C00085FFFCCF90934D
:107E3000C600319694919923B1F74B9B03C0E1ECB6
:107E4000F2E00AC0E6ECF2E007C08091C00085FFD6
:107E5000FCCF31969093C60090819923B1F7809121
:107E6000C00085FFFCCF8AE08093C600E2EFF5E01A
:107E7000949108C08091C00085FFFCCF9093C6000C
:107E8000319694919923B1F74A9B03C0E1ECF2E05B
:107E90000AC0E6ECF2E007C08091C00085FFFCCF8D
:107EA00031969093C60090819923B1F78091C000DC
:107EB00085FFFCCF8AE08093C6001AC70AE114E070
:107EC0009FEFE92E99E0F92EF80180810E946F2D35
:107ED000882349F00E94BF2D0E94E5B1F70160831D
:107EE0007183828393830F5F1F4F24E030E0E20EA3
:107EF000F31E34E00E31130739F70E94B652F8C66C
:107F00000AE114E08FEDE82E89E0F82EF801808177
:107F10000E946F2D882339F00E94BF2DF7016083E6
:107F20007183828393830F5F1F4F24E030E0E20E62
:107F3000F31E34E00E31130749F7DAC683E50E94D9
:107F40006F2D882351F00E94BF2D6093130A709308
:107F5000140A8093150A9093160A84E50E946F2DE7
:107F6000882309F4C5C60E94BF2D6093170A709339
:107F7000180A8093190A90931A0ABAC683E50E94D8
:107F80006F2D882351F00E94BF2D60930F0A7093CC
:107F9000100A8093110A9093120A84E50E946F2DB3
:107FA000882351F00E94BF2D6093270A7093280AFE
:107FB0008093290A90932A0A82E40E946F2D8823D5
:107FC00061F00E94BF2D0E94E5B16093DB097093C0
:107FD000DC098093DD099093DE0988E50E946F2D0E
:107FE000882351F00E94BF2D60931B0A70931C0AD6
:107FF00080931D0A90931E0A8AE50E946F2D8823A4
:1080000051F00E94BF2D60931F0A7093200A809345
:10801000210A9093220A85E40E946F2D882309F497
:1080200067C60E94BF2D6093230A7093240A809331
:10803000250A9093260A5CC60AE114E0BBEEEB2EFB
:10804000B7E0FB2EF80180810E946F2D882339F064
:108050000E94BF2DF70160837183828393830F5F3A
:108060001F4F24E030E0E20EF31E34E00D31130721
:1080700049F73EC683E50E946F2D882309F438C670
:108080000E94BF2D0E94E0B170938D0360938C031A
:108090002FC683E50E946F2D882309F429C60E940C
:1080A000BF2D0E94E0B170938F0360938E0320C6B2
:1080B00083E50E946F2D882321F4AEE6CA2ED12CD1
:1080C00005C00E94BF2D0E94E0B16B0180E50E94B7
:1080D0006F2D882319F468EE73E004C00E94BF2D51
:1080E0000E94E0B17B010027F7FC0095102F1C14C3
:1080F0001D0484F485E2B60120E030E040E050E069
:108100000E94A9ADC801B7010E941CAA85E20E9485
:1081100035ADEEC5C801B7010E941CAAE9C580E5CE
:108120000E946F2D882351F00E94BF2D6093BC03E5
:108130007093BD038093BE039093BF0389E40E94B4
:108140006F2D882361F00E94BF2D0E94687E60938E
:10815000C0037093C1038093C2039093C30384E46C
:108160000E946F2D882361F00E94BF2D0E94747EB3
:108170006093C4037093C5038093C6039093C703B1
:1081800083E40E946F2D882351F00E94BF2D6093DD
:10819000C8037093C9038093CA039093CB030E94D2
:1081A000297EE0EDF2E007C08091C00085FFFCCFA2
:1081B00031969093C60090819923B1F7E3EDF2E0F8
:1081C00007C08091C00085FFFCCF31969093C60018
:1081D00090819923B1F74091BC035091BD03609108
:1081E000BE037091BF0386E495E022E030E00E9478
:1081F000CB27E7EDF2E007C08091C00085FFFCCF00
:1082000031969093C60090819923B1F76091C00395
:108210007091C1038091C2039091C3030E946E7E4E
:10822000AB01BC0186E495E022E030E00E94CB2760
:10823000EBEDF2E007C08091C00085FFFCCF3196E6
:108240009093C60090819923B1F76091C403709117
:10825000C5038091C6039091C7030E947A7EAB014B
:10826000BC0186E495E022E030E00E94CB27EFEDF0
:10827000F2E007C08091C00085FFFCCF319690935B
:10828000C60090819923B1F74091C8035091C9036A
:108290006091CA037091CB0386E495E022E030E060
:1082A0000E94CB27EEEBF2E007C08091C00085FF73
:1082B000FCCF31969093C60090819923B1F78091BD
:1082C000C00085FFFCCF8AE08093C60011C583E51E
:1082D0000E946F2D882329F460E070E080E090E038
:1082E00002C00E94BF2D0E94AD5202C585E40E94CB
:1082F0006F2D882319F4CC24DD2412C00E94BF2DD9
:108300000E94E0B16B0177FF0BC00F2EF0E0EF2E63
:10831000F0E0FF2EFCE80F2FF2E41F2FF02D0AC033
:108320000F2EF0E0EF2EF0E0FF2EF6E10F2FF3E43A
:108330001F2FF02D83E50E946F2D882321F00E94CE
:10834000BF2D7B018C0183E40E946F2D882319F4DB
:1083500025E030E005C00E94BF2D0E94E0B19B01E6
:10836000C801B701A6010E94C283C2C40E944C7614
:10837000BFC40E9499200E944622BAC40E9499203C
:10838000B7C40E944622B4C48091C00085FFFCCFD0
:1083900031969093C60090819923B1F78091C000E7
:1083A00085FFFCCF8AE08093C60081E00E94588858
:1083B00006C080E090E00E9453880E94C19E0E9407
:1083C0005E888823B1F381E090E00E94538881E0C9
:1083D0000E9458888091A2039091A303A091A403C6
:1083E000B091A5038093480890934908A0934A0848
:1083F000B0934B0880918C0390918D039093DA0792
:108400008093D90784E690E090938D0380938C034A
:108410000E940EAA6093190870931A0880931B0893
:1084200090931C0881E00E9435758091DB07909144
:10843000DC07A091DD07B091DE0780932D089093B3
:108440002E08A0932F08B09330088091DF079091F9
:10845000E007A091E107B091E20780933108909383
:108460003208A0933308B09334088091E3079091C9
:10847000E407A091E507B091E60780933508909353
:108480003608A0933708B09338088091E707909199
:10849000E807A091E907B091EA0780933908909323
:1084A0003A08A0933B08B0933C0880E090E0A0E03D
:1084B000B0E08093A2039093A303A093A403B0938E
:1084C000A50388E50E946F2D882361F489E50E9449
:1084D0006F2D882339F48AE50E946F2D882311F4CB
:1084E00081E001C080E08093A603882329F488E519
:1084F0000E946F2D882321F080E090E00E94EC2BF9
:108500008091A603882329F489E50E946F2D882392
:1085100021F081E090E00E94EC2B8091A60388235B
:1085200029F48AE50E946F2D882321F082E090E0F3
:108530000E94EC2B88E50E946F2D8823D9F00E94C1
:10854000B42D6115710581059105A1F00E94BF2D23
:108550002091EB073091EC074091ED075091EE0729
:108560000E9498B06093DB077093DC078093DD076F
:108570009093DE0789E50E946F2D8823D9F00E9431
:10858000B42D6115710581059105A1F00E94BF2DE3
:108590002091EF073091F0074091F1075091F207D9
:1085A0000E9498B06093DF077093E0078093E10723
:1085B0009093E2078AE50E946F2D8823D9F00E94EC
:1085C000B42D6115710581059105A1F00E94BF2DA3
:1085D0002091F3073091F4074091F5075091F60789
:1085E0000E9498B06093E3077093E4078093E507D7
:1085F0009093E6078BED97E06FED77E043EE57E061
:1086000027EE37E00E94FE52809148089091490879
:10861000A0914A08B0914B088093A2039093A303C2
:10862000A093A403B093A5038091D9079091DA0792
:1086300090938D0380938C030E940EAA6093190877
:1086400070931A0880931B0890931C080E942E7543
:108650008BED97E06FED77E043EE57E027EE37E0E4
:108660000E94FE526091DB077091DC078091DD076C
:108670009091DE072091DF073091E0074091E107FC
:108680005091E2070F2EF0E0EF2EF0E0FF2EF0E227
:108690000F2FF1E41F2FF02D0E947C2BE090E307B9
:1086A000F090E4070091E5071091E60760E070E0C4
:1086B00084E193E420E030E048E453E40E947C2B22
:1086C0006091DB077091DC078091DD079091DE07F8
:1086D0002091DF073091E0074091E1075091E207D8
:1086E0000F2EF0E0EF2EF0E0FF2EF0E00F2FF0E085
:1086F0001F2FF02D0E947C2B02C00E940F820E942F
:108700005E888823D1F381E00E94588882E090E05F
:108710000E9453886091DB077091DC078091DD0730
:108720009091DE072091DF073091E0074091E1074B
:108730005091E2070F2EF0E0EF2EF0E0FF2EF0E276
:108740000F2FF1E41F2FF02D0E947C2BE090E30708
:10875000F090E4070091E5071091E60760E070E013
:108760008AEB92E420E030E040EA50E40E947C2B67
:108770006091DB077091DC078091DD079091DE0747
:108780002091DF073091E0074091E1075091E20727
:108790000F2EF0E0EF2EF0E0FF2EF0E00F2FF0E0D4
:1087A0001F2FF02D0E947C2B04C00E940F820E947C
:1087B0006D290E945E888823C1F381E00E94588859
:1087C00083E090E00E9453886091DB077091DC07A2
:1087D0008091DD079091DE072091DF073091E0075F
:1087E0004091E1075091E2070F2EF0E0EF2EF0E00C
:1087F000FF2EF0E20F2FF1E41F2FF02D0E947C2BB3
:10880000E090E307F090E4070091E5071091E60798
:1088100060E070E08FE493E420E030E040EA50E470
:108820000E947C2B6091DB077091DC078091DD0753
:108830009091DE072091DF073091E0074091E1073A
:108840005091E2070F2EF0E0EF2EF0E0FF2EF0E067
:108850000F2FF0E01F2FF02D0E947C2B04C00E94F0
:108860000F820E946D290E945E888823C1F381E0F7
:108870000E94588884E090E00E9453886091DB0752
:108880007091DC078091DD079091DE072091DF0772
:108890003091E0074091E1075091E2070F2EF0E0A0
:1088A000EF2EF0E0FF2EF0E20F2FF1E41F2FF02D5E
:1088B0000E947C2BE090E307F090E4070091E5072D
:1088C0001091E60760E070E086E193E420E030E09C
:1088D00042ED52E40E947C2B6091DB077091DC0733
:1088E0008091DD079091DE072091DF073091E0074E
:1088F0004091E1075091E2070F2EF0E0EF2EF0E0FB
:10890000FF2EF0E00F2FF0E01F2FF02D0E947C2BA8
:1089100004C00E940F820E946D290E945E888823F5
:10892000C1F381E00E94588885E090E00E9453885E
:108930006091DB077091DC078091DD079091DE0785
:108940002091DF073091E0074091E1075091E20765
:108950000F2EF0E0EF2EF0E0FF2EF8E40F2FF2E400
:108960001F2FF02D0E947C2BE090E307F090E4078E
:108970000091E5071091E60760E070E080E291E485
:108980009B01AC010E947C2BB3C18091C00085FF8C
:10899000FCCF31969093C60090819923B1F78091D6
:1089A000C00085FFFCCF8AE08093C6000E944C7611
:1089B0008BED97E06FED77E043EE57E027EE37E081
:1089C0000E94FE526091E7077091E8078091E907E5
:1089D0009091EA0720E030E048EC52E40E9498B021
:1089E0006093E7077093E8078093E9079093EA079D
:1089F0008BED97E06FED77E043EE57E027EE37E041
:108A00000F2EF0E0EF2EF0E0FF2EF0EA0F2FF0E453
:108A10001F2FF02DF3E0CF2EF8E0DF2E0E942E580E
:108A20000E944C7665C18091C00085FFFCCF3196D5
:108A30009093C60090819923B1F78091C00085FF83
:108A4000FCCF8AE08093C6000E944C768BED97E0C5
:108A50006FED77E043EE57E027EE37E00E94FE52DD
:108A60006091E7077091E8078091E9079091EA0724
:108A700020E030E040E251E40E9498B06093E707C4
:108A80007093E8078093E9079093EA078BED97E0EE
:108A90006FED77E043EE57E027EE37E00F2EF0E082
:108AA000EF2EF0E0FF2EF0EA0F2FF0E41F2FF02D55
:108AB000E3E0CE2EE8E0DE2E0E942E580E944C7697
:108AC0006091E7077091E8078091E9079091EA07C4
:108AD00020E030E040E752E40E9497B06093E7075F
:108AE0007093E8078093E9079093EA078BED97E08E
:108AF0006FED77E043EE57E027EE37E00E942E5807
:108B00000E944C76F5C010920E080E945B888091FE
:108B1000150890911608A0911708B0911808809335
:108B2000110890931208A0931308B09314080E94A0
:108B3000522BDEC084E50E946F2D882309F48DC07E
:108B40000E94BF2D0E94E5B1262F60931008662376
:108B5000B9F1ECE1F5E0949108C08091C00085FF87
:108B6000FCCF9093C600319694919923B1F7E3EE30
:108B7000F2E007C08091C00085FFFCCF3196909352
:108B8000C60090819923B1F786E495E0622F40E01A
:108B900050E00E94B426E5EEF2E007C08091C000EC
:108BA00085FFFCCF31969093C60090819923B1F751
:108BB0008091C00085FFFCCF8AE08093C60098C0FA
:108BC00086E40E946F2D8823E1F00E94BF2D7B0177
:108BD0008C0160933E0870933F0880934008909307
:108BE000410820E030E040E050E00E947FB31816DA
:108BF00044F4E092A203F092A3030093A403109321
:108C0000A503ECE1F5E0949108C08091C00085FFD8
:108C1000FCCF9093C600319694919923B1F7E6EF7B
:108C2000F2E007C08091C00085FFFCCF31969093A1
:108C3000C60090819923B1F76091030886E495E01E
:108C400070E04AE050E00E94F8268091C00085FF65
:108C5000FCCF8AE08093C6004BC0ECE1F5E0949134
:108C600008C08091C00085FFFCCF9093C60031966C
:108C700094919923B1F7EFEDF5E0949108C08091BC
:108C8000C00085FFFCCF9093C60031969491992344
:108C9000B1F7209142083091430880E690E0289F88
:108CA000F001299FF00D389FF00D1124E25BF74F82
:108CB00007C08091C00085FFFCCF31969093C6001D
:108CC00090819923B1F7EDEDF5E0949108C0809182
:108CD000C00085FFFCCF9093C600319694919923F4
:108CE000B1F78091C00085FFFCCF8AE08093C60079
:108CF0000E94442924C08FE197E00E94C29C0E94F8
:108D00000EAA609306087093070880930808909352
:108D100009080E940EAA6093190870931A0880939C
:108D20001B0890931C08E4CF0E944C7688E50E94B3
:108D30006F2D882311F00C947E3C0C947F3C6E9632
:108D40000FB6F894DEBF0FBECDBFCF91DF911F915C
:108D50000F91FF90EF90DF90CF90BF90AF909F90DA
:108D60008F907F906F905F904F903F902F900895DD
:108D70002F923F924F925F926F927F928F929F922B
:108D8000AF92BF92CF92DF92EF92FF920F931F9319
:108D9000DF93CF93CDB7DEB76E970FB6F894DEBFF3
:108DA0000FBECDBF80E6A82EB12CE3E3F8E084909F
:108DB0000AE0702EE9EAF8E094906624639413C206
:108DC0002D3071F02A3321F48091CF09882341F0AE
:108DD0008091D0099091D1098F3591050CF4DFC1B4
:108DE000E091D009F091D109309709F404C3A09122
:108DF000D209B091D309AA9D7001AB9DF00CBA9D28
:108E0000F00C1124EE0DFF1DE25BF74F10828091F4
:108E1000CF09882309F0BEC11092CF09AC5BB74FD0
:108E20001C928701025B174FC8016EE470E00E943C
:108E300066109C01009709F4F7C090934D08809349
:108E40004C082F5F3F4F201B310B2E0D3F1DC901DA
:108E5000825B974F60E070E04AE050E00E94CE0EE7
:108E60006093D4097093D5098093D6099093D7095C
:108E7000C0901108D0901208E0901308F0901408E8
:108E8000A70196012F5F3F4F4F4F5F4F6217730748
:108E90008407950709F457C38091D2099091D309AB
:108EA0009C012A9DC0012B9D900D3A9D900D11248F
:108EB000825B974F62E579E00E942B10892B09F0C5
:108EC00042C3E2E2F5E0949108C08091C00085FFC2
:108ED000FCCF9093C600319694919923B1F7EFE1BE
:108EE000F9E0949108C08091C00085FFFCCF909379
:108EF000C600319694919923B1F786E495E0B701C5
:108F0000A6012AE030E00E94C5268091C00085FFBE
:108F1000FCCF73C0FE264F5FFC01E40FF11DE25B46
:108F2000F74FE081EA32B1F730934D0820934C08B7
:108F3000C901019660E070E00E94710D0E94E0B1ED
:108F40002F2D30E02617370709F45DC0E2E2F5E087
:108F5000949108C08091C00085FFFCCF9093C6001B
:108F6000319694919923B1F7E0E0F9E0949108C02B
:108F70008091C00085FFFCCF9093C60031969491FC
:108F80009923B1F74091110850911208609113088C
:108F90007091140886E495E02AE030E00E94C5262E
:108FA0008091C00085FFFCCF28C0E2E2F5E09491FB
:108FB00008C08091C00085FFFCCF9093C600319619
:108FC00094919923B1F7E6EDF8E0949108C080916F
:108FD000C00085FFFCCF9093C600319694919923F1
:108FE000B1F786E495E0B701A6012AE030E00E94DF
:108FF000C5268091C00085FFFCCF8AE08093C60023
:109000000E94522B4AC08091D4099091D509A09119
:10901000D609B091D7098093110890931208A093B4
:109020001308B09314083EC0C8016AE270E00E94C1
:109030006610009709F436C0E2E2F5E0949108C0AA
:109040008091C00085FFFCCF9093C600319694912B
:109050009923B1F7ECEAF8E0949108C08091C00040
:1090600085FFFCCF9093C600319694919923B1F778
:1090700040911108509112086091130870911408E2
:1090800086E495E02AE030E00E94C5268091C00089
:1090900085FFFCCF8AE08093C6001092D109109220
:1090A000D00970C28091D2099091D3098A9D700134
:1090B0008B9DF00C9A9DF00C11248701025B174FD9
:1090C000C80167E470E00E9466109C01009709F4F3
:1090D0004BC090934D0880934C082F5F3F4F201B4F
:1090E000310B2E0D3F1DC901825B974F60E070E090
:1090F0000E94710D0E94E0B164307105A8F5809165
:109100000E088823C9F480914705882369F5992DB5
:10911000E9EAF8E008C08091C00085FFFCCF909399
:10912000C600319694919923B1F78091C00085FFD4
:10913000FCCF7092C60018C0982DE3E3F8E008C099
:109140008091C00085FFFCCF9093C600319694912A
:109150009923B1F78091C00085FFFCCF7092C600C3
:1091600089E298E00E94C29C8091D2099091D30933
:10917000019664E070E00E9456B59093D309809305
:10918000D2098091D8099091D90901969093D90973
:109190008093D8091092D1091092D00924C02B33A2
:1091A00011F46092CF098091CF098823E1F42091D6
:1091B000D0093091D1098091D2099091D3098A9D2B
:1091C000F0018B9DF00D9A9DF00D1124E20FF31F1D
:1091D000E25BF74F8091CE0980832F5F3F4F309342
:1091E000D1092093D00980914205909143052091A7
:1091F000440530914505821B930B8F779070892B26
:1092000009F4BBC18091D8099091D90904970CF059
:10921000B4C186E495E00E94E925282F8093CE0909
:109220008A3009F0CDCDDCCD8091D0099091D10963
:10923000892B09F0A7C18091D8099091D909892B70
:1092400009F02FC11092DA092CC14D3099F0433248
:1092500011F04A3321F48091CF09882359F080918D
:10926000D0099091D1098F35910524F42F5F3F4F9C
:1092700009F0F2C02091CA073091CB074091CC078A
:109280005091CD078091C2079091C307A091C40768
:10929000B091C507281739074A075B0708F49EC035
:1092A000932DE6E1F8E008C08091C00085FFFCCF77
:1092B0009093C600319694919923B1F78091C000A4
:1092C00085FFFCCF2092C6000E940EAA60930A0878
:1092D00070930B0880930C0890930D08209106085A
:1092E000309107084091080850910908621B730BE0
:1092F000840B950B28EE33E040E050E00E9469B506
:10930000F22EE32ED42EC52EEDB7FEB738970FB64A
:10931000F894FEBF0FBEEDBF0DB71EB70F5F1F4F16
:10932000B282A182F80153824282622F732F842F6E
:10933000952F20E13EE040E050E00E9469B5F80141
:10934000358324836F2D7E2D8D2D9C2D2CE330E0D5
:1093500040E050E00E9469B5CA01B9012CE330E059
:1093600040E050E00E9469B5F801778366830E946F
:109370009510982DECE1F5E02DB73EB7285F3F4FF3
:109380000FB6F8943EBF0FBE2DBF08C08091C0003D
:1093900085FFFCCF9093C600319694919923B1F745
:1093A000F50107C08091C00085FFFCCF31969093F6
:1093B000C60090819923B1F78091C00085FFFCCF52
:1093C0002092C600C5010E94E49C87E495E00E94BB
:1093D000821A87E495E061E00E94E71B8091CE0944
:1093E000833211F49092DA092091D0093091D10999
:1093F0002115310519F41092CF09C4C08091D2090A
:109400009091D309869DF001879DF00D969DF00DFA
:109410001124E20FF31FE25BF74F1082FC01EC5BBB
:10942000F74F90822091D8093091D9092F5F3F4F93
:109430003093D9092093D809019664E070E00E9426
:1094400056B59093D3098093D2091092CF09109208
:10945000D1091092D0093AC04B3311F49092CF0940
:109460008091CF09882391F52091D0093091D109BD
:109470008091D2099091D309869DF001879DF00DCE
:10948000969DF00D1124E20FF31FE25BF74F8091E0
:10949000CE0980832F5F3F4F3093D1092093D009AD
:1094A00015C010E6612E712C99249394E6E1F8E042
:1094B0003490BAE02B2E5E010894A11CB11CA2E0EE
:1094C0004A2EA8E05A2EECE1F5E084902091CA07DC
:1094D0003091CB074091CC075091CD078091C207C6
:1094E0009091C307A091C407B091C5072817390709
:1094F0004A075B0708F046C08091D8099091D909C6
:1095000004970CF03FC08091DA098823D9F5809147
:109510001D0790911E07A0911F07B091200780930F
:10952000CA079093CB07A093CC07B093CD0785E1F2
:1095300097E00E94266B9C01482F8093CE098A30C9
:1095400009F083CE97CE8091D2099091D3098A9D5C
:1095500080018B9D100D9A9D100D1124C801825B16
:10956000974F6AE270E00E9466109C01009709F430
:109570001CCDFF2440E0C801CFCC80914905882351
:1095800009F052CE6E960FB6F894DEBF0FBECDBF77
:10959000CF91DF911F910F91FF90EF90DF90CF90CF
:1095A000BF90AF909F908F907F906F905F904F9003
:1095B0003F902F900895CF93DF938091D809909199
:1095C000D90903970CF4D4DB87E495E060E00E94AE
:1095D000E71B8091D8099091D909892B09F46AC0B9
:1095E00080914705882309F44DC0209142083091AD
:1095F000430880E690E0289FE001299FD00D389F26
:10960000D00D1124C25BD74FCE016CE679E00E94E9
:109610002B10892BE1F487E495E0BE010E947814B9
:1096200080914805882371F5E9E6F9E0949108C036
:109630008091C00085FFFCCF9093C6003196949135
:109640009923B1F78091C00085FFFCCF17C087E454
:1096500095E060E00E945F14E7E5F9E0949108C0AE
:109660008091C00085FFFCCF9093C6003196949105
:109670009923B1F78091C00085FFFCCF8AE08093E9
:10968000C60002C00E94F82E8091D8099091D90995
:1096900001979093D9098093D809809142089091BD
:1096A0004308019664E070E00E9456B59093430829
:1096B000809342080E940F820E946D290E947F7D44
:1096C0000E94C19EDF91CF910895DF93CF930F92B7
:1096D0000F92CDB7DEB70E940429269A2E9886E411
:1096E00095E040E052EC61E070E00E94B125E9E5D0
:1096F000FAE0949108C08091C00085FFFCCF909360
:10970000C600319694919923B1F78091C00085FFEE
:10971000FCCF8AE08093C6004CE155E0FA019491B9
:1097200008C08091C00085FFFCCF9093C6003196A1
:1097300094919923B1F784B7282F80FF15C0E1E5F4
:10974000FAE0949108C08091C00085FFFCCF90930F
:10975000C600319694919923B1F78091C00085FF9E
:10976000FCCF8AE08093C60021FF15C0E1E4FAE057
:10977000949108C08091C00085FFFCCF9093C600F3
:10978000319694919923B1F78091C00085FFFCCF69
:109790008AE08093C60022FF15C0E0E3FAE09491CE
:1097A00008C08091C00085FFFCCF9093C600319621
:1097B00094919923B1F78091C00085FFFCCF8AE096
:1097C0008093C60023FF15C0E0E2FAE0949108C040
:1097D0008091C00085FFFCCF9093C6003196949194
:1097E0009923B1F78091C00085FFFCCF8AE0809378
:1097F000C60025FF15C0E0E1FAE0949108C0809111
:10980000C00085FFFCCF9093C600319694919923B8
:10981000B1F78091C00085FFFCCF8AE08093C6003D
:1098200014BEE8E0FAE0949108C08091C00085FF82
:10983000FCCF9093C600319694919923B1F7E2E062
:10984000FAE0949108C08091C00085FFFCCF90930E
:10985000C600319694919923B1F78091C00085FF9D
:10986000FCCF8AE08093C600FA019491ECE1F5E028
:1098700008C08091C00085FFFCCF9093C600319650
:1098800094919923B1F7E2EFF9E0949108C08091A7
:10989000C00085FFFCCF9093C60031969491992328
:1098A000B1F7EDEDF9E0949108C08091C00085FF1B
:1098B000FCCF9093C600319694919923B1F7E1EDD6
:1098C000F9E0949108C08091C00085FFFCCF90938F
:1098D000C600319694919923B1F7EDEAF9E094919D
:1098E00008C08091C00085FFFCCF9093C6003196E0
:1098F00094919923B1F78091C00085FFFCCF8AE055
:109900008093C600E2EAF9E0949108C08091C0001B
:1099100085FFFCCF9093C600319694919923B1F7BF
:10992000E6E9F9E0949108C08091C00085FFFCCF82
:109930009093C600319694919923B1F78091C0001D
:1099400085FFFCCF8AE08093C600FA019491ECE198
:10995000F5E008C08091C00085FFFCCF9093C60061
:10996000319694919923B1F7E7E8F9E0949108C012
:109970008091C00085FFFCCF9093C60031969491F2
:109980009923B1F72091181330911913CE01019644
:109990002115310519F48E51934102C0821B930B9E
:1099A0009A83898369817A8186E495E04AE050E070
:1099B0000E94F826E0E7F9E0949108C08091C00089
:1099C00085FFFCCF9093C600319694919923B1F70F
:1099D00086E495E060ED74E04AE050E00E94F826ED
:1099E0008091C00085FFFCCF8AE08093C600109272
:1099F00044081092450810924608109247080E94A9
:109A000099200E9446220E9482810E946B550E94EA
:109A10003E750E94F19D80E197E220E931E0F90175
:109A20003197F1F70197D9F70F900F90CF91DF9110
:109A30000895BC018091D8099091D90904970CF040
:109A400070C02091D2093091D30980E690E0AC013A
:109A5000249FC001259F900D349F900D1124825B9F
:109A6000974F0E94FD0FECE1F5E0949108C08091C2
:109A7000C00085FFFCCF9093C60031969491992346
:109A8000B1F7E1E6FAE0949108C08091C00085FF4B
:109A9000FCCF9093C600319694919923B1F7209111
:109AA000D2093091D30980E690E0289FF001299FE8
:109AB000F00D389FF00D1124E25BF74F07C0809145
:109AC000C00085FFFCCF31969093C600908199230A
:109AD000B1F7EFE5FAE0949108C08091C00085FFEE
:109AE000FCCF9093C600319694919923B1F7809161
:109AF000C00085FFFCCF8AE08093C600C9010196B3
:109B000064E070E00E9456B59093D3098093D20927
:109B10008091D8099091D90901969093D9098093A1
:109B2000D8090895BC018091D8099091D90904976A
:109B30000CF070C02091D2093091D30980E690E0FA
:109B4000AC01249FC001259F900D349F900D1124DE
:109B5000825B974F0E947110ECE1F5E0949108C090
:109B60008091C00085FFFCCF9093C6003196949100
:109B70009923B1F7EEE6FAE0949108C08091C00015
:109B800085FFFCCF9093C600319694919923B1F74D
:109B90002091D2093091D30980E690E0289FF0010E
:109BA000299FF00D389FF00D1124E25BF74F07C09D
:109BB0008091C00085FFFCCF31969093C6009081C4
:109BC0009923B1F7ECE6FAE0949108C08091C000C7
:109BD00085FFFCCF9093C600319694919923B1F7FD
:109BE0008091C00085FFFCCF8AE08093C600C90148
:109BF000019664E070E00E9456B59093D30980937B
:109C0000D2098091D8099091D90901969093D909E8
:109C10008093D80908952F923F924F925F926F924E
:109C20007F928F929F92AF92BF92CF92DF92EF92EC
:109C3000FF920F931F93DF93CF93CDB7DEB7CD5530
:109C4000D0400FB6F894DEBF0FBECDBF2F969FAFAA
:109C50008EAF2F9761967FAF6EAF61972A016296A4
:109C60002FAF629763960FAF63976496EFAE6497DA
:109C70006896ACAEBDAECEAEDFAE6897E22EFF24E6
:109C8000EE0CFF1CEE0CFF1C9A012E0D3F1D2D96B5
:109C90003FAF2EAF2D97D9016D907D908D909C9008
:109CA000FC01EE0DFF1DC401B30120813181428111
:109CB00053810E9498B069AF7AAF8BAF9CAF10E030
:109CC000000F111F000F111FF201E00FF11F2B9663
:109CD000FFAFEEAF2B97A080B180C280D3802F96CC
:109CE000EEADFFAD2F97E00FF11FC601B50120814A
:109CF0003181428153810E9498B06DAB7EAB8FABB6
:109D000098AF64962FAD6497E22FF0E0EE0FFF1F3F
:109D1000EE0FFF1F2F96AEADBFAD2F97AE0FBF1F3B
:109D20004D915D916D917C9129964CAF5DAF6EAF79
:109D30007FAF299761966EAD7FAD6197E60FF71FF4
:109D4000608171818281938129962CAD3DAD4EADAC
:109D50005FAD29970E9497B069AB7AAB8BAB9CAB98
:109D60006196AEADBFAD61971C968D919D910D90A2
:109D7000BC91A02D25968CAF9DAFAEAFBFAF259700
:109D80002F96AEADBFAD2F971C962D913D914D9165
:109D90005C911F9721962CAF3DAF4EAF5FAF2197DF
:109DA000A401930150582DA73EA74FA758ABB60169
:109DB000A501705849A75AA76BA77CA761966EADFD
:109DC0007FAD6197E60EF71ED7016D917D918D9164
:109DD0009C9129AD3AAD4BAD5CAD0E9497B03B0173
:109DE0004C016196EEADFFAD61970E0F1F1FD801BC
:109DF0006D917D918D919C912DA93EA94FA958AD52
:109E00000E9497B05B016C016DA57EA58FA598A9F6
:109E1000A60195010E9451B47B018C0169A57AA528
:109E20008BA59CA5A40193010E9451B49B01AC0198
:109E3000C801B7010E9497B01B012C016DA57EA53A
:109E40008FA598A9A40193010E9451B47B018C01B4
:109E500069A57AA58BA59CA5A60195010E9451B480
:109E60009B01AC01C801B7010E9498B09B01AC01F5
:109E7000C201B1010E940BB15B016C0120E030E036
:109E800040E050E00E9471B1882354F4C601B5014E
:109E90002BED3FE049EC50E40E9498B05B016C016F
:109EA000E8968FADE897882351F0C601B5012BEDF8
:109EB0003FE049EC50E40E9497B05B016C01C601A1
:109EC000B501E7962CAD3DAD4EAD5FADE7970E9475
:109ED00051B429A93AA94BA95CA95F770E948CB318
:109EE0007B018C012FE632E143E85AE30E9471B115
:109EF00087FDF4C1C801B7010E944EB20E94E5B1CE
:109F000078A76FA3672B21F4E1E0F0E0F8A7EFA3B7
:109F10002FA138A5B90180E090E00E9411B27B0129
:109F20008C01C601B501A80197010E9478B16BA30D
:109F30007CA38DA39EA369A97AA98BA99CA9A8013A
:109F400097010E9478B16F8F78A389A39AA3259671
:109F50006CAD7DAD8EAD9FAD259721962CAD3DAD01
:109F60004EAD5FAD21970E9497B0A80197010E9466
:109F700078B16B8F7C8F8D8F9E8F6BA17CA18DA113
:109F80009EA120E030E040E05FEB0E9451B42BA1A5
:109F90003CA14DA15EA10E9451B420E030E040E818
:109FA0005FE30E9498B06F8B788F898F9A8F649649
:109FB0003FAD6497E32FF0E0EE0FFF1FEE0FFF1FA2
:109FC0009E012F5F3F4FE20FF31F29964CAD5DAD11
:109FD0006EAD7FAD299740835183628373832F9643
:109FE000AEADBFAD2F971C964D915D916D917C915B
:109FF0001F974D875E876F87788B41E050E05A8BC3
:10A00000498B662462967FAD6297672F70E0660F7A
:10A01000771F660F771FC901860F971F6A969FAF3C
:10A020008EAF6A976396BFAD6397AB2FB0E0AA0F70
:10A03000BB1FAA0FBB1F21E030E02C0F3D1F2A0FD2
:10A040003B1F6C963FAF2EAF6C976E96FFAFEEAF97
:10A050006E9719C138E136150CF446C06DA57EA582
:10A060008FA598A92BA13CA14DA15EA10E9451B43E
:10A070007B018C0169A57AA58BA59CA52F89388DBC
:10A08000498D5A8D0E9451B49B01AC01C801B701A2
:10A090000E9498B07B018C016DA57EA58FA598A923
:10A0A0002F89388D498D5A8D0E9451B45B016C0106
:10A0B00069A57AA58BA59CA52BA13CA14DA15EA16C
:10A0C0000E9451B49B01AC01C601B5010E9497B03A
:10A0D0006DA77EA78FA798AB6394C701D80189A706
:10A0E0009AA7ABA7BCA765C049895A89BA0180E085
:10A0F00090E00E9411B22BA13CA14DA15EA10E9453
:10A1000051B47B018C01C8010E9475B16B8B7C8BB3
:10A110008D8B9E8BB701C8010E94B4B43B014C01EA
:10A120002D96AEADBFAD2D97ED90FD900D911C918C
:10A1300017FB109517F910952B96EEADFFAD2B97E9
:10A140002080318042805380C801B7012B893C892F
:10A150004D895E890E9451B45B016C01C201B1015D
:10A16000A40193010E9451B49B01AC01C601B50149
:10A170000E9498B06DA77EA78FA798ABC801B701C2
:10A18000A40193010E9451B47B018C01C201B10171
:10A190002B893C894D895E890E9451B49B01AC0199
:10A1A000C801B7010E9497B069A77AA78BA79CA79F
:10A1B000662469AD7AAD8BAD9CAD2DA53EA54FA5AE
:10A1C00058A90E9498B06A96AEADBFAD6A976D93DC
:10A1D0007D938D939C9313976DA97EA98FA998ADBC
:10A1E00029A53AA54BA55CA50E9498B06C96EEAD4A
:10A1F000FFAD6C9760837183828393836E96AEAD5F
:10A20000BFAD6E976D917D918D919C912F8D38A1F1
:10A2100049A15AA10E9498B06E96EEADFFAD6E971F
:10A2200060837183828393836D857E858F85988912
:10A230002B8D3C8D4D8D5E8D0E9498B06D877E87F5
:10A240008F87988BCE0101960E94CD27CE01019673
:10A25000BE016B5F7F4FAE01475F5F4F9E01235F83
:10A260003F4F6896ECACFDAC0EAD1FAD6897F8E7BC
:10A27000CF2ED12CCC0EDD1EF1D629893A892F5F45
:10A280003F4F3A8B298B49895A896FA178A5461788
:10A29000570708F4DFCE61964EAD5FAD6197485F1A
:10A2A0005F4F61962EAD3FAD6197245F3F4F619642
:10A2B0008EAD9FAD6197DC0114966196BFAFAEAFD6
:10A2C0006197BD016896ECACFDAC0EAD1FAD689713
:10A2D000E8E7CE2ED12CCC0EDD1EC0D6C35ADF4F00
:10A2E0000FB6F894DEBF0FBECDBFCF91DF911F91A7
:10A2F0000F91FF90EF90DF90CF90BF90AF909F9025
:10A300008F907F906F905F904F903F902F90089527
:10A310003F924F925F926F927F928F929F92AF92F5
:10A32000BF92CF92DF92EF92FF920F931F93CF9342
:10A33000DF9380914B0A882309F4F6C08090AB0329
:10A340009090AC03A090AD03B090AE0360918E11DD
:10A3500070918F11882777FD8095982F0E9413B2F6
:10A3600020E030E040E050E40E9498B0A501940164
:10A370000E9471B187FDD8C030901D0F0F2EF0E004
:10A380004F2EF0E05F2EF0E06F2EF0E07F2EF02DEC
:10A39000CDE4D0E058C0232D30E02C9FF0012D9F5C
:10A3A000F00D3C9FF00D1124E45BF54F808191810D
:10A3B000A281B3810097A105B10581F484819581C3
:10A3C000A681B7810097A105B10541F480859185EB
:10A3D000A285B3850097A105B10591F12C9F60017D
:10A3E0002D9FD00C3C9FD00C11248CE49AE0C80E19
:10A3F000D91EF60164857585868597850E9413B2FE
:10A400007B018C01F60160897189828993890E94A0
:10A4100011B29B01AC01C801B7010E9478B1F601ED
:10A4200022A133A144A155A10E9451B47B018C010A
:10A43000A30192010E947FB3181614F4270138017A
:10A440003394FFE03F2280911C0F381609F0A3CF10
:10A45000C301B2012091AF033091B0034091B10329
:10A460005091B2030E9451B49B01AC01C501B401EB
:10A470000E9498B07B018C01A50194010E9471B1EA
:10A4800087FD02C0470158011091A7030091A8035E
:10A49000F090A903E090AA03C501B401212F302F49
:10A4A0004F2D5E2D0E947FB3181634F4812F902F0C
:10A4B000AF2DBE2D4C015D014090320F5090330FF7
:10A4C0006090340F7090350FC301B201A501940163
:10A4D0000E947FB31816C4F4C501B40120E037ED23
:10A4E00043EA5CE30E9451B47B018C01C301B201D9
:10A4F00028E431EE4AE75FE30E9451B4A8019701D6
:10A500000E9498B04B015C018092320F9092330F01
:10A51000A092340FB092350FC501B4010E94E0B192
:10A5200070938F1160938E11DF91CF911F910F91D6
:10A53000FF90EF90DF90CF90BF90AF909F908F9063
:10A540007F906F905F904F903F90089580911C0F87
:10A5500090911D0F891B8F7008956093B3037093C2
:10A56000B4038093B5039093B60308950F931F939C
:10A57000CF93DF93C0E0D0E08E01055D154FFE0163
:10A58000E150F64F60817181828193810E9411B206
:10A59000FE01E151F64F20813181428153810E94B9
:10A5A00051B40E94E5B1F801608371838283938383
:10A5B0002496C031D10501F7DF91CF911F910F9102
:10A5C0000895FC0160817181828193812091FB0952
:10A5D0003091FC094091FD095091FE090E9451B44F
:10A5E0000E9421B46093470A7093480A8093490AF5
:10A5F00090934A0A87E49AE00C9406768F929F9291
:10A60000AF92BF92CF92DF92EF92FF920F931F9380
:10A61000FC018B015A014901608171818281938122
:10A620002091EF093091F0094091F1095091F20920
:10A630000E9451B40E9421B43BE3C32E3AE0D32ED2
:10A6400060933B0A70933C0A80933D0A90933E0AC4
:10A65000F80160817181828193812091F3093091A9
:10A66000F4094091F5095091F6090E9451B40E94F5
:10A6700021B424E0E22EF12CEC0CFD1C60933F0A87
:10A68000F701718382839383F501608171818281F7
:10A6900093812091F7093091F8094091F90950917F
:10A6A000FA090E9451B40E9421B48601085F1F4F2D
:10A6B0006093430AF801718382839383F40160817C
:10A6C0007181828193812091FB093091FC09409135
:10A6D000FD095091FE090E9451B40E9421B4F60177
:10A6E0003C966093470A718382839383C601B701C6
:10A6F000A8019F010E94CC7580E090E0A0E0B0E04E
:10A7000080931E0F90931F0FA093200FB093210FE3
:10A710008093220F9093230FA093240FB093250FC3
:10A720008093260F9093270FA093280FB093290FA3
:10A7300080932A0F90932B0FA0932C0FB0932D0F83
:10A7400080932E0F90932F0FA093300FB093310F63
:10A750001F910F91FF90EF90DF90CF90BF90AF903F
:10A760009F908F9008958F929F92AF92BF92CF92B9
:10A77000DF92EF92FF920F931F93CF93DF93EC0141
:10A780006B01009709F45CC08FA9882309F058C0B9
:10A79000EEA0FFA008A519A5FB01B6A0A7A090A454
:10A7A00081A4C801B7012B2D3A2D492D582D0E94A7
:10A7B00071B188230CF044C0C801B701A80197010A
:10A7C0000E9451B47B018C016AA97BA98CA99DA927
:10A7D000905820E030E040E050EC0E9451B42EA5AB
:10A7E0003FA548A959A90E9451B49B01AC01C801D9
:10A7F000B7010E9498B00E94BEB47B018C016B2D02
:10A800007A2D892D982D9701A8010E9471B1882376
:10A8100024F4EB2CFA2C092D182D6B2D7A2D892D73
:10A82000982D9701A8010E9471B1882349F0C701B2
:10A83000D801F60186A397A3A0A7B1A781E086ABB4
:10A84000DF91CF911F910F91FF90EF90DF90CF900C
:10A85000BF90AF909F908F900895EF92FF920F93CB
:10A860001F93CF93DF93F0901D0F00E010E020E0E6
:10A8700030E04DE4E42E11C0FE9CE0011124C45BE5
:10A88000D54FC901B801AE016EDF8F2D8F5F8031CA
:10A8900009F480E0F82E98018E0180911C0FF816C3
:10A8A00059F7C901B80140E050E05DDFDF91CF9179
:10A8B0001F910F91FF90EF900895AF92BF92CF92AA
:10A8C000DF92EF92FF920F931F93CF93DF93EB01F1
:10A8D0008A016115710509F466C04115510509F435
:10A8E00062C0DAA4CBA4BCA4ADA46EA17FA188A54C
:10A8F00099A52D2D3C2D4B2D5A2D0E9471B18823E9
:10A9000009F451C08FA9882309F043C0F801E6A0DB
:10A91000F7A000A511A56D2D7C2D8B2D9A2DA801DA
:10A9200097010E947FB31816A4F5C801B701A801CA
:10A9300097010E9451B47B018C016AA97BA98CA963
:10A940009DA9905820E030E040E050EC0E9451B4C6
:10A950002EA53FA548A959A90E9451B49B01AC015D
:10A96000C801B7010E9498B00E94BEB47B018C015F
:10A970006D2D7C2D8B2D9A2D9701A8010E9471B110
:10A98000882324F4ED2CFC2C0B2D1A2DC701D801A3
:10A9900004C08D2D9C2DAB2DBA2D8EA39FA3A8A7EF
:10A9A000B9A781E08EABDF91CF911F910F91FF90FE
:10A9B000EF90DF90CF90BF90AF900895CF92DF924D
:10A9C000EF92FF920F93DF93CF930F920F92CDB739
:10A9D000DEB780911C0F8FB7F894F0901D0F8FBFDA
:10A9E00080911C0F90E040968F1991098F709070A4
:10A9F0000497FCF000911C0F03500F70CC24DD2451
:10AA000040E050E06DE4E62E12C0802F002309F4F0
:10AA100080E1082F01500E9DC0011124845B954FE9
:10AA20009A838983B60149DFA601C980DA800F15B0
:10AA300061F70F900F90CF91DF910F91FF90EF9002
:10AA4000DF90CF9008956091040890911D0F809140
:10AA50001C0F981711F4362F30C040911D0F242F72
:10AA600030E08DE490E0289FF001299FF00D389FA1
:10AA7000F00D1124EC56F54F308120E06DE470E0CC
:10AA800016C0842F90E0869FF001879FF00D969F5F
:10AA9000F00D1124E45BF54F80859185A285B38587
:10AAA0000097A105B10509F02F5F4F5F4F708091AE
:10AAB0001C0F481731F7222341F49FB7F894809177
:10AAC00008018160809308019FBF89E0632F70E0D7
:10AAD0000E94E1AA1DCC10921C0F10921D0F80E164
:10AAE000EBE3FAE0DF011D928A95E9F780E090E060
:10AAF000A0E0B0E08093220F9093230FA093240F47
:10AB0000B093250F8093260F9093270FA093280FC3
:10AB1000B093290F80932A0F90932B0FA0932C0FA3
:10AB2000B0932D0F80932E0F90932F0FA093300F83
:10AB3000B093310F80931E0F90931F0FA093200F9F
:10AB4000B093210F08952F923F924F925F926F9290
:10AB50007F928F929F92AF92BF92CF92DF92EF92AD
:10AB6000FF920F931F93DF93CF93CDB7DEB7669716
:10AB70000FB6F894DEBF0FBECDBF9E8B8D8B6A01E2
:10AB80007B0148015901DC01D8966D917D918D9131
:10AB90009C91DB970E9411B2698B7A8B8B8B9C8B7B
:10ABA000A70196010E9451B40E945EB10E94E5B1D6
:10ABB0006D837E838F83988769897A898B899C8945
:10ABC000A50194010E9451B40E945EB10E94E5B1BA
:10ABD00069837A838B839C832D813E814F81588545
:10ABE000283731054105510540F448E750E060E061
:10ABF00070E04D835E836F83788769817A818B8172
:10AC00009C81683771058105910540F488E790E0E3
:10AC1000A0E0B0E089839A83AB83BC83AD89BE8911
:10AC2000AC5BBF4FAD90BD90CD90DC901397A4541A
:10AC3000B040BE8BAD8BDC966D917D918D919C91DA
:10AC4000DF970E9411B26D877E878F87988BC60130
:10AC5000B5010E9413B21B012C0120E030E040E05E
:10AC600050E00E9471B1882321F4E0E070E060E0E0
:10AC700028C069897A898B899C899B01AC010E94D3
:10AC800051B47B018C016D857E858F8598899B01F0
:10AC9000AC010E9451B49B01AC01C801B7010E94F4
:10ACA00097B07B018C01C201B101A20191010E9408
:10ACB00098B09B01AC01C801B7010E9478B1E62FA2
:10ACC000692F2E2F372F482F562FB901CA010E9406
:10ACD0005EB10E94E0B13B014C01ED89FE89E05C70
:10ACE000FF4F60817181828193810E9411B26987D7
:10ACF0007A878B879C8766277727CB016A197B0920
:10AD00008C099D090E9413B25B016C0120E030E0C8
:10AD100040E050E00E9471B1882321F4E0E070E04F
:10AD200060E028C069857A858B859C859B01AC0194
:10AD30000E9451B47B018C0169897A898B899C8935
:10AD40009B01AC010E9451B49B01AC01C801B70149
:10AD50000E9497B07B018C01C601B501A601950147
:10AD60000E9498B09B01AC01C801B7010E9478B164
:10AD7000E62F692F2E2F372F482F562FB901CA01E2
:10AD80000E944EB2ED89FE89A088B188C288D3881E
:10AD900086017501E618F708080919090E94E0B153
:10ADA000A8019701261B370B480B590B57FF71C0A1
:10ADB000C201B10120E030E040E050E00E9471B1FA
:10ADC000882321F4E0E070E060E044C0C201B101FA
:10ADD000A20191010E9498B07B018C01C601B501CE
:10ADE0000E9411B29B01AC01C801B7010E9451B48D
:10ADF0007B018C016D857E858F8598899B01AC01D7
:10AE00000E9451B49B01AC01C801B7010E9497B0E8
:10AE10007B018C0169857A858B859C859B01AC01C2
:10AE20000E9451B49B01AC01C801B7010E9498B0C7
:10AE30007B018C01C201B10120E030E040E850E428
:10AE40000E9451B49B01AC01C801B7010E9478B1C6
:10AE5000E62F692F2E2F372F482F562FB901CA0101
:10AE60000E945EB10E94E0B1AC01CB01DA013C016D
:10AE70004D0197FE03C06624772443016A147B04C6
:10AE80008C049D0410F03501460120E030E040E0E4
:10AE900050E09FB7F8946D897E89645B7F4FDB013A
:10AEA0008C91AC54B040BE8BAD8B882321F5FD0155
:10AEB000648A758A868A978A260D371D481D591D12
:10AEC00058962D933D934D935C935B972D813E81D6
:10AED0004F815885DC962D933D934D935C93DF977E
:10AEE000A05CBF4F29813A814B815C812D933D93BA
:10AEF0004D935C9313979FBF66960FB6F894DEBF91
:10AF00000FBECDBFCF91DF911F910F91FF90EF90BA
:10AF1000DF90CF90BF90AF909F908F907F906F9079
:10AF20005F904F903F902F9008954F925F927F9245
:10AF30008F929F92AF92BF92CF92DF92EF92FF9249
:10AF40000F931F93CF93DF9370901D0FC0E0D0E05D
:10AF50007DE4472E512C45C02097A9F18EA9882366
:10AF600061F4849CF001859CF00D949CF00D1124FB
:10AF7000E45BF54F86A9882331F1EAA0FBA00CA180
:10AF80001DA16EA17FA188A599A5A80197010E9486
:10AF900078B15B016C01849CF001859CF00D949C60
:10AFA000F00D1124E45BF54F66A177A180A591A572
:10AFB000A80197010E9478B18B019C01CE01B601D6
:10AFC000A501C1DD1EAA739480E1781609F47724E7
:10AFD000849CE001859CD00D949CD00D1124C45B11
:10AFE000D54F872C992487FC909480911C0F90E07A
:10AFF0008816990609F0B0CF2097E9F0EAA0FBA0E7
:10B000000CA11DA16EA17FA188A599A5A8019701FA
:10B010000E9478B15B016C016DEC7CEC8CE49DE3EB
:10B02000A80197010E9478B18B019C01CE01B60165
:10B03000A50189DD1EAADF91CF911F910F91FF908D
:10B04000EF90DF90CF90BF90AF909F908F907F90C8
:10B050005F904F900895B2DC00DC67CF2F923F9253
:10B060004F925F926F927F928F929F92AF92BF9218
:10B07000CF92DF92EF92FF920F931F93DF93CF93C4
:10B08000CDB7DEB7C859D0400FB6F894DEBF0FBEBB
:10B09000CDBF5C014B013A012901CB56DF4FE8825D
:10B0A000C559D040CA56DF4FF882C659D040C9565C
:10B0B000DF4F0883C759D040C856DF4F1883C8599F
:10B0C000D040E396DFAECEAEE39780911C0F8F5F4A
:10B0D000803109F480E0282F332727FD30953CA7E5
:10B0E0002BA706C00E940F820E946D290E94C19E5C
:10B0F00080911D0F90E04BA55CA58417950791F3F7
:10B100006091EF097091F0098091F1099091F20935
:10B11000E1966CAF7DAF8EAF9FAFE197D5012D91DA
:10B120003D914D915C910E9451B40E9421B4C1584F
:10B13000DF4F6883CF57D040C058DF4F7883C05867
:10B14000D040CF57DF4F8883C158D040CE57DF4F14
:10B150009883C258D0402091F3093091F40940916E
:10B16000F5095091F609AD962CAF3DAF4EAF5FAFEC
:10B17000AD97CA01B901D4012D913D914D915C91DA
:10B180000E9451B40E9421B4CD57DF4F6883C35849
:10B19000D040CC57DF4F7883C458D040CB57DF4FD7
:10B1A0008883C558D040CA57DF4F9883C658D040CF
:10B1B0002091F7093091F8094091F9095091FA0965
:10B1C000A9962CAF3DAF4EAF5FAFA997CA01B901A9
:10B1D000D3012D913D914D915C910E9451B40E94FB
:10B1E00021B4C957DF4F6883C758D040C857DF4FD5
:10B1F0007883C858D040C757DF4F8883C958D0409C
:10B20000C657DF4F9883CA58D0402091FB09309130
:10B21000FC094091FD095091FE09A5962CAF3DAF68
:10B220004EAF5FAFA597CA01B901D2012D913D91F3
:10B230004D915C910E9451B40E9421B4C557DF4FDB
:10B240006883CB58D040C457DF4F7883CC58D04068
:10B25000C357DF4F8883CD58D040C257DF4F988304
:10B26000CE58D0408091470A9091480AA091490A4F
:10B27000B0914A0AC557DF4F288139814A815B81E5
:10B28000CB58D040281739074A075B0709F4B8C0E4
:10B29000E0910308F0E0EE0FFF1FEE0FFF1FEC56EA
:10B2A000FE4E60817181828193812091B303309140
:10B2B000B4034091B5035091B6030E9471B1882345
:10B2C0000CF033C0C557DF4F488159816A817B81BB
:10B2D000CB58D0404093470A5093480A6093490A9C
:10B2E00070934A0AE9E7FAE0949108C08091C0009F
:10B2F00085FFFCCF9093C600319694919923B1F7C6
:10B30000EDE9FAE0949108C08091C00085FFFCCF80
:10B310009093C600319694919923B1F78091C00023
:10B3200085FFFCCF8AE08093C6008091470A909108
:10B33000480AA091490AB0914A0AC557DF4F2881AF
:10B3400039814A815B81CB58D040281B390B4A0B8D
:10B350005B0BCA01B90157FF07C0909580957095A6
:10B3600061957F4F8F4F9F4F0E9413B27B018C01DD
:10B37000A5966CAD7DAD8EAD9FADA59720E030E874
:10B380004DEF53E40E9451B49B01AC01C801B701D9
:10B390000E947FB318160CF033C0C557DF4F4881A9
:10B3A00059816A817B81CB58D0404093470A5093A2
:10B3B000480A6093490A70934A0AE9E7FAE09491CF
:10B3C00008C08091C00085FFFCCF9093C6003196E5
:10B3D00094919923B1F7EFE7FAE0949108C0809136
:10B3E000C00085FFFCCF9093C600319694919923BD
:10B3F000B1F78091C00085FFFCCF8AE08093C60042
:10B4000080911C0F682F70E0A1967FAF6EAFA1975F
:10B410008DE490E0689FF001699FF00D789FF00D3A
:10B420001124E45BF54FE45BFF4F1082EC54F040D5
:10B4300080913B0A90913C0AA0913D0AB0913E0A4E
:10B440006F968CAF9DAFAEAFBFAF6F97C158DF4F58
:10B45000288139814A815B81CF57D040281B390B25
:10B460004A0B5B0B6B962CAF3DAF4EAF5FAF6B974C
:10B47000208331834283538357FF0DC0DA01C90112
:10B48000B095A095909581959F4FAF4FBF4F80830A
:10B490009183A283B38340913F0A5091400A609107
:10B4A000410A7091420A67964CAF5DAF6EAF7FAFB5
:10B4B0006797CD57DF4F88819981AA81BB81C35897
:10B4C000D040841B950BA60BB70B63968CAF9DAF3A
:10B4D000AEAFBFAF63978DE490E0A196AEADBFADC8
:10B4E000A197A89FF001A99FF00DB89FF00D11241E
:10B4F000E45BF54F63962CAD3DAD4EAD5FAD63970C
:10B50000248335834683578357FF0DC0DA01C90171
:10B51000B095A095909581959F4FAF4FBF4F848375
:10B520009583A683B7834091430A5091440A609162
:10B53000450A7091460A2F964CAF5DAF6EAF7FAF54
:10B540002F97C957DF4F88819981AA81BB81C7583E
:10B55000D040841B950BA60BB70B2B968CAF9DAFE1
:10B56000AEAFBFAF2B978DE490E0A196AEADBFAD6F
:10B57000A197A89FF001A99FF00DB89FF00D11248D
:10B58000E45BF54F2B962CAD3DAD4EAD5FAD2B97EB
:10B59000208731874287538757FF0DC0DA01C901E1
:10B5A000B095A095909581959F4FAF4FBF4F8087E5
:10B5B0009187A287B3872090470A3090480A40902D
:10B5C000490A50904A0AC557DF4F488159816A811C
:10B5D0007B81CB58D04042195309640975094DA3AA
:10B5E0005EA36FA378A760918E0370918F03279657
:10B5F0007FAF6EAF27976DA17EA18FA198A597FF12
:10B6000007C090958095709561957F4F8F4F9F4FA4
:10B610002796AEADBFAD27979D01442737FD4095D6
:10B62000542F0E9423B524E630E040E050E00E9411
:10B630008BB58DE490E0A1966EAD7FADA197689F2C
:10B64000F001699FF00D789FF00D1124E45BF54F38
:10B65000DF011C96248711963C93119712964C9308
:10B66000129713965C936080718082809380A4808F
:10B67000B580C680D780E084F18402851385C90136
:10B68000DA018E159F05A007B10714F4D801C70190
:10B690008A159B05AC05BD0514F4D601C5019C01B6
:10B6A000AD0186159705A805B90514F4A401930109
:10B6B0008DE490E0A196AEADBFADA197A89FB0017B
:10B6C000A99F700DB89F700D1124645B754FFB012D
:10B6D000208B318B428B538B263031054105510530
:10B6E00010F40C946764E85BFF4F8091040890911C
:10B6F0000508AA2797FDA095BA2F80839183A2837E
:10B70000B383DB0190961C92C158DF4F28813981A9
:10B710004A815B81CF57D0406F968CAD9DADAEAD69
:10B72000BFAD6F97281739074A075B0724F481E0FC
:10B73000DB0190968C93CD57DF4F288139814A8168
:10B740005B81C358D04067966CAD7DAD8EAD9FAD2B
:10B750006797261737074807590794F48DE490E058
:10B76000A196AEADBFADA197A89FF001A99FF00D26
:10B77000B89FF00D1124E45BF54F80A1826080A397
:10B78000C957DF4F288139814A815B81C758D04032
:10B790002F966CAD7DAD8EAD9FAD2F9726173707D9
:10B7A0004807590794F48DE490E0A196AEADBFAD83
:10B7B000A197A89FF001A99FF00DB89FF00D11244B
:10B7C000E45BF54F80A1846080A3C557DF4F2881DB
:10B7D00039814A815B81CB58D0402215330544051D
:10B7E000550594F48DE490E0A1964EAD5FADA19720
:10B7F000489FF001499FF00D589FF00D1124E45B24
:10B80000F54F80A1886080A38DE490E0A1966EAD95
:10B810007FADA197689FF001699FF00D789FF00DB3
:10B820001124E45BF54FE396AEADBFADE3978C9189
:10B8300081A3208131814281538125962CAF3DAF78
:10B840004EAF5FAF2597211531054105510509F030
:10B850005F988DE490E0A1964EAD5FADA197489FB3
:10B86000F001499FF00D589FF00D1124E45BF54F56
:10B8700064807580868097806114710481049104CE
:10B8800009F08A988DE490E0A1966EAD7FADA19706
:10B89000689FF001699FF00D789FF00D1124E45B23
:10B8A000F54FA084B184C284D384A114B104C1042F
:10B8B000D10441F09FB7F894809108018E7F809366
:10B8C00008019FBF8DE490E0A196AEADBFADA197FA
:10B8D000A89FF001A99FF00DB89FF00D1124E45B23
:10B8E000F54F84859585A685B7850097A105B10597
:10B8F00051F0129820900F0A3090100A4090110ACF
:10B900005090120A08C02090270A3090280A4090D0
:10B91000290A50902A0ACB56DF4F6881C559D0407A
:10B92000CA56DF4F7881C659D040C956DF4F88814B
:10B93000C759D040C856DF4F9881C859D040A2019E
:10B9400091010E9471B187FD16C0CB56DF4F8881EF
:10B95000C559D040CA56DF4F9881C659D040C95604
:10B96000DF4FA881C759D040C856DF4FB881C859AA
:10B97000D0401C012D016B966CAD7DAD8EAD9FADA1
:10B980006B970E9413B2E1962CAD3DAD4EAD5FAD0D
:10B99000E1970E9478B1EC966FAFEC97ED967FAF90
:10B9A000ED97EE968FAFEE97EF969FAFEF97AC01C6
:10B9B000CB01DA0189839A83AB83BC8363966CAD38
:10B9C0007DAD8EAD9FAD63970E9413B2AD962CAD49
:10B9D0003DAD4EAD5FADAD970E9478B1E8966FAFCB
:10B9E000E897E9967FAFE997EA968FAFEA97EB96EB
:10B9F0009FAFEB97AC01CB01DA018D839E83AF83C0
:10BA0000B8872B966CAD7DAD8EAD9FAD2B970E9408
:10BA100013B2A9962CAD3DAD4EAD5FADA9970E9476
:10BA200078B1E4966FAFE497E5967FAFE597E69639
:10BA30008FAFE697E7969FAFE797AC01CB01DA01AE
:10BA400089879A87AB87BC876DA17EA18FA198A5B6
:10BA50000E9413B2A5962CAD3DAD4EAD5FADA5973E
:10BA60000E9478B17B018C012796EEADFFAD279740
:10BA7000BF01882777FD8095982F0E9413B29B0104
:10BA8000AC01C801B7010E9451B420E030E048EC9D
:10BA900052E40E9478B19B01AC016D877E878F874D
:10BAA000988B25966CAD7DAD8EAD9FAD259766309C
:10BAB0007105810591051CF576E067167104810416
:10BAC0009104ECF486E0A816B104C104D104BCF4DE
:10BAD0008DE490E0A196AEADBFADA197A89FF00117
:10BAE000A99FF00DB89FF00D1124E45BF54FDA012A
:10BAF000C901BF7786A797A7A0ABB1AB55C0EC969D
:10BB00002FADEC97ED963FADED97EE964FADEE97DE
:10BB1000EF965FADEF97B901CA010E9408B53B01EE
:10BB20004C01E8962FADE897E9963FADE997EA9684
:10BB30004FADEA97EB965FADEB97B901CA010E9452
:10BB400008B55B016C01E4962FADE497E5963FAD37
:10BB5000E597E6964FADE697E7965FADE797B901B3
:10BB6000CA010E9408B57B018C01C401B301A60182
:10BB700095010E9498B0A80197010E9498B00E9478
:10BB8000BEB42DE430E0A1964EAD5FADA197429FCB
:10BB9000F001439FF00D529FF00D1124E45BF54F2F
:10BBA00066A777A780AB91AB8DE490E0A1966EADD0
:10BBB0007FADA197689FF001699FF00D789FF00D10
:10BBC0001124E45BF54F86A597A5A0A9B1A92196FC
:10BBD0008CAF9DAFAEAFBFAF219760E070E080E863
:10BBE0009FE321962CAD3DAD4EAD5FAD21970E94F8
:10BBF00078B19B01AC01C201B1010E9451B42B018B
:10BC00003C0180911C0F90911D0FA82FB0E0509621
:10BC1000A91BB109AF70B070BAA7A9A7A230B1052E
:10BC20000CF451C05D01CC24B7FCC094DC2CC601DF
:10BC3000B5010E9413B220E030E040E051E40E94E0
:10BC400071B188230CF03FC060E074E284E799E4AE
:10BC5000A30192010E9478B10E9421B47B018C0162
:10BC60006091DB097091DC098091DD099091DE091A
:10BC7000E616F7060807190730F56E197F09800BDD
:10BC8000910B660F771F881F991FA60195010E94CF
:10BC900069B5CA01B9010E9411B20E9421B49B0189
:10BCA000AC012E0D3F1D401F511FCA01B9010E945A
:10BCB00011B29B01AC0160E074E284E799E40E9458
:10BCC00078B12B013C018DE490E0A196EEADFFAD83
:10BCD000A197E89F8001E99F100DF89F100D112496
:10BCE000045B154F21966CAD7DAD8EAD9FAD219758
:10BCF000A30192010E9451B4D80192966D937D9355
:10BD00008D939C93959750966D917D918D919C917B
:10BD100053970E9411B2A30192010E9451B40E9454
:10BD20005EB10E94E5B1F80160AF71AF82AF93AF31
:10BD3000C157DF4F1882CF58D040C057DF4F18820D
:10BD4000C059D04020E8222E9FE3392E8824992420
:10BD5000E1E0F0E0EC0FFD1FE80DF91DC301B201B9
:10BD600020813181428153810E9451B4E1E1F0E0B0
:10BD7000EC0FFD1FE80DF91D6083718382839383AF
:10BD80005B016C01E894D7F8F401E152F64FE080D2
:10BD9000F18002811381C601B501A80197010E94BB
:10BDA0007FB31816CCF4C801B701A60195010E9413
:10BDB00078B16B017C01C157DF4F6881CF58D0400B
:10BDC000C057DF4F7881C059D040C101A70196010B
:10BDD0000E9471B188236CF4C157DF4F8881CF581E
:10BDE000D040C057DF4F9881C059D040D1016C017D
:10BDF0007D0124E030E0820E931E30E18316910431
:10BE000071F0D701C601C157DF4FC882CF58D0406B
:10BE1000C057DF4F9883C059D0401D0199CFC7014B
:10BE2000B60120E030E040E85FE30E9471B1882372
:10BE30000CF04CC08E010F5E1F4F81E2A82EB12C7A
:10BE4000AC0EBD1ED8016D917D918D919C91A70185
:10BE500096010E9451B4F80161937193819391937B
:10BE60008F01EA15FB0571F78DE490E0A1962EADE8
:10BE70003FADA197289F8001299F100D389F100D7D
:10BE80001124045B154FD80192966D917D918D918F
:10BE90009C919597A70196010E9451B4F80162A365
:10BEA00073A384A395A360AD71AD82AD93AD0E94E1
:10BEB00011B2A70196010E9451B40E94E5B1D801C8
:10BEC000D8966D937D938D939C93DB978DE490E052
:10BED000A196EEADFFADA197E89F8001E99F100DFF
:10BEE000F89F100D1124045B154FD80150966D91E9
:10BEF0007D918D919C9153970E9411B2F80126A5D6
:10BF000037A540A951A90E9478B11B012C01F80165
:10BF100080819181A281B3810097A105B10549F586
:10BF200084819581A681B7810097A105B10509F5A6
:10BF300080859185A285B3850097A105B105C9F4D7
:10BF4000C201B1012091170A3091180A4091190AD3
:10BF500050911A0A0E9451B40E945EB10C5B1F4FAF
:10BF60000E94E5B1D8016D937D938D939C931397B7
:10BF700071C1C201B1012091130A3091140A40919C
:10BF8000150A5091160A0E9451B40E945EB10E9497
:10BF9000E5B12DE430E0A196EEADFFADA197E29FB3
:10BFA0006001E39FD00CF29FD00C11242CE43AE006
:10BFB000C20ED31EB4E46B2E712C6C0C7D1CD3010D
:10BFC0006D937D938D939C93139780902B0A909003
:10BFD0002C0AA0902D0AB0902E0A0E9411B27B016B
:10BFE0008C01F60160817181828193810E9413B27C
:10BFF0009B01AC01C801B7010E9451B47B018C01C7
:10C00000D60150966D917D918D919C9153970E9490
:10C0100011B29B01AC01C801B7010E9478B17B014C
:10C020008C01C501B4010E9411B29B01AC01C80191
:10C03000B7010E947FB318162CF4F301808291821D
:10C04000A282B38280902F0A9090300AA090310A89
:10C05000B090320A8DE490E0A1962EAD3FADA1974D
:10C06000289F6001299FD00C389FD00C11244CE4EC
:10C070005AE0C40ED51EA4E46A2E712C6C0C7D1CF3
:10C08000D3016D917D918D919C910E9411B27B01A4
:10C090008C01F60164817581868197810E9413B2BB
:10C0A0009B01AC01C801B7010E9451B47B018C0116
:10C0B000D60150966D917D918D919C9153970E94E0
:10C0C00011B29B01AC01C801B7010E9478B17B019C
:10C0D0008C01C501B4010E9411B29B01AC01C801E1
:10C0E000B7010E947FB318162CF4F301808291826D
:10C0F000A282B3828090370A9090380AA090390AC1
:10C10000B0903A0A8DE490E0A1962EAD3FADA19794
:10C11000289F6001299FD00C389FD00C11244CE43B
:10C120005AE0C40ED51EF4E46F2E712C6C0C7D1CED
:10C13000D3016D917D918D919C910E9411B27B01F3
:10C140008C01F60164857585868597850E9413B2FA
:10C150009B01AC01C801B7010E9451B47B018C0165
:10C16000D60150966D917D918D919C9153970E942F
:10C1700011B29B01AC01C801B7010E9478B17B01EB
:10C180008C01C501B4010E9411B29B01AC01C80130
:10C19000B7010E947FB318162CF4F30180829182BC
:10C1A000A282B3828090330A9090340AA090350A1C
:10C1B000B090360A8DE490E0A1962EAD3FADA197E8
:10C1C000289F6001299FD00C389FD00C11244CE48B
:10C1D0005AE0C40ED51EE4E46E2E712C6C0C7D1C4E
:10C1E000D3016D917D918D919C910E9411B27B0143
:10C1F0008C01F60160857185828593850E9413B25A
:10C200009B01AC01C801B7010E9451B47B018C01B4
:10C21000D60150966D917D918D919C9153970E947E
:10C2200011B29B01AC01C801B7010E9478B17B013A
:10C230008C01C501B4010E9411B29B01AC01C8017F
:10C24000B7010E947FB318162CF4F301808291820B
:10C25000A282B3828DE490E0A1962EAD3FADA1976E
:10C26000289F6001299FD00C389FD00C11244CE4EA
:10C270005AE0C40ED51EF601EC5BFF4F6081718160
:10C28000828193810E9411B27B018C01A2019101F4
:10C290000E9478B1D601D2966D937D938D939C9335
:10C2A000D597C801B7012DEB37E346E051E40E9472
:10C2B00051B40E94E0B1F601648F758F868F978F1D
:10C2C00060901B0A70901C0A80901D0A90901E0AB4
:10C2D000C401B30120E030E040E05FE30E9451B4CC
:10C2E0005B016C01298D3A8D4B8D5C8D29AF3AAF86
:10C2F0004BAF5CAF40911F0A5091200A6091210A18
:10C300007091220A4DAB5EAB6FAB78AFCB01BA0137
:10C3100020E030E040E05FE30E9451B47B018C01FB
:10C3200069AD7AAD8BAD9CAD9F77A80197010E9456
:10C330007FB3181644F4C601B501A80197010E9405
:10C3400071B1882314F4860175016D8D7E8D8F8DFA
:10C3500098A169AB7AAB8BAB9CAB8091230A90918F
:10C36000240AA091250AB091260A8DA79EA7AFA7FF
:10C37000B8ABBC01CD0120E030E040E05FE30E94BB
:10C3800051B41B012C0169A97AA98BA99CA99F779B
:10C39000A20191010E947FB3181644F4C801B701AD
:10C3A000A20191010E9471B1882314F417012801A0
:10C3B0008DE490E0A196AEADBFADA197A89FF0012E
:10C3C000A99FF00DB89FF00D1124E45BF54F22A159
:10C3D00033A144A155A129A33AA34BA35CA3C20155
:10C3E000B1010E9471B187FD04C029A03AA04BA001
:10C3F0005CA049A55AA5423051050CF405C15091E5
:10C400001E0FCF56DF4F5883C159D04060911F0F88
:10C41000CE56DF4F6883C259D0407091200FCD5661
:10C42000DF4F7883C359D0408091210FCC56DF4F26
:10C430008883C459D040652FCE56DF4F7881C259CA
:10C44000D040CD56DF4F8881C359D040CC56DF4F06
:10C450009881C459D04027E137EB41ED58E30E9461
:10C460007FB318160CF0D0C069897A898B899C89B2
:10C470002091220F3091230F4091240F5091250FCE
:10C480000E9497B09B01AC010E9451B47B018C01CA
:10C490006D897E898F89988D2091260F3091270F85
:10C4A0004091280F5091290F0E9497B09B01AC0139
:10C4B0000E9451B49B01AC01C801B7010E9498B021
:10C4C0000E94BEB47B018C01A40193010E947FB342
:10C4D00018165CF00F2EF0E06F2EF0E07F2EF0E8E3
:10C4E0008F2EFFE39F2EF02D08C0C401B301A801D9
:10C4F00097010E9478B13B014C0169AD7AAD8BADDB
:10C500009CAD20912A0F30912B0F40912C0F509110
:10C510002D0F0E9497B07B018C01E89417F9C80198
:10C52000B7012DA93EA94FA958AD0E947FB3181697
:10C5300094F46DA97EA98FA998ADA80197010E94D6
:10C5400078B15B016C01C401B301A60195010E94A1
:10C5500071B1882314F46401530169A97AA98BA9E4
:10C560009CA920912E0F30912F0F4091300F5091A8
:10C57000310F0E9497B07B018C01E89417F9C80134
:10C58000B7012DA53EA54FA558A90E947FB3181647
:10C5900094F46DA57EA58FA598A9A80197010E9486
:10C5A00078B17B018C01C601B501A80197010E94F9
:10C5B00071B1882314F48601750169A17AA18BA158
:10C5C0009CA1A80197010E9451B47B018C01CF5618
:10C5D000DF4F6881C159D040CE56DF4F7881C259B4
:10C5E000D040CD56DF4F8881C359D040CC56DF4F65
:10C5F0009881C459D040A80197010E9471B187FD6C
:10C6000019C0D801C70102C0D201C101CF56DF4F06
:10C610008883C159D040CE56DF4F9883C259D0404D
:10C62000CD56DF4FA883C359D040CC56DF4FB883D7
:10C63000C459D0408DE490E0A196AEADBFADA197B6
:10C64000A89F8001A99F100DB89F100D1124045BB5
:10C65000154FCF56DF4F8881C159D040CE56DF4F9E
:10C660009881C259D040CD56DF4FA881C359D040E0
:10C67000CC56DF4FB881C459D040F80182A793A7A8
:10C68000A4A7B5A762A973A984A995A9905820E089
:10C6900030E040E050EC0E9451B4D8019E962D91BC
:10C6A0003D914D915C91D1970E9451B42BE037EDB3
:10C6B00043E25BE30E9498B00E94BEB4F62EE72EE0
:10C6C000D82EC92ECF56DF4F6881C159D040CE56E3
:10C6D000DF4F7881C259D040CD56DF4F8881C35992
:10C6E000D040CC56DF4F9881C459D0402F2D3E2DDD
:10C6F0004D2D5C2D0E9471B187FD14C0CF56DF4FC8
:10C70000F882C159D040CE56DF4FE882C259D0409E
:10C71000CD56DF4FD882C359D040CC56DF4FC882A8
:10C72000C459D0408DE490E0A196EEADFFADA19745
:10C73000E89F8001E99F100DF89F100D1124045B04
:10C74000154FCF56DF4F8881C159D040CE56DF4FAD
:10C750009881C259D040CD56DF4FA881C359D040EF
:10C76000CC56DF4FB881C459D040F80186A397A3B7
:10C77000A0A7B1A762A173A184A195A12F2D3E2DE1
:10C780004D2D5C2D0E9471B118162CF081E0D8015E
:10C79000D7968C9302C0F80117AA8DE490E0A19679
:10C7A0002EAD3FADA197289FF001299FF00D389F36
:10C7B000F00D1124E45BF54F81E086ABA2E2BFE00F
:10C7C000FE01719680E101900D928150E1F78DE4B8
:10C7D00090E0A1964EAD5FADA197489F6001499F43
:10C7E000D00C589FD00C11246CE47AE0C60ED71EF2
:10C7F000D6019296ED90FD900D911C919597E09247
:10C800001E0FF0921F0F0093200F1093210F96968A
:10C810006D917D918D919C919997A80197010E94AE
:10C8200078B14B015C01C201B101A80197010E94DE
:10C8300078B18B019C01C601B501A4010E94A355EA
:10C84000BBA5B0931C0FC557DF4F288139814A81A2
:10C850005B81CB58D0402093470A3093480A4093DD
:10C86000490A50934A0AC957DF4F488159816A8162
:10C870007B81C758D0404093430A5093440A609349
:10C88000450A7093460ACD57DF4F688179818A81C6
:10C890009B81C358D04060933F0A7093400A8093B5
:10C8A000410A9093420AC158DF4F88819981AA8139
:10C8B000BB81CF57D04080933B0A90933C0AA09312
:10C8C0003D0AB0933E0A0E942B580E943875C85604
:10C8D000DF4F0FB6F894DEBF0FBECDBFCF91DF9113
:10C8E0001F910F91FF90EF90DF90CF90BF90AF908E
:10C8F0009F908F907F906F905F904F903F902F9080
:10C900000895FF920F931F93CF93DF938B010E94A3
:10C910000EAAEB01FF24FA9409C00E940EAA6C1B18
:10C920007D0B6017710710F080E008C0FEBC0DB4ED
:10C9300007FEFDCF8EB58F3F81F781E0DF91CF916C
:10C940001F910F91FF900895FC014281242F30E048
:10C95000C9019595879580658CBD40FF02C080E038
:10C9600004C080E0463009F081E08DBD808160E048
:10C970000C9472ACDF92EF92FF920F931F93CF93C0
:10C98000DF93EC01D62E79018A01DEDFCE016CE265
:10C9900071E0B7DF8D2D80648EBD0DB407FEFDCF35
:10C9A00028E130E0D801C701022E04C0B695A79552
:10C9B000979587950A94D2F78EBD0DB407FEFDCFEB
:10C9C000285030408FEF283F380761F7DD2011F401
:10C9D00085E906C088E0D81611F487E801C08FEF1A
:10C9E0008EBD0DB407FEFDCF8CE0D81631F48FEF6D
:10C9F0008EBD0DB407FEFDCF8EB59FEF2FEF2EBD80
:10CA00000DB407FEFDCF8EB587FF04C0992311F04A
:10CA10009150F5CF8B83DF91CF911F910F91FF90B4
:10CA2000EF90DF900895FC01808161E00C9472AC7E
:10CA3000DC016EBDFA0120E030E00DB407FEFDCF51
:10CA400080818EBD0DB407FEFDCF81818EBD2E5F2E
:10CA50003F4F329682E02030380779F70DB407FE59
:10CA6000FDCF8FEF8EBD0DB407FEFDCF8FEF8EBDD6
:10CA70000DB407FEFDCF8FEF8EBD0DB407FEFDCFC9
:10CA80008EB513968C9313978F71853011F481E0D6
:10CA9000089583E111968C931197CD01C4DF80E056
:10CAA0000895CF92DF92EF92FF920F931F93CF934F
:10CAB000DF93EC017A018B0169018C81833039F0BD
:10CAC00059E0EE0CFF1C001F111F5A95D1F7CE0143
:10CAD00068E1A80197014EDF882311F086E020C0AD
:10CAE000CE016EEFA601A4DF8823D9F0CE0168E560
:10CAF00072E007DF882311F487E112C0CE016DE0F8
:10CB000020E030E040E050E035DF882341F48FEF53
:10CB10008EBD0DB407FEFDCF8EB5882371F086E182
:10CB20008983CE0180DF80E0DF91CF911F910F914B
:10CB3000FF90EF90DF90CF900895CE0174DF81E0F9
:10CB4000F3CFBF92CF92DF92EF92FF920F931F939A
:10CB5000CF93DF93EC016B017A010E940EAA8B0147
:10CB6000BB24BA9409C00E940EAA601B710B6D52BF
:10CB7000714010F081E10BC0BEBC0DB407FEFDCFCB
:10CB80008EB58B838F3F79F38E3F31F08FE08983B1
:10CB9000CE0149DF80E02EC0D7011197EF28D9F0F0
:10CBA0008FEF8EBD20E030E09FEF0BC00DB407FE8D
:10CBB000FDCF8EB5F601E20FF31F80839EBD2F5F80
:10CBC0003F4F2A173B0790F30DB407FEFDCF8EB5FC
:10CBD000AC0DBD1D8C938FEF8EBD0DB407FEFDCF48
:10CBE0008EB58FEF8EBD0DB407FEFDCF8EB5CE0195
:10CBF0001ADF81E0DF91CF911F910F91FF90EF90AD
:10CC0000DF90CF90BF900895CF92DF92EF92FF9286
:10CC10000F931F93CF93DF93EC017A018B0169018E
:10CC20008C81833039F0A9E0EE0CFF1C001F111F2E
:10CC3000AA95D1F7CE0161E1A80197019BDE882377
:10CC400031F084E08983CE01EEDE80E005C0CE01C4
:10CC5000B60140E052E075DFDF91CF911F910F9157
:10CC6000FF90EF90DF90CF900895BF92CF92DF9228
:10CC7000EF92FF920F931F93CF93DF93EC01B62EA9
:10CC80001C82198248830E940EAA6B01888161E090
:10CC90000E94BFABCE01C7DE82E360E00E94BFAB63
:10CCA00083E361E00E94BFAB84E361E00E94BFAB1D
:10CCB00085E361E00E94BFAB85E361E00E9472AC56
:10CCC00085E08A8382E58CBD1DBC80E09FEF9EBD20
:10CCD0000DB407FEFDCF8F5F8A30C9F709C00E94EF
:10CCE0000EAA6C197D09615D774010F081E059C092
:10CCF000CE0160E020E030E040E050E03BDE182F65
:10CD00008B83813061F7CE0168E02AEA31E040E0B0
:10CD100050E030DE82FF02C01C8311C080E02FEFA4
:10CD20002EBD0DB407FEFDCF9EB58F5F8430C1F7D9
:10CD30009B839A3A11F082E034C082E08C838C812C
:10CD4000823021F0EE24FF2487010FC0E12CF12C6A
:10CD5000012D00E4102F09C00E940EAA6C197D0954
:10CD6000615D774010F08AE01CC0CE0167E320E0EF
:10CD700030E040E050E0FEDDCE0169E2A80197011D
:10CD8000F9DD8B83882341F78C81823019F5CE0140
:10CD90006AE320E030E040E050E0ECDD882329F059
:10CDA00088E08983CE013FDE20C08FEF8EBD0DB4B9
:10CDB00007FEFDCF8EB5807C803C11F483E08C8330
:10CDC00080E09FEF9EBD0DB407FEFDCF2EB58F5FB7
:10CDD0008330C1F7CE0127DE86E08B1518F488E199
:10CDE000898303C0BA8281E001C080E0DF91CF91E6
:10CDF0001F910F91FF90EF90DF90CF90BF9008951B
:10CE0000CF93DF93EB01DC0190E020E03EE28C91D8
:10CE1000803269F0283029F4FE01E90FF11D3083DA
:10CE20009F5FFE01E90FF11D8C9180839F5F2F5F53
:10CE300011962B3061F7C90FD11D1882DF91CF9168
:10CE400008950F931F93CF93DF93DC01EB018A01C9
:10CE500080E090E020E2FE01E80FF91F20830196B8
:10CE60008B309105C1F757E040E024C0622F2E328D
:10CE700019F087EB9AE007C05A3051F15AE048E0C8
:10CE800018C0321729F1FC01019634913323C9F7F8
:10CE90005417F0F02132E0F02F37D0F4822F815672
:10CEA0008A3110F4622F6052FE01E40FF11D60839D
:10CEB0004F5F11962C91222311F02F32B9F6F80111
:10CEC000B183A08390E08881803219F091E001C0A5
:10CED00090E0892FDF91CF911F910F9108956F926C
:10CEE0007F928F929F92AF92BF92CF92DF92EF92FA
:10CEF000FF920F931F93CF93DF93EC017A018B0185
:10CF00002B81222309F480C089899A89AB89BC8945
:10CF100084179507A607B70708F476C085C0E11403
:10CF2000F1040105110551F41C821D821E821F822D
:10CF3000188619861A861B8681E067C02885398580
:10CF40004A855B85E98DFA8D858590E009962150AB
:10CF500030404040504039014A01082E04C09694A8
:10CF60008794779467940A94D2F72F5F3F4F4F4F7F
:10CF70005F4F0894E108F1080109110957016801A0
:10CF800004C0D694C794B794A7948A95D2F708940E
:10CF9000E11CF11C011D111DA614B704C804D9041D
:10CFA00028F0211531054105510549F48D899E89E7
:10CFB000AF89B88D8C839D83AE83BF8316C0A618BE
:10CFC000B708C808D90811C04C815D816E817F8186
:10CFD000898D9A8D94010E94E7720894A108B10886
:10CFE000C108D108882331F40FC084E0882E912C29
:10CFF0008C0E9D1EA114B104C104D10429F7E8864A
:10D00000F9860A871B8798CF80E0DF91CF911F9127
:10D010000F91FF90EF90DF90CF90BF90AF909F90D7
:10D020008F907F906F900895223009F078CFE7CFEE
:10D03000CF93DF93EC018C859D85AE85BF8540E065
:10D04000611141E0BC01CD010E94C170882319F437
:10D0500020E030E00AC08889282F30E095E0220FD8
:10D06000331F9A95E1F7245C304FC901DF91CF91CE
:10D0700008950F931F93CF93DF938C01FC0183815D
:10D080008823D9F1818187FF35C0C80161E0D0DFF5
:10D09000EC01009791F18881853E79F1F801838157
:10D0A000823040F481899289A389B4898C8F9D8FC5
:10D0B000AE8FBF8FF80185899689A789B08D9B8F28
:10D0C0008A8FCD01AA27BB279D8B8C8BE091360FD1
:10D0D000F091370F309751F0BE016A5E7F4FCE015D
:10D0E00048961995888D998D9B8B8A8BF801818143
:10D0F0008F7781830E94867004C081E0F80180836D
:10D1000080E0DF91CF911F910F9108950F931F93AE
:10D110008C01AFDFF80113821F910F910895FC017C
:10D120008381882311F0CF01F1CF0895CF93DF934E
:10D13000FC01EB018381882381F08250823020F44E
:10D140008FE28883198207C0CF0160E071DF00970A
:10D1500021F0BE0155DE81E001C080E0DF91CF917A
:10D1600008956F927F928F929F92AF92BF92CF92CB
:10D17000DF92EF92FF920F931F93DF93CF9300D034
:10D180000F92CDB7DEB77C015A016B01DC0113961B
:10D190008C911397813009F08EC011968C9181FF8C
:10D1A0008AC09DC00097A105B10511F481E084C03B
:10D1B000F7016084718482849384C701B601A5015C
:10D1C0008EDE882309F477C0D70159968D919C9102
:10D1D0005A97A114B104C104D10489F455964D9114
:10D1E0005D916D917C9158970E945C73882309F43E
:10D1F00062C0F701158A168A178A108E44C0D701BB
:10D2000014964D915D916D917C9117979E012F5FC2
:10D210003F4F0E94E772882309F44DC0D701599609
:10D22000ED91FC915A9749815A816B817C81878964
:10D23000803149F4483FBFEF5B07B0E06B07B0E0D7
:10D240007B0748F020C0483F8FEF58078FEF6807F3
:10D250008FE07807C0F4CF010E945C73882359F1F6
:10D26000D70114964D915D916D917C9117975996C8
:10D270008D919C915A970FEF1FEF2FEF3FE00E9487
:10D2800061728823C1F0F701A18AB28AC38AD48A65
:10D29000818180688183C701ECDE882361F0B6015B
:10D2A000A5016A147B048C049D0410F4B401A3014D
:10D2B000C70115DE01C080E00F900F900F900F9016
:10D2C000CF91DF911F910F91FF90EF90DF90CF9062
:10D2D000BF90AF909F908F907F906F900895F701CF
:10D2E00081899289A389B48984179507A607B7070E
:10D2F00008F058CFE0CFCF93DF93EC0140E050E04F
:10D3000060E070E02EDF882359F0CE0161E090DE0E
:10D31000FC01009729F085EE80831B82F7D601C0BF
:10D3200080E0DF91CF9108952F923F924F925F92CC
:10D330006F927F928F929F92AF92BF92CF92DF9225
:10D34000EF92FF920F931F93CF93DF93EC012A018B
:10D350008B81882309F4B5C0898180FFB2C0C7C022
:10D3600025014E185F083B0174E0272E312C2C0E4E
:10D370003D1E4201A0C0288539854A855B856FEF37
:10D38000A62E61E0B62EA222B3228B8179018A01FA
:10D3900099E016950795F794E7949A95D1F7E98D5A
:10D3A000FA8D823049F4428D538D648D758D4E0D0A
:10D3B0005F1D601F711F3FC0D480DA94DE20A1146E
:10D3C000B104D9F4DD20C9F4211531054105510519
:10D3D00049F48D899E89AF89B88D8C839D83AE83F6
:10D3E000BF830BC04C815D816E817F81CF01910134
:10D3F0000E94E772882309F464C0E98DFA8D4C819C
:10D400005D816E817F814250504060407040058454
:10D4100004C0440F551F661F771F0A94D2F78685F4
:10D420009785A089B189480F591F6A1F7B1F4D0D31
:10D43000511D611D711D80E092E08A199B098401D4
:10D440008815990508F48C0182E00030180709F06E
:10D4500066C08091380F9091390FA0913A0FB0912A
:10D460003B0F481759076A077B0709F458C080919A
:10D470003C1190913D119301C7DB882349F421C0F1
:10D480009501245C304FC301B901A8010E945210DC
:10D49000600E711E980140E050E088859985AA854C
:10D4A000BB85820F931FA41FB51F88879987AA8702
:10D4B000BB87801A910A8114910409F05CCFA20104
:10D4C00002C04FEF5FEFCA01DF91CF911F910F9123
:10D4D000FF90EF90DF90CF90BF90AF909F908F9094
:10D4E0007F906F905F904F903F902F900895A98804
:10D4F000BA88CB88DC88E884F9840A851B859A0180
:10D5000040E050E0D601C5018E199F09A00BB10B78
:10D51000281739074A075B0708F022CF24CFCB0131
:10D52000BA0140E02ED6882309F0AACFCACFCF9205
:10D53000DF92EF92FF920F931F93CF93DF937C01C3
:10D54000EB018A01FC018381823008F46EC0808582
:10D550009185A285B3858F719070A070B07000978F
:10D56000A105B10509F061C06CC0F8011082EDE0C1
:10D57000CE2ED12CC701BE0140E250E0D5DE9C0189
:10D580008032910521F0009709F04FC050C04881CA
:10D59000442309F44CC0453E69F34E3259F38B8560
:10D5A0008F738F30E9F501151105D1F18A8D9B8DAF
:10D5B000892BB1F5842F90E08F719070009781F1E5
:10D5C000833091056CF58C9D90018D9D300D9C9D57
:10D5D000300D11242D503040F801E20FF31F8981E6
:10D5E00080838B8181838D8182838F8183838985F1
:10D5F00084838E858583888986838A8987838C89BD
:10D6000080878E898187888D82878C8D83878E8D98
:10D610008487888186FF04C0F801E20FF31F158616
:10D620008B8583FDA7CF822F03C08FEF01C080E0E1
:10D63000DF91CF911F910F91FF90EF90DF90CF90EE
:10D6400008954115510509F090CF91CFDF93CF9305
:10D650000F92CDB7DEB7BE016F5F7F4F41E050E064
:10D6600063DE019719F02FEF3FEF03C08981282F68
:10D6700030E0C9010F90CF91DF910895EF92FF92B2
:10D680000F931F93CF93DF93EC018B81823030F1A6
:10D69000E884F9840A851B85CE01D8DF97FD1EC07A
:10D6A00088859985AA85BB854F96A11DB11D888760
:10D6B0009987AA87BB87A5E016950795F794E79405
:10D6C000AA95D1F72E2D30E02F703070F5E0220FA3
:10D6D000331FFA95E1F7245C304F02C020E030E0C0
:10D6E000C901DF91CF911F910F91FF90EF900895A5
:10D6F0000F931F93CF93DF93EC018B018B818823D2
:10D7000009F040C0FB018789803109F041C082E007
:10D710008B831D8A1E8A1F8A188E808D918DA0E0B2
:10D72000B0E045E0880F991FAA1FBB1F4A95D1F7AB
:10D73000898B9A8BAB8BBC8B13C083E08B83F801F6
:10D74000428D538D648D758D4D8B5E8B6F8B788F75
:10D750009E012F5E3F4FC8010E94B873882391F04D
:10D760001A8F098F81E089831C821D821E821F828D
:10D77000188619861A861B861C861D861E861F869D
:10D78000188A01C080E0DF91CF911F910F91089519
:10D790008032C1F7D2CF1F93CF93DF93EC01142FC8
:10D7A000262F30E0F90175E0EE0FFF1F7A95E1F7C3
:10D7B000E45CF04F8385817121F0842F827109F040
:10D7C00066C08091380F9091390FA0913A0FB091B7
:10D7D0003B0F8C879D87AE87BF87688BF90165E01B
:10D7E000EE0FFF1F6A95E1F7E45CF04F848995899D
:10D7F000A0E0B0E0DC01992788278D8B9E8BAF8B52
:10D80000B88F228D338DA90160E070E0482B592B31
:10D810006A2B7B2B4D8B5E8B6F8B788F838590E093
:10D8200088719070009751F4848D958DA68DB78D79
:10D83000898B9A8BAB8BBC8B81E00BC0409739F501
:10D840009E012F5E3F4F898D9A8D92D78823F9F0E4
:10D8500084E08B83812F8F7089831C821D821E82BE
:10D860001F82188619861A861B8614FF16C0CE01E1
:10D8700040E050E060E070E074DC882371F409C09F
:10D8800049895A896B897C89CE0129DB02C01B82B8
:10D8900080E0DF91CF911F91089515FDF1CF81E0D8
:10D8A000F8CFCF93DF93EC019C012C5F3F4F898D24
:10D8B0009A8D41E050E060E070E0C5D78823A1F088
:10D8C0008D899E89AF89B88D0097A105B10559F45E
:10D8D0008C819D81AE81BF818D8B9E8BAF8BB88FEC
:10D8E00089818068898381E0DF91CF9108952F92AB
:10D8F0003F924F925F927F928F929F92AF92BF9290
:10D90000CF92DF92EF92FF920F931F93DF93CF930B
:10D9100000D000D0CDB7DEB76C01162F072F5E8385
:10D920004D83DC0113968C911397813009F069C106
:10D9300011968C9181FF65C182C1F601418952899E
:10D940006389748980859185A285B385841795073D
:10D95000A607B70729F0C601C2DA882309F451C126
:10D96000812F902F9C0119014D805E800FC1D6013F
:10D970005996ED91FC915A97DA01C90149E0B695A3
:10D98000A795979587954A95D1F774807A947822D0
:10D990008FEF882E81E0982E82229322772009F043
:10D9A00051C08114910409F04DC0D60114964D91D7
:10D9B0005D916D917C911797411551056105710538
:10D9C00081F455968D919D910D90BC91A02D00975D
:10D9D000A105B10559F1F60184839583A683B78328
:10D9E00031C0CF019E012F5F3F4FF1D5882309F44D
:10D9F00008C129813A814B815C81D6015996ED910C
:10DA0000FC915A978789803149F4283FBFEF3B0743
:10DA1000B0E04B07B0E05B0770F008C0283FEFEFC5
:10DA20003E07EFEF4E07EFE05E0728F0C60139DF53
:10DA3000882341F4E6C0D60114962D933D934D936F
:10DA40005C93179780E092E0881999095201841538
:10DA5000950508F45C01D6015996ED91FC915A9711
:10DA60001496ED90FD900D911C9117978EEF9FEFFE
:10DA7000AFEFBFEFE80EF91E0A1F1B1F058404C09D
:10DA8000EE0CFF1C001F111F0A94D2F786859785A4
:10DA9000A089B189E80EF91E0A1F1B1FE70CF11CB3
:10DAA000011D111D90E0A91692E0B90639F580918B
:10DAB000380F9091390FA0913A0FB0913B0F8E150E
:10DAC0009F05A007B10771F410923E118FEF9FEFF1
:10DAD000AFEFBFEF8093380F9093390FA0933A0FB9
:10DAE000B0933B0F80913C1190913D11B801A7017B
:10DAF00091010E9451658823A9F583C08114910486
:10DB000011F5D60118962D913D914D915C911B9781
:10DB100051968D919D910D90BC91A02D281739079C
:10DB20004A075B0780F0F2D2882309F46AC081E0DB
:10DB300080933E11E092380FF092390F00933A0F24
:10DB400010933B0F07C0C801B70141E01AD38823E7
:10DB500009F457C09401245C304FC901B101A501FB
:10DB60000E945210950140E050E0F60180859185B9
:10DB7000A285B385820F931FA41FB51F808791874D
:10DB8000A287B3872A0C3B1C4A185B08D60118965B
:10DB90002D913D914D915C911B974114510409F0D9
:10DBA000E6CE51968D919D910D90BC91A02D82173E
:10DBB0009307A407B50748F4F601218B328B438BFA
:10DBC000548B81818068818311C08091360F909140
:10DBD000370F892B59F08D819E81892B39F0D60121
:10DBE00011968C911197806811968C93F601818122
:10DBF00083FF04C0C6013DDA882319F04D815E81A0
:10DC000005C081E0D6018C934FEF5FEFCA012696E5
:10DC10000FB6F894DEBF0FBECDBFCF91DF911F913D
:10DC20000F91FF90EF90DF90CF90BF90AF909F90BB
:10DC30008F907F905F904F903F902F90089582FD3E
:10DC40007CCE8ECEDF92EF92FF920F931F93CF93F5
:10DC5000DF93EC0189899A89AB89BC89805E9F4FEB
:10DC6000AF41B04008F06FC0CE011BDE882309F43D
:10DC70006AC04CD2882309F466C0E98DFA8DEC8025
:10DC8000FD800E811F818EEF9FEFAFEFBFEFE80E9B
:10DC9000F91E0A1F1B1F058404C0EE0CFF1C001F89
:10DCA000111F0A94D2F786859785A089B189E80E5D
:10DCB000F91E0A1F1B1F81E080933E11E092380F6E
:10DCC000F092390F00933A0F10933B0F80E092E0EF
:10DCD000ECE3FFE0DF019C011D9221503040E1F7B1
:10DCE000DD24D39411C0B801A7014D0D511D611D54
:10DCF000711D80913C1190913D112CE33FE00E94F9
:10DD00005165882301F1D394E98DFA8D8481D81669
:10DD100050F320E032E040E050E0058404C0220FE0
:10DD2000331F441F551F0A94D2F789899A89AB89FA
:10DD3000BC89820F931FA41FB51F898B9A8BAB8B55
:10DD4000BC8B81E001C080E0DF91CF911F910F91EA
:10DD5000FF90EF90DF9008958F929F92AF92BF92C5
:10DD6000CF92DF92EF92FF920F931F93CF93DF93A7
:10DD70006C01EB01942E852EA22E898D9A8DD601F1
:10DD80005A969C938E935997CB0140E050E060E007
:10DD900070E0A5D8BB2437C0CE0170DCFC01009731
:10DDA00009F48FC055E016950795F794E7945A95B6
:10DDB000D1F71E2D1F708081882311F0853EC9F494
:10DDC000BB2099F42091380F3091390F40913A0FD0
:10DDD00050913B0FD6011C962D933D934D935C9330
:10DDE0001F9750961C93BB24B3948081882359F4C9
:10DDF00018C0892D982DBF014BE050E00E944510BE
:10DE0000009709F46CC0E884F9840A851B85898928
:10DE10009A89AB89BC89E816F9060A071B0708F43A
:10DE2000BBCFA6FE4EC0A1FE4CC0BB2049F0F60100
:10DE30001089C60161E0FCD8EC01009761F441C093
:10DE40008B81823009F43DC0CE01FCDE8823C9F10C
:10DE500010E0CCE3DFE080E2DE011D928A95E9F775
:10DE6000DE01292D382DC901FC018BE001900D92B6
:10DE70008150E1F7E091360FF091370F309739F08C
:10DE8000BE01625F7F4FCE014096199508C081E2C6
:10DE900098E2998B888B80E098E09F878E878889AD
:10DEA00099899B8B8A8B998F888F8E859F859F8B75
:10DEB0008E8B2CD1882329F0C601612F4A2D6BDC73
:10DEC00001C080E0DF91CF911F910F91FF90EF9003
:10DED000DF90CF90BF90AF909F908F900895A7FE56
:10DEE000EBCFEFCF2F923F924F925F926F927F9244
:10DEF0008F929F92AF92BF92CF92DF92EF92FF925A
:10DF00000F931F93DF93CF93CDB7DEB7C654D040A6
:10DF10000FB6F894DEBF0FBECDBF3C016B01DE0132
:10DF2000AE5BBF4F11965C934E9325962FAF25970E
:10DF30001C861F861FA21AA66115710509F47CC0F4
:10DF4000FC018381882309F077C0FA0180818F3238
:10DF5000F1F08601ECE0EE2EF12CEC0EFD1E72E4E9
:10DF6000A72EB12CAC0EBD1E4E010894811C911C35
:10DF70002796FFAEEEAE279767E2262E312C2C0EA9
:10DF80003D1E270123C01196B183A08301C0FD016E
:10DF9000A081B1818C918F32B1F3D60113968C910F
:10DFA000139782508230A8F28E01095D1F4F599657
:10DFB0006D917C915A97C8019BDB882359F63CC030
:10DFC000342D252D8701832F922F7C01F50180812F
:10DFD0009181B401A5010E942167882329F42CC0F6
:10DFE0003196D501ED93FC93D501ED91FC918081A3
:10DFF0008F32B1F38823B9F0C701B801A40121E041
:10E00000ABDE8823C9F00C151D0511F0C8017ED8C0
:10E010002796EEADFFAD2797EE16FF0689F6C101F4
:10E02000322D292FCFCFC301B801A40125962FADE2
:10E03000259792DE182F01C010E0CE0187966FD889
:10E04000CE010C966CD8812FCA5BDF4F0FB6F894C7
:10E05000DEBF0FBECDBFCF91DF911F910F91FF901B
:10E06000EF90DF90CF90BF90AF909F908F907F9078
:10E070006F905F904F903F902F9008950F931F9354
:10E08000DF93CF93CDB7DEB76B970FB6F894DEBFB3
:10E090000FBECDBF9C01AB0119821C828E010F5FA8
:10E0A0001F4FC801B90122E01DDF882311F410E0E1
:10E0B00003C0C80120D9182FCE01019630D8812F76
:10E0C0006B960FB6F894DEBF0FBECDBFCF91DF9138
:10E0D0001F910F910895DB010D900020E9F7119732
:10E0E000A61BB70B0496AD0102CCDF93CF930F9222
:10E0F000CDB7DEB769830496BE016F5F7F4F41E005
:10E1000050E0F5DB0F90CF91DF91089580913E11A3
:10E11000882399F14091380F5091390F60913A0F4F
:10E1200070913B0F80913C1190913D112CE33FE0A9
:10E130000E945165882319F140913F11509140117F
:10E1400060914111709142114115510561057105B0
:10E1500091F080913C1190913D112CE33FE00E94A1
:10E160005165882361F010923F1110924011109276
:10E1700041111092421110923E1181E0089580E009
:10E180000895DF92EF92FF920F931F937B018C0112
:10E19000D42E8091380F9091390FA0913A0FB09101
:10E1A0003B0F8E159F05A007B107B9F0AFDF88239D
:10E1B000E1F080913C1190913D11B801A7012CE351
:10E1C0003FE00E940466882381F0E092380FF092CD
:10E1D000390F00933A0F10933B0FDD2011F481E0CB
:10E1E00005C081E080933E1101C080E01F910F9136
:10E1F000FF90EF90DF9008958F929F92AF92BF9221
:10E20000CF92DF92EF92FF920F931F93CF93DF9302
:10E210006C01142F70933D1160933C11FC01178A1F
:10E2200082E090E0A0E0B0E080839183A283B3839A
:10E2300010923E1110923F11109240111092411114
:10E24000109242118FEF9FEFAFEFBFEF8093380F27
:10E250009093390FA0933A0FB0933B0F442321F4CE
:10E260008824992454013FC0453008F01CC160E067
:10E2700070E080E090E040E084DF882309F413C17F
:10E28000C12FD0E02197FE0174E0EE0FFF1F7A95B9
:10E29000E1F7E45CF04FE254FE4F8081EE5BF14029
:10E2A00090E08F779070892B09F0FDC0E653FE4F08
:10E2B00080819181A281B38184369105A105B10548
:10E2C00008F4F1C064E0CC0FDD1F6A95E1F7CE5F82
:10E2D000DE4E88809980AA80BB8081149104A104BD
:10E2E000B10409F4E0C0C501B40140E04ADF88236D
:10E2F00009F4D9C08091470F9091480F8050924007
:10E3000009F0D1C020914C0F222309F4CCC0809198
:10E310004A0F90914B0F892B09F4C5C08091490F8A
:10E32000882309F4C0C0F601228B8091490F8483B1
:10E33000158661E070E007C04F5FF60145874150E8
:10E34000483008F0B0C0F6014585848190E09B011B
:10E35000042E02C0220F331F0A94E2F7821793079C
:10E3600059F72091520F3091530F2115310519F0B3
:10E3700040E050E008C02091600F3091610F409163
:10E38000620F5091630FF6012583368347835087D0
:10E39000E0904A0FF0904B0F00E010E0E80CF91C01
:10E3A0000A1D1B1DE38AF48A058B168B80914D0F85
:10E3B00090914E0F918F808F60914C0F70E080E0B4
:10E3C00090E00E9423B56E0D7F1D801F911FF60106
:10E3D000628F738F848F958F20914D0F30914E0FE8
:10E3E00055E0220F331F5A95E1F721503E4F232F5E
:10E3F0003327269540E050E0260F371F481F591F4E
:10E4000026873787408B518B80914F0F9091500F0B
:10E41000009719F0A0E0B0E008C080915C0F9091E7
:10E420005D0FA0915E0FB0915F0F85017401E21A3C
:10E43000F30A040B150BA8019701280F391F4A1F77
:10E440005B1FF601058404C05695479537952795BF
:10E450000A94D2F72187328743875487253FFFE00C
:10E460003F07F0E04F07F0E05F0720F48CE0F60193
:10E47000878B19C0255F3F4F4040504018F480E122
:10E48000F6010EC08091680F9091690FA0916A0FFC
:10E49000B0916B0FF601828F938FA48FB58F80E2BE
:10E4A000878B81E001C080E0DF91CF911F910F91B8
:10E4B000FF90EF90DF90CF90BF90AF909F908F90A4
:10E4C00008956F927F928F929F92AF92BF92CF9258
:10E4D000DF92EF92FF920F931F93CF93DF93EC01A4
:10E4E0005A016B013801490142305105610571053E
:10E4F00008F45DC089859A85AB85BC850196A11D10
:10E50000B11D84179507A607B70708F450C08F8977
:10E51000803129F4E52EF62E072F11270CC080320A
:10E5200009F045C07A018B0187E016950795F794AD
:10E53000E7948A95D1F78B899C89AD89BE89E80ECD
:10E54000F91E0A1F1B1FC801B70141E01ADE88230C
:10E5500071F18F89803149F4F501F070EE0FFF1FE2
:10E56000E45CF04F718260820DC0F501EF77F070CE
:10E57000EE0FFF1FEE0FFF1FE45CF04F6082718211
:10E58000828293828A89823080F08D819E81AF81E0
:10E59000B885E80EF91E0A1F1B1FE0923F11F0928A
:10E5A0004011009341111093421181E001C080E0BD
:10E5B000DF91CF911F910F91FF90EF90DF90CF905F
:10E5C000BF90AF909F908F907F906F900895CF9263
:10E5D000DF92EF92FF920F931F93CF93DF93EC01A3
:10E5E0007A018B01690189859A85AB85BC85019685
:10E5F000A11DB11D84179507A607B70708F452C0DF
:10E600008F89803129F45527412F302F2F2D0CC0B1
:10E61000803209F047C09A01AB0167E056954795F3
:10E62000379527956A95D1F78B899C89AD89BE89E5
:10E63000280F391F4A1F5B1F8091380F9091390FA7
:10E64000A0913A0FB0913B0F281739074A075B0793
:10E6500031F0CA01B90140E094DD882319F18F89B6
:10E66000803159F4F701F070EE0FFF1FE45CF04FBA
:10E6700080819181A0E0B0E00EC0F701EF77F070EB
:10E68000EE0FFF1FEE0FFF1FE45CF04F80819181C2
:10E69000A281B381BF70F60180839183A283B3838B
:10E6A00081E001C080E0DF91CF911F910F91FF9039
:10E6B000EF90DF90CF900895AF92BF92CF92DF920C
:10E6C000EF92FF920F931F93DF93CF9300D00F929F
:10E6D000CDB7DEB76C017A018B0182E090E0A0E05B
:10E6E000B0E0F60180839183A283B3835E01089436
:10E6F000A11CB11CC601B801A701950168DF8823E0
:10E7000039F1C601B801A70100E010E020E030E0D7
:10E71000D8DE8823E9F0E980FA800B811C81F601BC
:10E720008789803151F4F8EFEF16FFEFFF06F0E034
:10E730000F07F0E01F07F0F209C088EFE8168FEF2F
:10E74000F8068FEF08078FE01807A0F281E001C0FC
:10E7500080E00F900F900F900F90CF91DF911F915D
:10E760000F91FF90EF90DF90CF90BF90AF90089502
:10E770004F925F926F927F928F929F92AF92BF92D1
:10E78000CF92DF92EF92FF920F931F93DF93CF937D
:10E7900000D00F92CDB7DEB76C0149835A836B83EB
:10E7A0007C833901EE24FF2487012E010894411C4B
:10E7B000511C812CE2E09E2EA12CB12C49815A8162
:10E7C0006B817C81C601920102DF882339F1D5017A
:10E7D000C401F601058404C0880F991FAA1FBB1F3E
:10E7E0000A94D2F7E80EF91E0A1F1B1F29813A81ED
:10E7F0004B815C818789803131F4285F3F4F4040F5
:10E800005040E0F205C0285F3F4F4F4F5F40B0F2ED
:10E81000F301E082F1820283138381E00F900F9075
:10E820000F900F90CF91DF911F910F91FF90EF907C
:10E83000DF90CF90BF90AF909F908F907F906F9020
:10E840005F904F9008952F923F924F925F926F92F8
:10E850007F928F929F92AF92BF92CF92DF92EF9270
:10E86000FF920F931F93DF93CF93CDB7DEB72F9710
:10E870000FB6F894DEBF0FBECDBF1C014A875B8781
:10E880006C877D873F872E87DC0119968D919D913E
:10E890000D90BC91A02D0196A11DB11D8E839F836B
:10E8A000A887B987F901008111812281338101157F
:10E8B00011052105310549F0480159010894811CD1
:10E8C000911CA11CB11C1D8210C0D1018D909D9086
:10E8D000AD90BC901D828A859B85AC85BD850197D6
:10E8E000A105B10511F491E09D83750164014424F3
:10E8F000552432018E010F5F1F4FF10181859285F2
:10E90000A385B485481659066A067B0608F08CC0B4
:10E910008E819F81A885B9858C159D05AE05BF05A3
:10E9200050F4A2E08A2E912CA12CB12CF2E0CF2E33
:10E93000D12CE12CF12CC101B701A601980147DED1
:10E94000882309F471C089819A81AB81BC81A701B8
:10E9500096012F5F3F4F4F4F5F4F0097A105B105C5
:10E9600019F049015A010DC0281939094A095B09F2
:10E970008A859B85AC85BD85281739074A075B07C3
:10E9800059F00894411C511C611C711C0894C11C55
:10E99000D11CE11CF11CB1CFC101A601B7010FEFE1
:10E9A0001FEF2FEF3FE08DDD882391F43DC026015E
:10E9B000370108944108510861087108C101B30189
:10E9C000A201970186017DDD882371F17301620147
:10E9D0008C149D04AE04BF0450F3AE85BF854D91E9
:10E9E0005D916D917C91411551056105710531F085
:10E9F000C1019501840165DD8823B1F0EE85FF85B5
:10EA000080829182A282B382FD81FF2359F0089413
:10EA1000811C911CA11CB11CD1018D929D92AD92C3
:10EA2000BC92139781E001C080E02F960FB6F89456
:10EA3000DEBF0FBECDBFCF91DF911F910F91FF9031
:10EA4000EF90DF90CF90BF90AF909F908F907F908E
:10EA50006F905F904F903F902F9008951092771194
:10EA600010927A1110927D1108958093BB0308953E
:10EA7000EFE6F0E08081826080830895819A879A32
:10EA8000EAE0F1E08081826080830E9A3B9A579A97
:10EA90005F9A829A8A9AE7E0F1E0808181608083C0
:10EAA0009FB7F894E8E0F1E08081816080839FBFA8
:10EAB0000A9A129A3F9A479A6D98759AE4E0F1E0A3
:10EAC00080818D7F80839FB7F894E5E0F1E08081BD
:10EAD000826080839FBF53985B9A6C98749AE4E03D
:10EAE000F1E080818E7F80839FB7F894E5E0F1E0CC
:10EAF0008081816080839FBF52985A9A809A8898BB
:10EB00005F9A869A8E988A9AEAE0F1E0808188601E
:10EB100080839FB7F894EBE0F1E08081877F80836A
:10EB20009FBF9FB7F894E8E0F1E080818160808327
:10EB30009FBF0C9A1498129A399A4198A1E8B0E0B4
:10EB40008C918F7E8C938C9188608C93E0E8F0E0C0
:10EB500080818D7F808380818E7F808380818F7391
:10EB6000808380818F7C80838C91887F82608C936E
:10EB700080E090E490938900809388001092850053
:10EB800010928400EFE6F0E080818260808381E073
:10EB90008093BB03789408951F93FC011FB7F894EA
:10EBA00080819181A281B381809351119093521100
:10EBB000A0935311B0935411FB0180819181A281E4
:10EBC000B3818093551190935611A0935711B09330
:10EBD0005811FA0180819181A281B38180935911EA
:10EBE00090935A11A0935B11B0935C11F90180814D
:10EBF0009181A281B38180935D1190935E11A09366
:10EC00005F11B09360111FBF1F910895FC012FB7D2
:10EC1000F89480819181A281B38180935D1190935A
:10EC20005E11A0935F11B09360112FBF0895E82F7C
:10EC30008FB7F894F0E0EE0FFF1FEE0FFF1FEF5AB3
:10EC4000FE4E20813181428153818FBFB901CA01BB
:10EC5000089580916F008D7F80936F0006C0809132
:10EC60001D0F8F5F8F7080931D0F90911C0F8091EF
:10EC70001D0F981751F41092441110924311809176
:10EC80006F00826080936F00089590911C0F8091B7
:10EC90001D0F981751F3E3CF90911C0F80911D0F1A
:10ECA000981739F00E940F820E946D290E94C19E20
:10ECB000F3CF0895F1DF5F9A8A9A9FB7F894E8E05E
:10ECC000F1E08081816080839FBF129A08951F9236
:10ECD0000F920FB60F920BB60F921124AF92BF9204
:10ECE000CF92DF92EF92FF920F931F932F933F9358
:10ECF0004F935F936F937F938F939F93AF93BF9344
:10ED0000CF93DF93EF93FF93809143119091441140
:10ED1000892B09F097C190911C0F80911D0F9817B6
:10ED200019F4E0E0F0E014C080911D0F90E02DE4B4
:10ED300030E0829FF001839FF00D929FF00D11242F
:10ED4000E45BF54FE45BFF4F81E08083EC54F040DF
:10ED5000F0934411E0934311309709F46DC1E45BE3
:10ED6000FF4F81E08083EC54F040109286111092A6
:10ED70008711109288111092891160AD71AD2CE944
:10ED80006134720718F060E47CE904C03EE461324B
:10ED9000730730F0769567957695679584E007C0A0
:10EDA00047E26131740730F07695679582E0809391
:10EDB0007F1107C080937F116032710510F460E20B
:10EDC00070E06052704058E060307507E8F0472FFF
:10EDD00050E0440F551F440F551F4551554F9A01A0
:10EDE0002E5F3F4FF901859194919C01AA27639F63
:10EDF000C001629F810D9A1F06948A1F9A1F1124D9
:10EE0000FA01459154911EC0CB01969587958C7F50
:10EE10008551914FFC0145915491FC013296259109
:10EE20003491862F90E087709070FC012E9FC00176
:10EE30002F9F900D3E9F900D1124B3E096958795DE
:10EE4000BA95E1F7481B590B44365105A8F4E8E0A0
:10EE5000F3E007C08091C00085FFFCCF319690930E
:10EE6000C60090819923B1F786E495E04AE050E02E
:10EE70000E941F2744E650E050938B1140938A1163
:10EE800080917F11992787FD909590938D118093A4
:10EE90008C11E0914311F091441164AD75AD709304
:10EEA000851160938411FCE961347F0718F060E4F8
:10EEB0007CE904C02EE46132720730F076956795E4
:10EEC0007695679584E007C037E26131730730F0CB
:10EED0007695679582E080937F1108C081E08093EA
:10EEE0007F116032710510F460E270E06052704092
:10EEF00048E060307407E8F0472F50E0440F551F9A
:10EF0000440F551F4551554F9A012E5F3F4FF90150
:10EF1000859194919C01AA27639FC001629F810DF6
:10EF20009A1F06948A1F9A1F1124FA014591549141
:10EF30001EC0CB01969587958C7F8551914FFC0122
:10EF400045915491FC01329625913491862F90E0A1
:10EF500087709070FC012E9FC0012F9F900D3E9FE7
:10EF6000900D112433E0969587953A95E1F7481B6B
:10EF7000590B44365105A8F4E8E0F3E007C080914E
:10EF8000C00085FFFCCF31969093C60090819923F5
:10EF9000B1F786E495E04AE050E00E941F2744E67E
:10EFA00050E0CA01A0E0B0E08093801190938111FD
:10EFB000A0938211B09383115093890040938800ED
:10EFC000E0914311F091441180899189A289B3891C
:10EFD000B695A79597958795B095A09590958195AD
:10EFE0009F4FAF4FBF4F8093611190936211A093D9
:10EFF0006311B09364118093651190936611A0938F
:10F000006711B09368118093691190936A11A0936E
:10F010006B11B0936C1180936D1190936E11A0934E
:10F020006F11B093701110927111109272111092B1
:10F0300073111092741106C080ED97E090938900CF
:10F0400080938800C0914311D0914411209709F416
:10F0500039C588A18093751180FF03C0899A8FEF0D
:10F0600002C0899881E08093B7038091751181FF78
:10F0700003C08F988FEF02C08F9A81E08093B8030E
:10F08000809175112091BB0380FF3BC0222309F4BE
:10F0900070C08CB18295869587708095282F2170DD
:10F0A00080FF2CC080917611882341F1888199815D
:10F0B000AA81BB81181619061A061B06FCF480915A
:10F0C000511190915211A0915311B091541180930C
:10F0D000451190934611A0934711B093481181E0D8
:10F0E0008093771188899989AA89BB898093711146
:10F0F00090937211A0937311B093741120937611B1
:10F1000038C02223B1F18CB182958F708095282F61
:10F11000217080FF2CC080917811882341F1888173
:10F120009981AA81BB81181619061A061B06FCF4E0
:10F130008091511190915211A0915311B09154119D
:10F140008093451190934611A0934711B0934811B5
:10F1500081E08093771188899989AA89BB898093F6
:10F16000711190937211A0937311B0937411209345
:10F170007811809175112091BB0381FF3AC0222341
:10F1800009F46CC08091030186958095282F217029
:10F1900080FF2CC080917911882341F18C819D8161
:10F1A000AE81BF81181619061A061B06FCF4809161
:10F1B000551190915611A0915711B091581180930B
:10F1C000491190934A11A0934B11B0934C1181E0D7
:10F1D00080937A1188899989AA89BB898093711152
:10F1E00090937211A0937311B093741120937911BD
:10F1F00035C0222399F120910301217031E02327AA
:10F2000059F180917B11882339F18C819D81AE81E8
:10F21000BF81181619061A061B06F4F480915511C1
:10F2200090915611A0915711B091581180934911A6
:10F2300090934A11A0934B11B0934C1130937A11D3
:10F2400088899989AA89BB898093711190937211D9
:10F25000A0937311B093741120937B118091751159
:10F260002091BB0382FF46C08FB7F89490910B01A9
:10F27000926090930B018FBF8FEF8093B90322238D
:10F2800009F47AC089B18695869586958095282F50
:10F29000217080FF2CC080917C11882341F18885EA
:10F2A0009985AA85BB85181619061A061B06FCF453
:10F2B0008091591190915A11A0915B11B0915C11FC
:10F2C00080934D1190934E11A0934F11B093501114
:10F2D00081E080937D1188899989AA89BB8980936F
:10F2E000711190937211A0937311B09374112093C4
:10F2F0007C1142C09FB7F89480910B018D7F809361
:10F300000B019FBF31E03093B9032223A9F189B1EA
:10F31000869586958095282F217080FF2BC080913F
:10F320007E11882339F188859985AA85BB851816B1
:10F3300019061A061B06F4F48091591190915A117E
:10F34000A0915B11B0915C1180934D1190934E117F
:10F35000A0934F11B093501130937D1188899989F2
:10F36000AA89BB898093711190937211A093731134
:10F37000B093741120937E118091751183FF03C0A7
:10F3800016988FEF02C0169A81E08093BA0360E06E
:10F3900078C18091C00087FF19C04091C600E091FC
:10F3A0004205F091430531969F012F7730703197D8
:10F3B00080914405909145052817390739F0EE539F
:10F3C000FB4F4083309343052093420528813981C8
:10F3D0004A815B818091611190916211A0916311CA
:10F3E000B0916411280F391F4A1F5B1F20936111D0
:10F3F00030936211409363115093641112161306F7
:10F40000140615066CF5889A88899989AA89BB899A
:10F41000281B390B4A0B5B0B20936111309362114F
:10F420004093631150936411209151113091521106
:10F4300040915311509154118091B703992787FD42
:10F440009095A92FB92F820F931FA41FB51F8093EA
:10F45000511190935211A0935311B0935411889865
:10F460002C813D814E815F81809165119091661163
:10F47000A0916711B0916811280F391F4A1F5B1FB7
:10F480002093651130936611409367115093681172
:10F4900012161306140615066CF58E9A888999893A
:10F4A000AA89BB89281B390B4A0B5B0B209365117A
:10F4B0003093661140936711509368112091551154
:10F4C0003091561140915711509158118091B803C5
:10F4D000992787FD9095A92FB92F820F931FA41FFD
:10F4E000B51F8093551190935611A0935711B09367
:10F4F00058118E98288539854A855B8580916911D8
:10F5000090916A11A0916B11B0916C11280F391F65
:10F510004A1F5B1F2093691130936A1140936B114E
:10F5200050936C111216130614061506DCF59FB7DE
:10F53000F89480910B01886080930B019FBF8889AC
:10F540009989AA89BB89281B390B4A0B5B0B20932D
:10F55000691130936A1140936B1150936C11209193
:10F56000591130915A1140915B1150915C11809169
:10F57000B903992787FD9095A92FB92F820F931F63
:10F58000A41FB51F8093591190935A11A0935B113A
:10F59000B0935C119FB7F89480910B01877F8093A3
:10F5A0000B019FBF2C853D854E855F8580916D1138
:10F5B00090916E11A0916F11B0917011280F391FA9
:10F5C0004A1F5B1F20936D1130936E1140936F1192
:10F5D0005093701112161306140615066CF5149A42
:10F5E00088899989AA89BB89281B390B4A0B5B0B2F
:10F5F00020936D1130936E1140936F1150937011E1
:10F6000020915D1130915E1140915F115091601118
:10F610008091BA03992787FD9095A92FB92F820F62
:10F62000931FA41FB51F80935D1190935E11A0934B
:10F630005F11B093601114988091711190917211C3
:10F64000A0917311B09174110196A11DB11D809309
:10F65000711190937211A0937311B0937411209152
:10F660007111309172114091731150917411888908
:10F670009989AA89BB89281739074A075B0730F49B
:10F680006F5F80917F1168170CF483CE2091711108
:10F690003091721140917311509174118C899D8930
:10F6A000AE89BF8982179307A407B50708F4E3C0A2
:10F6B000E0908011F09081110091821110918311DE
:10F6C000AC8CBD8CCE8CDF8CA8019701C601B50136
:10F6D000AA27279FB12D389FF001489FF00D479F23
:10F6E000E00DF11D289FB00DE11DFA1F379FB00DF1
:10F6F000E11DFA1F469FB00DE11DFA1F369FB10DA7
:10F70000EA1FFA1FB695EA1FFA1F11248CAD9DADB2
:10F710008E0F9F1F909385118093841128AD39AD72
:10F720004AAD5BADA0E0B0E0281739074A075B0798
:10F7300020F430938511209384116091841170918D
:10F7400085118CE96134780718F060E47CE904C025
:10F750009EE46132790730F07695679576956795E6
:10F7600084E007C0E7E261317E0730F07695679567
:10F7700082E080937F1108C081E080937F11603226
:10F78000710510F460E270E060527040F8E06030A3
:10F790007F07E8F0472F50E0440F551F440F551FD7
:10F7A0004551554F9A012E5F3F4FF9018591949134
:10F7B0009C01AA27639FC001629F810D9A1F069436
:10F7C0008A1F9A1F1124FA01459154911EC0CB0142
:10F7D000969587958C7F8551914FFC014591549169
:10F7E000FC01329625913491862F90E087709070BD
:10F7F000FC012E9FC0012F9F900D3E9F900D112464
:10F80000B3E096958795BA95E1F7481B590B4436B6
:10F810005105A8F4E8E0F3E007C08091C00085FF3F
:10F82000FCCF31969093C60090819923B1F786E47E
:10F8300095E04AE050E00E941F2744E650E05093D4
:10F840008900409388009A0140E050E08091801147
:10F8500090918111A0918211B0918311820F931F19
:10F86000A41FB51F8093801190938111A0938211E2
:10F87000B093831102C120917111309172114091A6
:10F88000731150917411888D998DAA8DBB8D82173B
:10F890009307A407B50708F0E4C060918611709142
:10F8A000871180918811909189112C8D3D8D4E8DFD
:10F8B0005F8DAA27639FB12D749FF001849FF00D87
:10F8C000839FE00DF11D649FB00DE11DFA1F739F32
:10F8D000B00DE11DFA1F829FB00DE11DFA1F729F4E
:10F8E000B10DEA1FFA1FB695EA1FFA1F1124809185
:10F8F0008411909185118E179F0738F4C05CDF4FFB
:10F9000068817981C054D04003C0BC016E1B7F0B5D
:10F91000C05CDF4F288139814A815B81CB01A0E047
:10F92000B0E082179307A407B50708F4B901FCE912
:10F9300061347F0718F060E47CE904C02EE4613292
:10F94000720730F0769567957695679584E007C0E5
:10F9500037E26131730730F07695679582E08093E6
:10F960007F1108C081E080937F116032710510F42F
:10F9700060E270E06052704048E060307407E8F088
:10F98000472F50E0440F551F440F551F4551554F09
:10F990009A012E5F3F4FF901859194919C01AA270E
:10F9A000639FC001629F810D9A1F06948A1F9A1F50
:10F9B0001124FA01459154911EC0CB01969587956B
:10F9C0008C7F8551914FFC0145915491FC013296F9
:10F9D00025913491862F90E087709070FC012E9FC6
:10F9E000C0012F9F900D3E9F900D112423E096950E
:10F9F00087952A95E1F7481B590B44365105A8F421
:10FA0000E8E0F3E007C08091C00085FFFCCF3196AD
:10FA10009093C60090819923B1F786E495E04AE07F
:10FA200050E00E941F2744E650E050938900409325
:10FA300088009A0140E050E08091861190918711F2
:10FA4000A0918811B0918911820F931FA41FB51F37
:10FA50008093861190938711A0938811B093891198
:10FA60000CC080918A1190918B11909389008093A2
:10FA7000880080918C1180937F11209171113091B9
:10FA800072114091731150917411E0914311F091F2
:10FA9000441180899189A289B389281739074A07B7
:10FAA0005B0780F0109244111092431190911C0F4B
:10FAB00080911D0F981731F080911D0F8F5F8F700F
:10FAC00080931D0FFF91EF91DF91CF91BF91AF9187
:10FAD0009F918F917F916F915F914F913F912F9166
:10FAE0001F910F91FF90EF90DF90CF90BF90AF905C
:10FAF0000F900BBE0F900FBE0F901F901895809126
:10FB00007711882349F480917A11882329F4809110
:10FB10007D11882309F49CC0EBEEF2E1949108C0BA
:10FB20008091C00085FFFCCF9093C60031969491E0
:10FB30009923B1F7EDE2F3E1949108C08091C00000
:10FB400085FFFCCF9093C600319694919923B1F72D
:10FB5000809177118823F1F06091451170914611E1
:10FB600080914711909148110E9413B22091EF09A2
:10FB70003091F0094091F1095091F2090E9478B159
:10FB8000AB01BC0189E293E10E94902D89E193E1F0
:10FB90000E94C29C80917A118823F1F060914911F2
:10FBA00070914A1180914B1190914C110E9413B2A7
:10FBB0002091F3093091F4094091F5095091F6092B
:10FBC0000E9478B1AB01BC0185E193E10E94902DC8
:10FBD00085E093E10E94C29C80917D118823F1F021
:10FBE00060914D1170914E1180914F119091501173
:10FBF0000E9413B22091F7093091F8094091F90958
:10FC00005091FA090E9478B1AB01BC0181E093E107
:10FC10000E94902D81EF92E10E94C29CECE1F3E002
:10FC200007C08091C00085FFFCCF31969093C6003D
:10FC300090819923B1F78091C00085FFFCCF8AE0C5
:10FC40008093C6001092771110927A1110927D1154
:10FC5000089560E070E08FE793E42091C003309155
:10FC6000C1034091C2035091C3030E9478B16093D5
:10FC7000BB117093BC118093BD119093BE11089578
:10FC8000FC0197FF03C080919F1103C0E256FE4E16
:10FC9000808190E00895089510928F1110928E1136
:10FCA00010929E112C981092911110929011109216
:10FCB0009F11109291111092901110929F119FB765
:10FCC000F894E2E0F1E080818F7D80839FBF08950A
:10FCD0002DEB37E346E05EE30C9451B42DEB37E3B4
:10FCE00046E05EE30C9478B12DEB37E346E05EE34B
:10FCF0000C9478B12DEB37E346E05EE30C9451B4FD
:10FD00001F93182FC9DF0E945F28882309F036C08F
:10FD1000ECE3F3E1949108C08091C00085FFFCCF33
:10FD20009093C600319694919923B1F786E495E0BB
:10FD3000612F70E04AE050E00E94F8268091C000F8
:10FD400085FFFCCF8AE08093C600EBE9F3E1949154
:10FD500008C08091C00085FFFCCF9093C60031960B
:10FD600094919923B1F78091C00085FFFCCF8AE080
:10FD70008093C6008EE893E10E94D19C0E94C22825
:10FD80001F9108951F93182F87DF0E945F288823F3
:10FD900009F036C0ECE3F3E1949108C08091C00013
:10FDA00085FFFCCF9093C600319694919923B1F7CB
:10FDB00086E495E0612F70E04AE050E00E94F8266A
:10FDC0008091C00085FFFCCF8AE08093C600E5EDFE
:10FDD000F3E1949108C08091C00085FFFCCF90931F
:10FDE000C600319694919923B1F78091C00085FFA8
:10FDF000FCCF8AE08093C60088EC93E10E94D19CFE
:10FE00000E94C2281F9108951F920F920FB60F9261
:10FE10000BB60F9211242F933F934F935F936F93E1
:10FE20007F938F939F93AF93BF93EF93FF93209113
:10FE3000CE032223A1F480919E118093A4118111FD
:10FE40002C9A80919F118093A311882341F09FB732
:10FE5000F894809102018062809302019FBF80919B
:10FE6000A411281708F02C988091A311281740F0AE
:10FE70009FB7F894809102018F7D809302019FBF0C
:10FE80002F5F2F772093CE038091A511833009F443
:10FE900050C0843028F48130F9F08230D8F50DC09C
:10FEA000853009F471C0853008F45FC0863009F4EC
:10FEB00087C0873009F08FC087C088E080937B00BF
:10FEC00085E480937C0080917A00806480937A003E
:10FED0000E94318A81E01BC0809178009091790066
:10FEE000A0E0B0E02091B2113091B3114091B41173
:10FEF0005091B511280F391F4A1F5B1F2093B21173
:10FF00003093B3114093B4115093B51182E08093B4
:10FF1000A51161C088E080937B0086E480937C001B
:10FF200080917A00806480937A000E94318A83E015
:10FF3000EECF8091780090917900A0E0B0E0209120
:10FF4000A6113091A7114091A8115091A911280F25
:10FF5000391F4A1F5B1F2093A6113093A7114093AE
:10FF6000A8115093A91184E0D2CF88E080937B0040
:10FF700087E480937C0080917A00806480937A008B
:10FF80000E94318A85E0C3CF8091780090917900FA
:10FF9000A0E0B0E02091AE113091AF114091B011CE
:10FFA0005091B111280F391F4A1F5B1F2093AE11CA
:10FFB0003093AF114093B0115093B11186E0A7CFA9
:10FFC0000E94318A87E0A3CF1092A5118091B611CB
:10FFD0008F5F8093B6118091B611803108F453C0C1
:10FFE0008091A011882381F48091B2119091B31176
:10FFF00090939311809392118091A6119091A711E3
:020000021000EC
:10000000909399118093981181E08093A0111092A0
:10001000B6111092B2111092B3111092B411109245
:10002000B5111092AE111092AF111092B011109242
:10003000B1111092AA111092AB111092AC11109242
:10004000AD111092A6111092A7111092A811109242
:10005000A91120919211309193118091A111909149
:10006000A2118217930714F080E08CDE2091921188
:10007000309193118091CC039091CD0328173907CB
:1000800014F080E03DDEFF91EF91BF91AF919F9121
:100090008F917F916F915F914F913F912F910F9031
:1000A0000BBE0F900FBE0F901F9018952F926F925E
:1000B0007F928F929F92AF92BF92CF92DF92EF92F8
:1000C000FF920F931F93DF93CF93CDB7DEB729979E
:1000D0000FB6F894DEBF0FBECDBF8C01E62E6623AF
:1000E00069F1ECE3F3E1949108C08091C00085FFD1
:1000F000FCCF9093C600319694919923B1F786E492
:1001000095E06E2D70E04AE050E00E94F826E2E0B3
:10011000F4E1949108C08091C00085FFFCCF9093DA
:10012000C600319694919923B1F78091C00085FF64
:10013000FCCF8AE08093C6000E940A29AE2DB0E071
:10014000FD01EE0FFF1FE25AFB4F6081718179873D
:100150006887672B09F49FC0A05ABB4F7C917B83B3
:100160002224239479C0222D30E0A901440F551F89
:10017000440F551FE885F985E40FF51F859194918B
:10018000081719070CF067C0C9010197880F991F5C
:10019000880F991FFC013296A885B985EA0FFB1FCD
:1001A000C590D4908A0F9B1FFC01659174917A834E
:1001B0006983FA013296EA0FFB1FE590F490FD0186
:1001C000E40FF51FA590B490B601882777FD8095C0
:1001D000982F0E9413B26C837D838E839F838981C5
:1001E0009A81081B190BB801882777FD8095982FF5
:1001F0000E9413B23B014C01EC18FD080027F7FCEC
:100200000095102FC801B7010E9413B29B01AC01E9
:10021000C401B3010E9451B47B018C01A981BA8150
:10022000AA1ABB0ACC24B7FCC094DC2CC601B501C9
:100230000E9413B29B01AC01C801B7010E9478B1C2
:100240009B01AC016C817D818E819F810E9498B061
:10025000E62F692F09C02394BB812B1608F483CFA6
:10026000E0E070E080E060E0FB812F1679F5E22DA0
:10027000F0E0EE0FFF1FEE0FFF1F329768857985C4
:10028000E60FF71F65917491882777FD8095982F69
:100290000E9413B219C0B801882777FD8095982F66
:1002A0000E9413B220E030E04AEF5EE30E9451B4B6
:1002B00020E030E040E85DE30E9451B420E030E00F
:1002C00040E050E00E9498B0E62F692F2E2F372F84
:1002D000482F562FB901CA0129960FB6F894DEBFF0
:1002E0000FBECDBFCF91DF911F910F91FF90EF9087
:1002F000DF90CF90BF90AF909F908F907F906F9046
:100300002F90089580E090E0A0E0B0E08093B711D6
:100310009093B811A093B911B093BA1160E070E056
:100320008FE793E42091C0033091C1034091C20351
:100330005091C3030E9478B16093BB117093BC11BC
:100340008093BD119093BE11249A80910101806227
:10035000809301018091010180648093010187ED08
:1003600080937A0010927E0010927D0080917D0033
:10037000806280937D0080917D00806880937D0005
:1003800080917D00806480937D0080E888BD8091AD
:100390006E00846080936E006AEF70E080E090E011
:1003A0000E941CAA85E090E09093C0118093BF1139
:1003B00009C08091CC039091CD0340979093CD03D9
:1003C0008093CC038091CC039091CD0360E06EDEEE
:1003D00020E030E040EA50E40E9471B187FDE9CFAF
:1003E00085EF90E09093D0038093CF0309C0809174
:1003F000A1119091A21140969093A2118093A11106
:100400008091A1119091A21160E050DE20E030E0D7
:1004100045E753E40E947FB318164CF308952F92DA
:100420003F924F925F926F927F928F929F92AF9284
:10043000BF92CF92DF92EF92FF920F931F93809122
:10044000A011882309F48DC180919211909193118C
:1004500060E02CDE3B014C01609394117093951188
:10046000809396119093971180E090E0A0E0B0E027
:1004700080939A1190939B11A0939C11B0939D111E
:100480008FB7F8941092A0118FBFC0908E11D090AA
:100490008F11B601882777FD8095982F0E9413B29F
:1004A000A40193010E9497B07B018C016093C1115C
:1004B0007093C2118093C3119093C41120E030E077
:1004C00040E251E40E947FB3181624F481E0809347
:1004D000C511E9C0C801B70120E030E040E251ECAD
:1004E0000E9471B187FD02C0CD2821F481E0809384
:1004F000C511C4C08091C511882371F080E090E0DF
:10050000A0E0B0E08093C6119093C711A093C811EA
:10051000B093C9111092C511C801B7012091BC0355
:100520003091BD034091BE035091BF030E9451B46E
:100530001B012C016093CA117093CB118093CC11D5
:100540009093CD11C801B7012091C6113091C71108
:100550004091C8115091C9110E9498B05B016C0183
:10056000E090B711F090B8110091B9111091BA1143
:10057000A80197010E9471B187FD12C0E090BB11E4
:10058000F090BC110091BD111091BE11C601B501D2
:10059000A80197010E947FB3181614F08601750117
:1005A000E092C611F092C7110093C8111093C911BF
:1005B000C801B7012091C0033091C1034091C2032B
:1005C0005091C3030E9451B45B016C016093CE1142
:1005D0007093CF118093D0119093D111C401B301C6
:1005E0002091D2113091D3114091D4115091D51155
:1005F0000E9497B02091C4033091C5034091C60377
:100600005091C7030E9451B420ED3CEC4CE45DE3F3
:100610000E9451B47B018C016091D6117091D71169
:100620008091D8119091D91123E333E343E75FE33D
:100630000E9451B49B01AC01C801B7010E9498B05F
:100640007B018C016093D6117093D7118093D811E0
:100650009093D911C201B101A60195010E9498B0F1
:10066000A80197010E9497B07B018C0120E030E047
:1006700040E050E00E9471B188235CF40F2EF0E05E
:10068000EF2EF0E0FF2EF0E00F2FF0E01F2FF02D07
:1006900014C0C801B70120E030E04FE753E40E94E6
:1006A0007FB3181654F40F2EF0E0EF2EF0E0FF2E7B
:1006B000FFE70F2FF3E41F2FF02D6092D2117092FD
:1006C000D3118092D4119092D5116091BF11709185
:1006D000C011882777FD8095982F0E9413B29B0147
:1006E000AC01C401B3010E947FB31816DCF4609121
:1006F000CF037091D003882777FD8095982F0E94B3
:1007000013B29B01AC01C401B3010E9471B18823F3
:100710004CF4C801B7010E94E0B1759567956093EC
:100720009E1102C010929E110E940EAA2091DA1111
:100730003091DB114091DC115091DD11621B730B84
:10074000840B950B685873418040904050F00E9494
:100750000EAA6093DA117093DB118093DC119093F1
:10076000DD111F910F91FF90EF90DF90CF90BF9020
:10077000AF909F908F907F906F905F904F903F9041
:100780002F9008952F923F924F925F926F927F9297
:100790008F929F92AF92BF92CF92DF92EF92FF9291
:1007A0000F931F93DF93CF93CDB7DEB7E6970FB6C6
:1007B000F894DEBF0FBECDBF6C8F7D8F8E8F9F8F65
:1007C0005EAB4DAB39A328A30E940EAA698B7A8B2E
:1007D0008B8B9C8B2DA93EA9223031051CF4EDE1B9
:1007E000F3E019C0E0E3F3E007C08091C00085FFAB
:1007F000FCCF31969093C60090819923B1F78091F8
:10080000C00085FFFCCF30C48091C00085FFFCCFC5
:1008100031969093C60090819923B1F78091C000E2
:1008200085FFFCCF8AE08093C60036DA4DA95EA929
:1008300057FF74C08FE780939F1189899A89AB898C
:10084000BC898D879E87AF87B88B89879A87AB874E
:10085000BC8719AA1AAA1BAA1CAA1F8A1E8A91E081
:100860009D8B1D821E821F8218867FE7A72EB12CCA
:10087000C12CD12C6FE7262E312C412C512C20E09D
:1008800030E040E050E029833A834B835C830F2EB5
:10089000F0E06F2EF0E47F2EFCE18F2EF6E49F2E29
:1008A000F02D4DA95EA942565E4E5BA34AA3E0E03F
:1008B000F5E154915CA3EBEFF4E184918DA3E4EFB7
:1008C000F4E194919EA3EDEEF4E1A491AFA3E7EEE1
:1008D000F4E1B491B8A7E1EEF4E1249129A7E4EDA5
:1008E000F4E134913AA7EEECF4E144914BA7E8EC43
:1008F000F4E154915CA7E2ECF4E184918DA7ADA9F9
:10090000BEA9AA0FBB1FAA0FBB1FAC56BE4EBFA7E6
:10091000AEA7E8E8F4E1B491B8AB07C0EDA9FEA931
:10092000E256FE4E8FE7808388CF8091A011882306
:1009300009F4C0C2809192119091931160E0B6DBEE
:1009400060939411709395118093961190939711E1
:1009500080E090E0A0E0B0E080939A1190939B112A
:10096000A0939C11B0939D118FB7F8941092A01191
:100970008FBFEDA9FEA9F7FF0DC0F0919A11F9AB59
:1009800020919B112AAB30919C113BAB40919D1162
:100990004CAB11C0AEA5BFA5BC91B9ABEEA5FFA5F0
:1009A000F181FAABAEA5BFA51296BC91BBABEEA58B
:1009B000FFA5F381FCAB69817A818B819C8129A998
:1009C0003AA94BA95CA90E947FB3181644F089A9E3
:1009D0009AA9ABA9BCA989839A83AB83BC83C401C0
:1009E000B30129A93AA94BA95CA90E9471B187FD5D
:1009F00006C089A99AA9ABA9BCA93C014D012D89C2
:100A0000222309F451C069A97AA98BA99CA92C8D2C
:100A10003D8D4E8D5F8D0E947FB318160CF04AC23B
:100A20000E940EAA29853A854B855C85621B730B53
:100A3000840B950B695873418040904008F43AC28A
:100A4000D601C50182199309A409B5094DA95EA96A
:100A500057FF07C0B595A7959795879580939F11E8
:100A600007C0B595A79597958795EAA1FBA18083C7
:100A70000E940EAA6D877E878F87988B9B01AC01A1
:100A800089859A85AB85BC85281B390B4A0B5B0B86
:100A90002D833E834F8358872C8D3D8D4E8D5F8DEA
:100AA00029833A834B835C8369A97AA98BA99CA982
:100AB0002C8D3D8D4E8D5F8D0E9471B188230CF081
:100AC000F8C10E940EAA2D853E854F855889621B6C
:100AD000730B840B950B695873418040904008F468
:100AE000E8C10E940EAA69877A878B879C874E8906
:100AF0005F89452B09F4B8C1DC01CB012D853E850A
:100B00004F855889821B930BA40BB50B2D813E8119
:100B10004F815885280F391F4A1F5B1F288F398F37
:100B20004A8F5B8F2D813E814F815885281B390B61
:100B30004A0B5B0BCA01B901A20191010E9423B5C6
:100B4000288D398D4A8D5B8D0E948BB52A0D3B1DFA
:100B50004C1D5D1D24313105410551055CF424E136
:100B6000222E312C412C512C94E1A92EB12CC12CD8
:100B7000D12C1FC059016A013CEEA316B104C10477
:100B8000D1042CF08BEEA82EB12CC12CD12C40E836
:100B9000A416B104C104D1041CF41501260109C036
:100BA0000EEF202E312C412C512C2A183B084C08DA
:100BB0005D089CA1E0E0F5E108C08091C00085FFE0
:100BC000FCCF9093C600319694919923B1F786E4B7
:100BD00095E0B601A5012AE030E00E94C5269DA15E
:100BE000EBEFF4E108C08091C00085FFFCCF90934B
:100BF000C600319694919923B1F786E495E0B2014D
:100C0000A1012AE030E00E94C5269EA1E4EFF4E1B4
:100C100008C08091C00085FFFCCF9093C60031963C
:100C200094919923B1F786E495E0B401A30122E001
:100C300030E00E94CB279FA1EDEEF4E108C0809147
:100C4000C00085FFFCCF9093C60031969491992304
:100C5000B1F786E495E049815A816B817C8122E07D
:100C600030E00E94CB278091C00085FFFCCF8AE056
:100C70008093C6008E899F8903970CF4F5C0C2014A
:100C8000B1010E9413B220E030E040E850E40E943D
:100C900051B47B018C0169817A818B819C81A40193
:100CA00093010E9497B020ED3FE049E450E40E9498
:100CB00051B420E030E040E05FE30E9451B49B017A
:100CC000AC01C801B7010E9478B17B018C01688D2D
:100CD000798D8A8D9B8D0E9413B220E030E04AE727
:100CE00054E40E9478B13B014C0198A5E7EEF4E191
:100CF00008C08091C00085FFFCCF9093C60031965C
:100D000094919923B1F786E495E0B801A70122E018
:100D100030E00E94CB2799A5E1EEF4E108C0809174
:100D2000C00085FFFCCF9093C60031969491992323
:100D3000B1F786E495E0B401A30122E030E00E941F
:100D4000CB278091C00085FFFCCF8AE08093C6004E
:100D5000C801B7012AE939E949E15FE30E9451B4CA
:100D60007B018C019AA5E4EDF4E108C08091C000FC
:100D700085FFFCCF9093C600319694919923B1F7EB
:100D80008091C00085FFFCCF8AE08093C6009BA5C0
:100D9000EEECF4E108C08091C00085FFFCCF909399
:100DA000C600319694919923B1F786E495E0B80195
:100DB000A70122E030E00E94CB278091C00085FF90
:100DC000FCCF8AE08093C6009CA5E8ECF4E108C063
:100DD0008091C00085FFFCCF9093C600319694911E
:100DE0009923B1F7C801B701A80197010E9498B0F3
:100DF000A40193010E9478B1AB01BC0186E495E0A7
:100E000022E030E00E94CB278091C00085FFFCCF1C
:100E10008AE08093C6009DA5E2ECF4E108C08091D1
:100E2000C00085FFFCCF9093C60031969491992322
:100E3000B1F7C801B701A40193010E9451B420E0A9
:100E400030E040E05EE30E9451B4AB01BC0186E4B7
:100E500095E022E030E00E94CB278091C00085FF22
:100E6000FCCF8AE08093C600D201C1018A0D9B1D90
:100E7000AC1DBD1DEDA9FEA9F7FF07C0B595A7954F
:100E80009795879580939F1107C0B595A7959795DE
:100E90008795EAA1FBA180832E893F892F5F3F4F71
:100EA0003F8B2E8B6C8C7D8C8E8C9F8C31E03D8BA0
:100EB00001C01D8A6C8D7D8D8E8D9F8D20E030E070
:100EC00040EA51E40E9498B09B01AC0169A97AA95B
:100ED0008BA99CA90E947FB318169CF4E8E9F4E161
:100EE000949108C08091C00085FFFCCF9093C6000C
:100EF000319694919923B1F78091C00085FFFCCF82
:100F0000B3C00E940EAA29893A894B895C89621B69
:100F1000730B840B950B615D77408040904008F423
:100F200054C04DA95EA957FF11C060919F11E2E91D
:100F3000F4E1949108C08091C00085FFFCCF9093AC
:100F4000C600319694919923B1F711C0AAA1BBA113
:100F50006C91ECE8F4E1949108C08091C00085FFA9
:100F6000FCCF9093C600319694919923B1F7162F38
:100F700086E495E049A95AA96BA97CA922E030E052
:100F80000E94CB2798A9E8E8F4E108C08091C0004E
:100F900085FFFCCF9093C600319694919923B1F7C9
:100FA00086E495E0612F70E04AE050E00E94F82668
:100FB0008091C00085FFFCCF8AE08093C6000E942C
:100FC0000EAA698B7A8B8B8B9C8B0E940EAA7B015D
:100FD0008C010E940EAA2D853E854F855889E21A04
:100FE000F30A040B150B29853A854B855C85E21ABB
:100FF000F30A040B150BE60EF71E081F191F31E844
:10100000E3163FE4F30632E1030730E0130798F0FC
:10101000EBE6F4E1949108C08091C00085FFFCCF1D
:101020009093C600319694919923B1F78091C000B6
:1010300085FFFCCF19C04E895F8988A199A18417CB
:10104000950774F5EFE1F4E1949108C08091C00038
:1010500085FFFCCF9093C600319694919923B1F708
:101060008091C00085FFFCCF8AE08093C600E696A1
:101070000FB6F894DEBF0FBECDBFCF91DF911F91A9
:101080000F91FF90EF90DF90CF90BF90AF909F9027
:101090008F907F906F905F904F903F902F9008952A
:1010A0000E94C19E42CC9093031280930212089535
:1010B0008093041208951092EB1108958091051207
:1010C00090E0969587959695879581700895FC0197
:1010D0002081822F90E06AE070E00E9456B5CB013B
:1010E0006AE070E00E9456B5805D80931A12822FEC
:1010F00090E06AE070E00E9456B5805D80931B121C
:1011000010921C128AE192E10895FC0160817181C4
:101110008281938120E030E040E251E40E9451B4AA
:101120000E94E0B19B0177FF02C08DE201C08BE21B
:1011300080931A1237FF03C0309521953F4FC901A4
:1011400068EE73E00E9456B5CB016AE070E00E9441
:1011500056B5805D80931B12C90164E670E00E9461
:1011600056B5CB016AE070E00E9456B5805D809371
:101170001C12C9016AE070E00E9456B5CB016AE01A
:1011800070E00E9456B5805D80931D128EE28093C0
:101190001E12C9016AE070E00E9456B5805D80931E
:1011A0001F12109220128AE192E10895EF92FF92AD
:1011B0000F931F93FC01608171818281938120E0F4
:1011C00030E048EC52E40E9451B40E94E0B17B014F
:1011D0008C0197FD12C020E137E240E050E00E9410
:1011E0008BB5CA01B9012AE030E040E050E00E942E
:1011F0008BB5605D60931A1203C08DE280931A1262
:1012000017FF08C010950095F094E094E11CF11CC4
:10121000011D111DC801B70128EE33E040E050E088
:101220000E948BB5CA01B9012AE030E040E050E0ED
:101230000E948BB5605D60931B12C801B70124E664
:1012400030E040E050E00E948BB5CA01B9012AE0CD
:1012500030E040E050E00E948BB5605D60931C126E
:101260008EE280931D12C801B7012AE030E040E011
:1012700050E00E948BB5CA01B9012AE030E040E09D
:1012800050E00E948BB5605D60931E12C801B701EB
:101290002AE030E040E050E00E948BB5605D609352
:1012A0001F12109220128AE192E11F910F91FF907C
:1012B000EF900895FC0180819181843691055CF066
:1012C00064E670E00E9456B5CB016AE070E00E94CF
:1012D00056B5805D01C080E280931A1280819181B1
:1012E0008A3091055CF06AE070E00E9456B5CB014F
:1012F0006AE070E00E9456B5805D01C080E2809394
:101300001B12808191816AE070E00E9456B5805D79
:1013100080931C1210921D128AE192E10895DF93CE
:10132000CF930F920F92CDB7DEB7FC016081718130
:10133000828193810E94E0B17A836983CE01019614
:10134000B9DF0F900F90CF91DF910895FC0180815C
:1013500091818436910534F164E670E00E9456B5BF
:10136000CB016AE070E00E9456B5805D80931A124E
:10137000808191816AE070E00E9456B5CB016AE0FD
:1013800070E00E9456B5805D80931B128081918130
:101390006AE070E00E9456B5805D80931C12109246
:1013A0001D1224C08A309105C4F06AE070E00E94EA
:1013B00056B5CB016AE070E00E9456B5805D80931F
:1013C0001A12808191816AE070E00E9456B5805DBA
:1013D00080931B1210921C1209C06AE070E00E94F8
:1013E00056B5805D80931A1210921B128AE192E129
:1013F00008950F931F93CF93DF93382FEB01142F92
:10140000022F8CEE91E160E0432F0E94BDA88CEE8C
:1014100091E1612F0E94DCAC11E1FE016491662331
:1014200079F0112369F08CEE91E10E94DCAC2196F9
:101430001150F3CF8CEE91E160E20E94DCAC1150D0
:101440001123C1F78CEE91E1602F0E94DCAC8CEE91
:1014500091E160E20E94DCACDF91CF911F910F918E
:1014600008950F93DF93CF9300D00F92CDB7DEB7DF
:1014700006B1029506950695037000950170349BA0
:101480000260209107123091081240910912509188
:101490000A1229833A834B835C830E940EAA298116
:1014A0003A814B815C81261737074807590710F4AA
:1014B000329B046000930512909105129170809107
:1014C000051281FD926080910B12981729F19130DD
:1014D000B1F0913028F0923041F09330E9F40AC035
:1014E000813079F08230C1F412C0882351F083300A
:1014F00099F40DC0823029F0813071F408C0833036
:1015000021F48091DE118F5F05C0882329F480913A
:10151000DE1181508093DE1190930B120F900F908B
:101520000F900F90CF91DF910F910895CF93DF939C
:10153000EC0104C08CEE91E10E9487A8FE01219687
:1015400064916623B9F7DF91CF910895EF92FF92EE
:101550000F931F93DF93CF93CDB7DEB728970FB6C6
:10156000F894DEBF0FBECDBF6091941170919511BC
:10157000809196119091971120E030E040E05FE378
:101580000E9498B00E94E0B17C836B8360918E11C1
:1015900070918F11882777FD8095982F0E9413B244
:1015A00020E030E040E05FE30E9498B00E94E0B1AC
:1015B0007E836D838CEE91E160E040E00E94BDA8E7
:1015C0008CEE91E162E00E94DCACCE01039672DE0B
:1015D000BC018CEE91E10E9400AD8CEE91E16FE2D6
:1015E0000E94DCACCE010596B1DEBC018CEE91E12F
:1015F0000E9400AD8CE096E199DF8D819E810A9773
:101600002CF48CEE91E160E20E94DCAC8CEE91E176
:1016100060E041E00E94BDA88CEE91E168E50E9487
:10162000DCAC8BED97E07BDEBC018CEE91E10E949F
:1016300000AD89E096E17ADF8FED97E070DEBC01C6
:101640008CEE91E10E9400AD8CEE91E16CE041E006
:101650000E94BDA88CEE91E16AE50E94DCAC83EEAD
:1016600097E0A4DDBC018CEE91E10E9400AD8CEE10
:1016700091E160E042E00E94BDA88CEE91E166E05D
:101680000E94DCAC8CE893E015DEBC018CEE91E1AD
:101690000E9400AD8CEE91E165E20E94DCAC8CEE24
:1016A00091E167E042E00E94BDA886E096E13EDF5E
:1016B00080914905882391F180911807882311F1C1
:1016C0006091C2077091C3078091C4079091C507CC
:1016D0006115710581059105A9F06D597F4F8F4FF7
:1016E0009F4F24E630E040E050E00E9469B56091F1
:1016F000CA077091CB078091CC079091CD070E94CB
:1017000069B501C020E02F831886CE010796D2DD8F
:10171000BC018CEE91E10E9400AD03C082E096E135
:1017200005DF8CEE91E165E20E94DCAC8CEE91E18C
:101730006EE042E00E94BDA88CEE91E167E00E945D
:10174000DCAC8091060890910708A0910808B09140
:1017500009080097A105B105E1F10E940EAA20E653
:101760003AEE40E050E00E9469B579018A0160914B
:10177000060870910708809108089091090820E6F2
:101780003AEE40E050E00E9469B5E21AF30AC70160
:101790006CE370E00E9442B56983CE01019697DC4C
:1017A000BC018CEE91E10E9400AD8CEE91E16AE308
:1017B0000E94DCACC7016CE370E00E9442B58A83F2
:1017C000CE01029684DCBC018CEE91E10E9400AD5A
:1017D00003C08CEF95E1AADE8CEE91E160E043E07E
:1017E0000E94BDA88CEE91E161ED73E00E9400AD16
:1017F00028960FB6F894DEBF0FBECDBFCF91DF9114
:101800001F910F91FF90EF9008951F9382E08093B6
:10181000E8030E940EAA6C507E4F8F4F9F4F60933B
:101820000712709308128093091290930A12389A43
:1018300010E0409A84E690E00E9475AA409884E601
:1018400090E00E9475AA1F5F1A3099F71F910895C2
:1018500080911512882321F081508093151203C0C6
:1018600081E08093E8038091E803882321F06EDE15
:101870008AE0809315128091051282FF0FC08FEFCE
:1018800099E99093E7038093E60310920C1210926B
:101890000D1210920E1210920F12B7CF0895AF9240
:1018A000BF92CF92DF92EF92FF920F931F9380919E
:1018B0000C1290910D12A0910E12B0910F12815046
:1018C0009048A040B04040F010920C1210920D12BF
:1018D00010920E1210920F1260910C1270910D1254
:1018E00080910E1290910F1225E030E040E050E020
:1018F0000E9469B579018A018091061290E0A0E00A
:10190000B0E0E816F9060A071B0710F42093061248
:10191000009106128091051290E096958795969514
:101920008795FF24F394F82210E033E1A32EB12C25
:10193000C12CD12CEE24E394002379F58091E803A7
:101940008823B9F080910C1290910D12A0910E1283
:10195000B0910F120597A105B10528F4812F65EE0E
:1019600076E143E004C0812F65EE76E140E223E0BA
:1019700040DDFF2009F4DBC080910C1290910D1224
:10198000A0910E12B0910F120597A105B10508F0B4
:10199000CEC03BDF8DE990E9BDC0013009F03DC00C
:1019A0008091E8038823F1F060910C1270910D1280
:1019B00080910E1290910F1225E030E040E050E04F
:1019C0000E9469B5213031054105510529F4812F67
:1019D0006BED76E14EE304C0812F6BED76E140E2E2
:1019E0002EE707DDFF2009F4A2C060910C12709170
:1019F0000D1280910E1290910F1225E030E040E020
:101A000050E00E9469B5213031054105510509F0CA
:101A10008EC0FBDE85EA96E97DC0023009F03DC04C
:101A20008091E8038823F1F060910C1270910D12FF
:101A300080910E1290910F1225E030E040E050E0CE
:101A40000E9469B5223031054105510529F4812FE5
:101A500062ED76E14EE304C0812F62ED76E140E273
:101A60002EE7C7DCFF2009F462C060910C12709170
:101A70000D1280910E1290910F1225E030E040E09F
:101A800050E00E9469B5223031054105510509F049
:101A90004EC0BBDE88E996E93DC0033009F047C07F
:101AA0008091E8038823F1F060910C1270910D127F
:101AB00080910E1290910F1225E030E040E050E04E
:101AC0000E9469B5233031054105510529F4812F64
:101AD00067EC76E14EE304C0812F67EC76E140E2EB
:101AE0002EE787DCFF2019F160910C1270910D1226
:101AF00080910E1290910F1225E030E040E050E00E
:101B00000E9469B5233031054105510581F47DDE20
:101B10008BE896E99093E7038093E60310920C120A
:101B200010920D1210920E1210920F1238C0809166
:101B30000C1290910D12A0910E12B0910F124497B9
:101B4000A105B10540F0A0920C12B0920D12C09206
:101B50000E12D0920F1260910C1270910D128091A2
:101B60000E1290910F1225E030E040E050E00E940C
:101B700069B5422F8091061290E0039630E08217FB
:101B8000930744F4435040930612E092E803042F75
:101B900001501FEF1F5F143010F40F5FCDCE1F9167
:101BA0000F91FF90EF90DF90CF90BF90AF9008958E
:101BB000AF92BF92CF92DF92EF92FF920F931F935B
:101BC00080910C1290910D12A0910E12B0910F12F3
:101BD00081509048A040B04040F010920C121092FA
:101BE0000D1210920E1210920F1260910C12709141
:101BF0000D1280910E1290910F1225E030E040E01E
:101C000050E00E9469B579018A018091061290E046
